** EXPERIMENTAL (HLL) ** Open Watcom Linker Version 1.6beta1 Limited Availability
Portions Copyright (c) 1985-2002 Sybase, Inc. All Rights Reserved.
Created on:       12/01/07 19:00:19
Warning! W1121: file U:/tmp\ldconv__ssl_obj_ddb24f08029a193378.obj(U:\DEV\python-2.7.2\Modules\_ssl.c): '_init_ssl' has already been exported
Executable Image: build/lib.os2knix-2.7/_ssl.pyd
creating an OS/2 EMX dynamic link library


                        +------------+
                        |   Groups   |
                        +------------+

Group                           Address              Size
=====                           =======              ====

CGROUP                          0001:00000000        00140300
DGROUP                          0002:00000000        00009b90



                        +--------------+
                        |   Segments   |
                        +--------------+

Segment                Class          Group          Address         Size
=======                =====          =====          =======         ====

TEXT32                 CODE           CGROUP         0001:00000000   001402f8
________TEXT           CODE           CGROUP         0001:00140300   00000000
DATA32                 DATA           DGROUP         0002:00000000   00007530
SET1__os2dll           DATA           DGROUP         0002:00007530   00000004
SET2__os2dll           DATA           DGROUP         0002:00007534   00000000
SET3__os2dll           DATA           DGROUP         0002:00007534   00000004
SET1___CTOR_LIST__     DATA           DGROUP         0002:00007538   00000004
SET2___CTOR_LIST__     DATA           DGROUP         0002:0000753c   00000000
SET3___CTOR_LIST__     DATA           DGROUP         0002:0000753c   00000004
SET1___DTOR_LIST__     DATA           DGROUP         0002:00007540   00000004
SET2___DTOR_LIST__     DATA           DGROUP         0002:00007544   00000000
SET3___DTOR_LIST__     DATA           DGROUP         0002:00007544   00000004
SET1___crtinit1__      DATA           DGROUP         0002:00007548   00000004
SET2___crtinit1__      DATA           DGROUP         0002:0000754c   00000000
SET3___crtinit1__      DATA           DGROUP         0002:0000754c   00000004
SET1___crtexit1__      DATA           DGROUP         0002:00007550   00000004
SET2___crtexit1__      DATA           DGROUP         0002:00007554   00000000
SET3___crtexit1__      DATA           DGROUP         0002:00007554   00000004
SET1___eh_frame__      DATA           DGROUP         0002:00007558   00000004
SET2___eh_frame__      DATA           DGROUP         0002:0000755c   00000008
SET3___eh_frame__      DATA           DGROUP         0002:00007564   00000004
SET1___eh_init__       DATA           DGROUP         0002:00007568   00000004
SET2___eh_init__       DATA           DGROUP         0002:0000756c   00000004
SET3___eh_init__       DATA           DGROUP         0002:00007570   00000004
SET1___eh_term__       DATA           DGROUP         0002:00007574   00000004
SET2___eh_term__       DATA           DGROUP         0002:00007578   00000004
SET3___eh_term__       DATA           DGROUP         0002:0000757c   00000004
SET1___fork_parent1__  DATA           DGROUP         0002:00007580   00000004
SET2___fork_parent1__  DATA           DGROUP         0002:00007584   00000000
SET3___fork_parent1__  DATA           DGROUP         0002:00007584   00000004
SET1___fork_child1__   DATA           DGROUP         0002:00007588   00000004
SET2___fork_child1__   DATA           DGROUP         0002:0000758c   00000000
SET3___fork_child1__   DATA           DGROUP         0002:0000758c   00000004
________DATA           DATA           DGROUP         0002:00007590   00000000
BSS32                  BSS            DGROUP         0002:00007590   000025e0
c_common               BSS            DGROUP         0002:00009b70   00000020
________BSS            BSS            DGROUP         0002:00009b90   00000000


                        +----------------+
                        |   Memory Map   |
                        +----------------+

* = unreferenced symbol
+ = symbol only referenced locally

Address        Symbol
=======        ======

Module: U:\usr\lib\dll0hi.obj({standard input})
0001:00000000* __text
0002:00000000* __data
0002:00000000* ___data_start
0002:00007590* ___bss_start
0002:00007530+ __os2dll
0002:00007538  ___CTOR_LIST__
0002:00007540  ___DTOR_LIST__
0002:00007548* ___crtinit1__
0002:00007550* ___crtexit1__
0002:00007558  ___eh_frame__
0002:00007568  ___eh_init__
0002:00007574  ___eh_term__
0002:00007580+ ___fork_parent1__
0002:00007588+ ___fork_child1__
Module: U:/tmp\ldconv__ssl_obj_ddb24f08029a193378.obj(U:\DEV\python-2.7.2\Modules\_ssl.c)
0001:0000158b  _init_ssl
Module: U:\usr\local446\lib\libc_dll.lib(dllinit.obj)
0001:00003240  _DLL_InitTerm
Module: U:\usr\lib\libend.lib(src/libend/386/endlink386.asm)
0002:00009b90  _end
0002:00007590  _edata
Module: U:\usr\lib\libend.lib(src/libend/386/end.asm)
0001:00140300* _etext
0001:00140300* __etext
0000:00000000  WEAK$ZERO
0002:00009b90  __end
0002:00007590  __edata
Module: U:\extras\lib\libcrypto.lib(rand_lib.obj)
0001:000032a0  _RAND_set_rand_method
0001:000032d5* _RAND_get_rand_method
0001:0000333e* _RAND_set_rand_engine
0001:000033a7* _RAND_cleanup
0001:000033db  _RAND_seed
0001:0000340e  _RAND_add
0001:0000345d  _RAND_bytes
0001:00003499  _RAND_pseudo_bytes
0001:000034d5  _RAND_status
Module: U:\extras\lib\libcrypto.lib(rand_egd.obj)
0001:00003510* _RAND_query_egd_bytes
0001:00003824* _RAND_egd_bytes
0001:0000386c  _RAND_egd
Module: U:\extras\lib\libssl.lib(ssl_lib.obj)
0001:00007b2b  _ssl_undefined_function
0001:000038b4  _SSL_clear
0001:00008118* _ssl_clear_cipher_ctx
0001:00008ae5* _ssl_clear_hash_ctx
0001:00003ad8* _SSL_CTX_set_ssl_version
0001:00003b9f  _SSL_new
0001:00006921  _SSL_CTX_free
0001:00004016* _SSL_CTX_set_session_id_context
0001:00004087* _SSL_set_session_id_context
0001:000040f8* _SSL_CTX_set_generate_session_id
0001:00004159* _SSL_set_generate_session_id
0001:000041ba  _SSL_has_matching_session_id
0001:000042c0* _SSL_CTX_set_purpose
0001:000042e0* _SSL_set_purpose
0001:000042fd* _SSL_CTX_set_trust
0001:0000431d* _SSL_set_trust
0001:0000433a* _SSL_CTX_set1_param
0001:0000435a* _SSL_set1_param
0001:00004377  _SSL_free
0001:000046b0* _SSL_set_bio
0001:00004756  _SSL_get_rbio
0001:00004761  _SSL_get_wbio
0001:0000476c* _SSL_get_fd
0001:0000477f* _SSL_get_rfd
0001:000047dd* _SSL_get_wfd
0001:0000483b  _SSL_set_fd
0001:000048da* _SSL_set_wfd
0001:00004a01* _SSL_set_rfd
0001:00004b28* _SSL_get_finished
0001:00004b83* _SSL_get_peer_finished
0001:00004bde* _SSL_get_verify_mode
0001:00004bec* _SSL_get_verify_depth
0001:00004c02* _SSL_get_verify_callback
0001:00004c10  _SSL_CTX_get_verify_mode
0001:00004c1e* _SSL_CTX_get_verify_depth
0001:00004c37* _SSL_CTX_get_verify_callback
0001:00004c45* _SSL_set_verify
0001:00004c68* _SSL_set_verify_depth
0001:00004c85  _SSL_set_read_ahead
0001:00004c93* _SSL_get_read_ahead
0001:00004c9e  _SSL_pending
0001:00004cb7  _SSL_get_peer_certificate
0001:00004d29* _SSL_get_peer_cert_chain
0001:00004d77* _SSL_copy_session_id
0001:00004e7b* _SSL_CTX_check_private_key
0001:00004f46* _SSL_check_private_key
0001:0000507d  _SSL_accept
0001:00007a6b  _SSL_set_accept_state
0001:000050ab  _SSL_connect
0001:00007acb  _SSL_set_connect_state
0001:000050d9  _SSL_get_default_timeout
0001:000050ec  _SSL_read
0001:0000516e  _SSL_peek
0001:000051e6  _SSL_write
0001:00005294  _SSL_shutdown
0001:000085d6  _SSL_state
0001:0000530b* _SSL_renegotiate
0001:00005338* _SSL_renegotiate_pending
0001:0000534b  _SSL_ctrl
0001:00008496  _SSL_version
0001:00005618* _SSL_callback_ctrl
0001:00005657* _SSL_CTX_sessions
0001:00005662  _SSL_CTX_ctrl
0001:000059a9* _SSL_CTX_callback_ctrl
0001:000059ea* _ssl_cipher_id_cmp
0001:00005a26  _ssl_cipher_ptr_id_cmp
0001:00005a66  _SSL_get_ciphers
0001:00005ab3  _ssl_get_ciphers_by_id
0001:00005b00* _SSL_get_cipher_list
0001:00005b68  _SSL_CTX_set_cipher_list
0001:00005bf4* _SSL_set_cipher_list
0001:00005c86* _SSL_get_shared_ciphers
0001:00005d71  _ssl_cipher_list_to_bytes
0001:00005e92  _ssl_bytes_to_cipher_list
0001:0000609f* _SSL_get_servername
0001:000060e5* _SSL_get_servername_type
0001:0000622a  _SSL_CTX_new
0001:00006b28* _SSL_CTX_set_default_passwd_cb
0001:00006b36* _SSL_CTX_set_default_passwd_cb_userdata
0001:00006b44* _SSL_CTX_set_cert_verify_callback
0001:00006b5b  _SSL_CTX_set_verify
0001:00006b78* _SSL_CTX_set_verify_depth
0001:00006ba8  _ssl_set_cert_masks
0001:00007100  _ssl_check_srvr_ecc_cert_and_alg
0001:0000734d  _ssl_get_server_send_cert
0001:000074c8  _ssl_get_sign_pkey
0001:00007586  _ssl_update_cache
0001:000076f8* _SSL_get_ssl_method
0001:00007703  _SSL_set_ssl_method
0001:000077bf  _SSL_get_error
0001:0000873a* _SSL_want
0001:000079d2  _SSL_do_handshake
0001:00007b64  _ssl_undefined_void_function
0001:00007b9d  _ssl_undefined_const_function
0001:00007bd6* _ssl_bad_method
0001:00007c1b* _SSL_get_version
0001:00007c5c* _SSL_dup
0001:000084a0* _SSL_get_SSL_CTX
0001:000085c8* _SSL_get_info_callback
0001:000085b7* _SSL_set_info_callback
0001:000081ee* _SSL_get_certificate
0001:00008214* _SSL_get_privatekey
0001:0000823b  _SSL_get_current_cipher
0001:00008276* _SSL_get_current_compression
0001:0000829a* _SSL_get_current_expansion
0001:000082be  _ssl_init_wbio_buffer
0001:000083f4  _ssl_free_wbio_buffer
0001:00008445* _SSL_CTX_set_quiet_shutdown
0001:00008456* _SSL_CTX_get_quiet_shutdown
0001:00008464* _SSL_set_quiet_shutdown
0001:00008472* _SSL_get_quiet_shutdown
0001:0000847d* _SSL_set_shutdown
0001:0000848b  _SSL_get_shutdown
0001:000084ae* _SSL_set_SSL_CTX
0001:0000857d* _SSL_CTX_set_default_verify_paths
0001:00008593  _SSL_CTX_load_verify_locations
0001:000085e1* _SSL_set_verify_result
0001:000085f2* _SSL_get_verify_result
0001:00008600* _SSL_get_ex_new_index
0001:00008637* _SSL_set_ex_data
0001:0000865e* _SSL_get_ex_data
0001:0000867e* _SSL_CTX_get_ex_new_index
0001:000086b5* _SSL_CTX_set_ex_data
0001:000086dc* _SSL_CTX_get_ex_data
0001:000086fc  _ssl_ok
0001:00008706* _SSL_CTX_get_cert_store
0001:00008711* _SSL_CTX_set_cert_store
0001:00008745* _SSL_CTX_set_tmp_rsa_callback
0001:00008767* _SSL_set_tmp_rsa_callback
0001:00008789* _SSL_CTX_set_tmp_dh_callback
0001:000087ab* _SSL_set_tmp_dh_callback
0001:000087cd* _SSL_CTX_set_tmp_ecdh_callback
0001:000087ef* _SSL_set_tmp_ecdh_callback
0001:00008811* _SSL_CTX_use_psk_identity_hint
0001:000088c2* _SSL_use_psk_identity_hint
0001:000089bd* _SSL_get_psk_identity_hint
0001:000089eb* _SSL_get_psk_identity
0001:00008a19* _SSL_set_psk_client_callback
0001:00008a2a* _SSL_CTX_set_psk_client_callback
0001:00008a3b* _SSL_set_psk_server_callback
0001:00008a4c* _SSL_CTX_set_psk_server_callback
0001:00008a5d* _SSL_CTX_set_msg_callback
0001:00008a7f* _SSL_set_msg_callback
0001:00008aa1  _ssl_replace_hash
0001:00008b32  _OBJ_bsearch_ssl_cipher_id
0002:000008f0* _SSL_version_str
0002:00000900  _ssl3_undef_enc_method
Module: U:\extras\lib\libcrypto.lib(err.obj)
0001:00009061* _ERR_get_implementation
0001:00009073* _ERR_set_implementation
0001:00009ac6  _ERR_load_ERR_strings
0001:00009b6d  _ERR_load_strings
0001:00009b8c* _ERR_unload_strings
0001:00009bd1* _ERR_free_strings
0001:00009be8  _ERR_put_error
0001:0000a653  _ERR_get_state
0001:00009d45  _ERR_clear_error
0001:00009e2a  _ERR_get_error
0001:00009e66* _ERR_get_error_line
0001:00009ea0  _ERR_get_error_line_data
0001:00009ed8  _ERR_peek_error
0001:00009f14* _ERR_peek_error_line
0001:00009f4e* _ERR_peek_error_line_data
0001:00009f86  _ERR_peek_last_error
0001:00009fc2* _ERR_peek_last_error_line
0001:00009ffc* _ERR_peek_last_error_line_data
0001:0000a27e  _ERR_error_string_n
0001:0000a4b4* _ERR_lib_error_string
0001:0000a4fe  _ERR_func_error_string
0001:0000a565* _ERR_reason_error_string
0001:0000a42a  _ERR_error_string
0001:0000a45c* _ERR_get_string_table
0001:0000a479* _ERR_get_err_state_table
0001:0000a497* _ERR_release_err_state_table
0001:0000a5f1* _ERR_remove_thread_state
0001:0000a63f* _ERR_remove_state
0001:0000a790* _ERR_get_next_error_library
0001:0000a7a7* _ERR_set_error_data
0001:0000a84c  _ERR_add_error_data
0001:0000a959  _ERR_set_mark
0001:0000a9b0  _ERR_pop_to_mark
Module: U:\extras\lib\libcrypto.lib(bio_lib.obj)
0001:0000ab4a  _BIO_new
0001:0000abdc  _BIO_set
0001:0000acd0  _BIO_free
0001:0000add0  _BIO_vfree
0001:0000ade3  _BIO_clear_flags
0001:0000adfb  _BIO_test_flags
0001:0000ae09  _BIO_set_flags
0001:0000ae1f* _BIO_get_callback
0001:0000ae2a* _BIO_set_callback
0001:0000ae38* _BIO_set_callback_arg
0001:0000ae46* _BIO_get_callback_arg
0001:0000ae51* _BIO_method_name
0001:0000ae5e  _BIO_method_type
0001:0000ae6a  _BIO_read
0001:0000afc5  _BIO_write
0001:0000b12a  _BIO_puts
0001:0000b280  _BIO_gets
0001:0000b3c6  _BIO_indent
0001:0000b41e  _BIO_int_ctrl
0001:0000b489  _BIO_ctrl
0001:0000b44c* _BIO_ptr_ctrl
0001:0000b59c  _BIO_callback_ctrl
0001:0000b6aa* _BIO_ctrl_pending
0001:0000b6d5* _BIO_ctrl_wpending
0001:0000b700  _BIO_push
0001:0000b76b  _BIO_pop
0001:0000b7f4* _BIO_get_retry_BIO
0001:0000b84e  _BIO_get_retry_reason
0001:0000b859  _BIO_find_type
0001:0000b8c4  _BIO_next
0001:0000b8dc  _BIO_free_all
0001:0000b918* _BIO_dup_chain
0001:0000ba50  _BIO_copy_next_retry
0001:0000ba8c* _BIO_get_ex_new_index
0001:0000bac3* _BIO_set_ex_data
0001:0000bae7* _BIO_get_ex_data
0001:0000bb04* _BIO_number_read
0001:0000bb1c* _BIO_number_written
Module: U:\extras\lib\libssl.lib(ssl_ciph.obj)
0001:0000cb01  _ssl_load_ciphers
0001:0000ce98  _ssl_cipher_get_evp
0001:0000d146  _ssl_get_handshake_digest
0001:0000e329  _ssl_create_cipher_list
0001:0000ec2e* _SSL_CIPHER_description
0001:0000f0c4  _SSL_CIPHER_get_version
0001:0000f104  _SSL_CIPHER_get_name
0001:0000f11c  _SSL_CIPHER_get_bits
0001:0000f14e  _ssl3_comp_find
0001:0000f1b4  _SSL_COMP_get_compression_methods
0001:0000f1c6* _SSL_COMP_add_compression_method
0001:0000f357* _SSL_COMP_get_name
Module: U:\extras\lib\libcrypto.lib(x_x509.obj)
0001:0000f500  _X509_CINF_it
0001:0000f51c* _d2i_X509_CINF
0001:0000f545* _i2d_X509_CINF
0001:0000f567* _X509_CINF_new
0001:0000f57b* _X509_CINF_free
0001:0000f7a0  _X509_it
0001:0000f7bc  _d2i_X509
0001:0000f7e5  _i2d_X509
0001:0000f807* _X509_new
0001:0000f81b  _X509_free
0001:0000f836* _X509_dup
0001:0000f851* _X509_get_ex_new_index
0001:0000f888* _X509_set_ex_data
0001:0000f8ac* _X509_get_ex_data
0001:0000f8c9  _d2i_X509_AUX
0001:0000f954  _i2d_X509_AUX
Module: U:\extras\lib\libcrypto.lib(x509_cmp.obj)
0001:0000f9a0* _X509_issuer_and_serial_cmp
0001:0000fc76  _X509_NAME_cmp
0001:0000f9f6* _X509_issuer_and_serial_hash
0001:0000fafd* _X509_issuer_name_cmp
0001:0000fb21  _X509_subject_name_cmp
0001:0000fb45  _X509_CRL_cmp
0001:0000fb69  _X509_CRL_match
0001:0000fb91  _X509_get_issuer_name
0001:0000fb9e* _X509_issuer_name_hash
0001:0000fd30  _X509_NAME_hash
0001:0000fbb6* _X509_issuer_name_hash_old
0001:0000fdb9* _X509_NAME_hash_old
0001:0000fbce  _X509_get_subject_name
0001:0000fbdb  _X509_get_serialNumber
0001:0000fbe8* _X509_subject_name_hash
0001:0000fc00* _X509_subject_name_hash_old
0001:0000fc18  _X509_cmp
0001:0000fe45  _X509_find_by_issuer_and_serial
0001:0000fecd* _X509_find_by_subject
0001:0000ff2e  _X509_get_pubkey
0001:0000ff5c  _X509_get0_pubkey_bitstr
0001:0000ff84  _X509_check_private_key
Module: U:\extras\lib\libcrypto.lib(x509_obj.obj)
0001:000100a8  _X509_NAME_oneline
Module: U:\extras\lib\libssl.lib(ssl_err2.obj)
0001:000104f0  _SSL_load_error_strings
Module: U:\extras\lib\libssl.lib(ssl_algs.obj)
0001:00010569  _SSL_library_init
Module: U:\extras\lib\libcrypto.lib(c_all.obj)
0001:00010750  _OPENSSL_add_all_algorithms_noconf
Module: U:\extras\lib\libcrypto.lib(cryptlib.obj)
0001:0001095f* _CRYPTO_get_new_lockid
0001:00010a2e  _CRYPTO_num_locks
0001:00010a38* _CRYPTO_get_new_dynlockid
0001:000110fd  _CRYPTO_lock
0001:00010ced* _CRYPTO_destroy_dynlockid
0001:00010e2b* _CRYPTO_get_dynlock_value
0001:00010ee3* _CRYPTO_get_dynlock_create_callback
0001:00010eed* _CRYPTO_get_dynlock_lock_callback
0001:00010ef7* _CRYPTO_get_dynlock_destroy_callback
0001:00010f01* _CRYPTO_set_dynlock_create_callback
0001:00010f0e* _CRYPTO_set_dynlock_lock_callback
0001:00010f1b* _CRYPTO_set_dynlock_destroy_callback
0001:00010f28* _CRYPTO_get_locking_callback
0001:00010f32* _CRYPTO_get_add_lock_callback
0001:00010f3c  _CRYPTO_set_locking_callback
0001:00010f49* _CRYPTO_set_add_lock_callback
0001:00010f56* _CRYPTO_THREADID_set_numeric
0001:00010f8a* _CRYPTO_THREADID_set_pointer
0001:00010fd6* _CRYPTO_THREADID_set_callback
0001:00010ff8* _CRYPTO_THREADID_get_callback
0001:00011002  _CRYPTO_THREADID_current
0001:00011058  _CRYPTO_THREADID_cmp
0001:0001107a  _CRYPTO_THREADID_cpy
0001:0001109c  _CRYPTO_THREADID_hash
0001:000110a7* _CRYPTO_get_id_callback
0001:000110b1  _CRYPTO_set_id_callback
0001:000110be* _CRYPTO_thread_id
0001:0001132a  _OpenSSLDie
0001:000111a4  _CRYPTO_add_lock
0001:00011251* _CRYPTO_get_lock_name
0001:000112b2* _OPENSSL_ia32cap_loc
0001:000112bc  _OPENSSL_cpuid_setup
0001:000112c1* _OPENSSL_showfatal
0001:000112ea* _OPENSSL_isservice
0001:00011356* _OPENSSL_stderr
0002:00008d00* _OPENSSL_ia32cap_P
0002:00008d04* _OPENSSL_NONPIC_relocated
Module: U:\extras\lib\libcrypto.lib(cversion.obj)
0001:00011402  _SSLeay_version
0001:000114bf  _SSLeay
Module: U:\extras\lib\libssl.lib(ssl_rsa.obj)
0001:000114da  _SSL_use_certificate
0001:0001157a* _SSL_use_certificate_file
0001:00011733* _SSL_use_certificate_ASN1
0001:000117b4* _SSL_use_RSAPrivateKey
0001:00011a6a* _SSL_use_RSAPrivateKey_file
0001:00011c1d* _SSL_use_RSAPrivateKey_ASN1
0001:00011ca4  _SSL_use_PrivateKey
0001:00011d4a* _SSL_use_PrivateKey_file
0001:00011efd* _SSL_use_PrivateKey_ASN1
0001:00011f8b* _SSL_CTX_use_certificate
0001:0001221b* _SSL_CTX_use_certificate_file
0001:000123c8* _SSL_CTX_use_certificate_ASN1
0001:00012449* _SSL_CTX_use_RSAPrivateKey
0001:00012566* _SSL_CTX_use_RSAPrivateKey_file
0001:0001270d* _SSL_CTX_use_RSAPrivateKey_ASN1
0001:00012794* _SSL_CTX_use_PrivateKey
0001:00012834  _SSL_CTX_use_PrivateKey_file
0001:000129db* _SSL_CTX_use_PrivateKey_ASN1
0001:00012a69  _SSL_CTX_use_certificate_chain_file
Module: U:\extras\lib\libssl.lib(s2_meth.obj)
0001:00012cca  _SSLv2_method
Module: U:\extras\lib\libssl.lib(s3_meth.obj)
0001:00012d7d  _SSLv3_method
Module: U:\extras\lib\libssl.lib(t1_meth.obj)
0001:00012e2d  _TLSv1_method
Module: U:\extras\lib\libssl.lib(s23_meth.obj)
0001:00012efa  _SSLv23_method
Module: U:\extras\lib\libcrypto.lib(obj_dat.obj)
0001:000220d1  _OBJ_bsearch_
0001:00021324  _check_defer
0001:00021345  _OBJ_cleanup
0001:000213d0* _OBJ_new_nid
0001:000213fa* _OBJ_add_object
0001:00021612  _OBJ_nid2obj
0001:00021709  _OBJ_nid2sn
0001:00021804  _OBJ_nid2ln
0001:000219c2  _OBJ_obj2nid
0001:00021a6c  _OBJ_txt2obj
0001:0002203e  _OBJ_sn2nid
0001:00021fab  _OBJ_ln2nid
0001:00021bc9  _OBJ_obj2txt
0001:00021f71* _OBJ_txt2nid
0001:00022108  _OBJ_bsearch_ex_
0001:0002220a* _OBJ_create_objects
0001:000223d7* _OBJ_create
0002:00008e20  _obj_cleanup_defer
Module: U:\extras\lib\libcrypto.lib(a_strex.obj)
0001:000233cc  _X509_NAME_print_ex
0001:0002341d* _X509_NAME_print_ex_fp
0001:000234a2  _ASN1_STRING_print_ex
0001:000234cb* _ASN1_STRING_print_ex_fp
0001:000234f4  _ASN1_STRING_to_UTF8
Module: U:\extras\lib\libcrypto.lib(mem.obj)
0001:00023609* _CRYPTO_set_mem_functions
0001:00023682* _CRYPTO_set_mem_ex_functions
0001:000236fb* _CRYPTO_set_locked_mem_functions
0001:00023742* _CRYPTO_set_locked_mem_ex_functions
0001:00023789* _CRYPTO_set_mem_debug_functions
0001:000237cb* _CRYPTO_get_mem_functions
0001:00023827* _CRYPTO_get_mem_ex_functions
0001:00023883* _CRYPTO_get_locked_mem_functions
0001:000238bc* _CRYPTO_get_locked_mem_ex_functions
0001:000238f5* _CRYPTO_get_mem_debug_functions
0001:0002394f  _CRYPTO_malloc_locked
0001:00023a27  _CRYPTO_free_locked
0001:00023a7b  _CRYPTO_malloc
0001:00023b53* _CRYPTO_strdup
0001:00023b95  _CRYPTO_realloc
0001:00023c78  _CRYPTO_realloc_clean
0001:00023d93  _CRYPTO_free
0001:00023ded* _CRYPTO_remalloc
0001:00023e27* _CRYPTO_set_mem_debug_options
0001:00023e46* _CRYPTO_get_mem_debug_options
Module: U:\extras\lib\libcrypto.lib(x509name.obj)
0001:00023e70* _X509_NAME_get_text_by_NID
0001:00023eb3* _X509_NAME_get_text_by_OBJ
0001:00023fa7* _X509_NAME_get_index_by_OBJ
0001:00024026  _X509_NAME_get_entry
0001:000247dc  _X509_NAME_ENTRY_get_data
0001:00023f49  _X509_NAME_entry_count
0001:00023f6b  _X509_NAME_get_index_by_NID
0001:00024067  _X509_NAME_delete_entry
0001:00024156* _X509_NAME_add_entry_by_OBJ
0001:000245b0* _X509_NAME_ENTRY_create_by_OBJ
0001:000242b4  _X509_NAME_add_entry
0001:000241c7* _X509_NAME_add_entry_by_NID
0001:00024529* _X509_NAME_ENTRY_create_by_NID
0001:00024238  _X509_NAME_add_entry_by_txt
0001:0002447f* _X509_NAME_ENTRY_create_by_txt
0001:00024661* _X509_NAME_ENTRY_set_object
0001:000246d2* _X509_NAME_ENTRY_set_data
0001:000247c5  _X509_NAME_ENTRY_get_object
Module: U:\usr\local446\lib\gcc\i386-pc-os2-emx\4.4.6\libgcc.lib(_alloca.obj)
0001:00024800  __alloca
Module: U:\extras\lib\libcrypto.lib(a_int.obj)
0001:00024830* _ASN1_INTEGER_dup
0001:00024843  _ASN1_INTEGER_cmp
0001:000248a2  _i2c_ASN1_INTEGER
0001:00024a74  _c2i_ASN1_INTEGER
0001:00024ca6  _d2i_ASN1_UINTEGER
0001:00024e72  _ASN1_INTEGER_set
0001:00024fb5  _ASN1_INTEGER_get
0001:0002505f  _BN_to_ASN1_INTEGER
0001:000251d0  _ASN1_INTEGER_to_BN
Module: U:\extras\lib\libcrypto.lib(bss_mem.obj)
0001:0002525e  _BIO_s_mem
0001:00025272  _BIO_new_mem_buf
Module: U:\extras\lib\libcrypto.lib(f_int.obj)
0001:000258a8  _i2a_ASN1_INTEGER
0001:00025a19* _a2i_ASN1_INTEGER
Module: U:\extras\lib\libcrypto.lib(t_x509.obj)
0001:00025e30* _X509_print_fp
0001:00025e63* _X509_print_ex_fp
0001:000260a1* _X509_print_ex
0001:00025f07* _X509_print
0001:00026ba9  _ASN1_TIME_print
0001:00026984* _X509_signature_print
0001:00026774* _X509_ocspid_print
0001:00026aa7  _ASN1_STRING_print
0001:00026fdd  _ASN1_UTCTIME_print
0001:00026c63  _ASN1_GENERALIZEDTIME_print
0001:00027275  _X509_NAME_print
Module: U:\extras\lib\libcrypto.lib(x509_ext.obj)
0001:000273f0* _X509_CRL_get_ext_count
0001:00027408  _X509_CRL_get_ext_by_NID
0001:0002742e* _X509_CRL_get_ext_by_OBJ
0001:00027454* _X509_CRL_get_ext_by_critical
0001:0002747a  _X509_CRL_get_ext
0001:00027499* _X509_CRL_delete_ext
0001:000274b8  _X509_CRL_get_ext_d2i
0001:000274e5* _X509_CRL_add1_ext_i2d
0001:00027519* _X509_CRL_add_ext
0001:00027547  _X509_get_ext_count
0001:0002755f  _X509_get_ext_by_NID
0001:00027585* _X509_get_ext_by_OBJ
0001:000275ab* _X509_get_ext_by_critical
0001:000275d1  _X509_get_ext
0001:000275f0* _X509_delete_ext
0001:0002760f* _X509_add_ext
0001:0002763d  _X509_get_ext_d2i
0001:0002766a* _X509_add1_ext_i2d
0001:0002769e* _X509_REVOKED_get_ext_count
0001:000276b4* _X509_REVOKED_get_ext_by_NID
0001:000276d8* _X509_REVOKED_get_ext_by_OBJ
0001:000276fc* _X509_REVOKED_get_ext_by_critical
0001:00027720* _X509_REVOKED_get_ext
0001:0002773d* _X509_REVOKED_delete_ext
0001:0002775a* _X509_REVOKED_add_ext
0001:00027786  _X509_REVOKED_get_ext_d2i
0001:000277b1* _X509_REVOKED_add1_ext_i2d
Module: U:\extras\lib\libcrypto.lib(v3_lib.obj)
0001:000277f9* _X509V3_EXT_add
0001:00027918  _X509V3_EXT_get_nid
0001:000279ac  _X509V3_EXT_get
0001:000279dc* _X509V3_EXT_add_list
0001:00027a0f* _X509V3_EXT_add_alias
0001:00027afb* _X509V3_EXT_cleanup
0001:00027b43* _X509V3_add_standard_extensions
0001:00027b4d  _X509V3_EXT_d2i
0001:00027bd3  _X509V3_get_d2i
0001:00027cfb  _X509V3_add1_i2d
Module: U:\extras\lib\libcrypto.lib(tasn_dec.obj)
0001:00027f70  _ASN1_tag2bit
0001:00027f92  _ASN1_item_d2i
0001:0002805b  _ASN1_item_ex_d2i
0001:00028000* _ASN1_template_d2i
0001:00029884* _asn1_ex_c2i
Module: U:\extras\lib\libcrypto.lib(stack.obj)
0001:0002a3e0* _STACK_version
0001:0002a408  _sk_set_cmp_func
0001:0002a442  _sk_dup
0001:0002a52f  _sk_new
0001:0002aa65  _sk_free
0001:0002a51b  _sk_new_null
0001:0002a5f5  _sk_insert
0001:0002a70e  _sk_delete_ptr
0001:0002a75a  _sk_delete
0001:0002ab19  _sk_sort
0001:0002a8c0  _sk_find
0001:0002a8e2* _sk_find_ex
0001:0002a904  _sk_push
0001:0002a927* _sk_unshift
0001:0002a949  _sk_shift
0001:0002a981  _sk_pop
0001:0002a9bb  _sk_zero
0001:0002aa07  _sk_pop_free
0001:0002aa99  _sk_num
0001:0002aab0  _sk_value
0001:0002aae2  _sk_set
0001:0002ab6c  _sk_is_sorted
Module: U:\extras\lib\libcrypto.lib(v3_alt.obj)
0001:0002ab90  _v3_alt
0001:0002ac38  _i2v_GENERAL_NAMES
0001:0002ad15  _i2v_GENERAL_NAME
0001:0002b0c1  _GENERAL_NAME_print
0001:0002ba61  _v2i_GENERAL_NAME
0001:0002b98a  _v2i_GENERAL_NAMES
0001:0002be11  _v2i_GENERAL_NAME_ex
0001:0002ba99* _a2i_GENERAL_NAME
Module: U:\extras\lib\libcrypto.lib(bss_file.obj)
0001:0002c217  _BIO_new_file
0001:0002c3cf  _BIO_s_file
0001:0002c373  _BIO_new_fp
Module: U:\extras\lib\libcrypto.lib(pem_xaux.obj)
0001:0002ca54  _PEM_read_bio_X509_AUX
0001:0002ca8d* _PEM_read_X509_AUX
0001:0002cac6* _PEM_write_bio_X509_AUX
0001:0002cb19* _PEM_write_X509_AUX
0001:0002cb7d* _PEM_read_bio_X509_CERT_PAIR
0001:0002cbb6* _PEM_read_X509_CERT_PAIR
0001:0002cbef* _PEM_write_bio_X509_CERT_PAIR
0001:0002cc42* _PEM_write_X509_CERT_PAIR
Module: U:\usr\local446\lib\gcc\i386-pc-os2-emx\4.4.6\libgcc.lib(emx-ctordtor.obj)
0001:0002cca0  ___ctordtorTerm
0001:0002ccd2  ___ctordtorInit
Module: U:\extras\lib\libcrypto.lib(eng_init.obj)
0001:0002cd10  _engine_unlocked_init
0001:0002cd76  _engine_unlocked_finish
0001:0002ce67  _ENGINE_init
0001:0002cf01  _ENGINE_finish
Module: U:\extras\lib\libcrypto.lib(tb_rand.obj)
0001:0002cff4* _ENGINE_unregister_RAND
0001:0002d023* _ENGINE_register_RAND
0001:0002d06f* _ENGINE_register_all_RAND
0001:0002d0a0* _ENGINE_set_default_RAND
0001:0002d0ec  _ENGINE_get_default_RAND
0001:0002d109  _ENGINE_get_RAND
0001:0002d114* _ENGINE_set_RAND
Module: U:\extras\lib\libcrypto.lib(md_rand.obj)
0001:0002d130* _RAND_version
0001:0002d157  _RAND_SSLeay
0002:00000df0* _rand_ssleay_meth
Module: U:\extras\lib\libcrypto.lib(buffer.obj)
0001:0002dd99  _BUF_MEM_new
0001:0002de19  _BUF_MEM_free
0001:0002de6d  _BUF_MEM_grow
0001:0002dfc9  _BUF_MEM_grow_clean
0001:0002e158  _BUF_strdup
0001:0002e187  _BUF_strndup
0001:0002e296  _BUF_strlcpy
0001:0002e211  _BUF_memdup
0001:0002e2e6  _BUF_strlcat
0001:0002e32b* _BUF_reverse
Module: U:\usr\local446\lib\libc_dll.lib(socket.obj)
0001:0002e3b0  _socket
Module: U:\usr\local446\lib\libc_dll.lib(connect.obj)
0001:0002e430  _connect
Module: U:\extras\lib\libssl.lib(ssl_sess.obj)
0001:0002e4d0  _SSL_get_session
0001:0002e4e9* _SSL_get1_session
0001:0002e563* _SSL_SESSION_get_ex_new_index
0001:0002e59a* _SSL_SESSION_set_ex_data
0001:0002e5c1* _SSL_SESSION_get_ex_data
0001:0002e5e1  _SSL_SESSION_new
0001:0002e73f* _SSL_SESSION_get_id
0001:0002e7c3  _ssl_get_new_session
0001:0002f5ed  _SSL_SESSION_free
0001:0002ee5a  _ssl_get_prev_session
0001:0002f2f5  _SSL_CTX_add_session
0001:0002f4b6  _SSL_CTX_remove_session
0001:0002f7e9  _SSL_set_session
0001:0002f9c1* _SSL_SESSION_set_timeout
0001:0002f9e4* _SSL_SESSION_get_timeout
0001:0002f9ff* _SSL_SESSION_get_time
0001:0002fa1a* _SSL_SESSION_set_time
0001:0002fa3b* _SSL_CTX_set_timeout
0001:0002fa65* _SSL_CTX_get_timeout
0001:0002fa7d* _SSL_set_session_secret_cb
0001:0002faac* _SSL_set_session_ticket_ext_cb
0001:0002fadb* _SSL_set_session_ticket_ext
0001:0002fcbf  _SSL_CTX_flush_sessions
0001:0002fd68  _ssl_clear_bad_session
0001:0002ffa5* _SSL_CTX_sess_set_new_cb
0001:0002ffb3* _SSL_CTX_sess_get_new_cb
0001:0002ffbe* _SSL_CTX_sess_set_remove_cb
0001:0002ffcc* _SSL_CTX_sess_get_remove_cb
0001:0002ffd7* _SSL_CTX_sess_set_get_cb
0001:0002ffe5* _SSL_CTX_sess_get_get_cb
0001:0002fff0* _SSL_CTX_set_info_callback
0001:00030001* _SSL_CTX_get_info_callback
0001:0003000f* _SSL_CTX_set_client_cert_cb
0001:0003001d* _SSL_CTX_get_client_cert_cb
0001:00030028* _SSL_CTX_set_client_cert_engine
0001:000300d0* _SSL_CTX_set_cookie_generate_cb
0001:000300de* _SSL_CTX_set_cookie_verify_cb
0001:00030103* _PEM_read_bio_SSL_SESSION
0001:0003013c* _PEM_read_SSL_SESSION
0001:00030175* _PEM_write_bio_SSL_SESSION
0001:000301c8* _PEM_write_SSL_SESSION
Module: U:\extras\lib\libssl.lib(ssl_cert.obj)
0001:00030243  _SSL_get_ex_data_X509_STORE_CTX_idx
0001:00030361  _ssl_cert_new
0001:000303f4  _ssl_cert_dup
0001:00030899  _ssl_cert_free
0001:0003099b  _ssl_cert_inst
0001:00030a30  _ssl_sess_cert_new
0001:00030ac4  _ssl_sess_cert_free
0001:00030bbb  _ssl_set_peer_cert_type
0001:00030be4  _ssl_verify_cert_chain
0001:00030db9* _SSL_dup_CA_list
0001:00030e3c* _SSL_set_client_CA_list
0001:00030e5c* _SSL_CTX_set_client_CA_list
0001:00030e7c* _SSL_CTX_get_client_CA_list
0001:00030e8a  _SSL_get_client_CA_list
0001:00030f7b* _SSL_add_client_CA
0001:00030f9b* _SSL_CTX_add_client_CA
0001:00030fd9* _SSL_load_client_CA_file
0001:000311ca* _SSL_add_file_cert_subjects_to_stack
0001:00031366* _SSL_add_dir_cert_subjects_to_stack
Module: U:\extras\lib\libcrypto.lib(x509_vpm.obj)
0001:000315e2  _X509_VERIFY_PARAM_new
0001:00031632  _X509_VERIFY_PARAM_free
0001:00031650  _X509_VERIFY_PARAM_inherit
0001:0003199a* _X509_VERIFY_PARAM_set1_policies
0001:000317f8  _X509_VERIFY_PARAM_set1
0001:0003183b* _X509_VERIFY_PARAM_set1_name
0001:0003187e  _X509_VERIFY_PARAM_set_flags
0001:000318b6* _X509_VERIFY_PARAM_clear_flags
0001:000318d3* _X509_VERIFY_PARAM_get_flags
0001:000318de  _X509_VERIFY_PARAM_set_purpose
0001:000318fb  _X509_VERIFY_PARAM_set_trust
0001:00031918  _X509_VERIFY_PARAM_set_depth
0001:00031926  _X509_VERIFY_PARAM_set_time
0001:00031945* _X509_VERIFY_PARAM_add0_policy
0001:00031a9b  _X509_VERIFY_PARAM_get_depth
0001:00031c17* _X509_VERIFY_PARAM_add0_table
0001:00031cc1  _X509_VERIFY_PARAM_lookup
0001:00031d26* _X509_VERIFY_PARAM_table_cleanup
Module: U:\extras\lib\libcrypto.lib(ex_data.obj)
0001:00031dcd* _CRYPTO_get_ex_data_implementation
0001:00031de8* _CRYPTO_set_ex_data_implementation
0001:00032b71  _CRYPTO_get_ex_data
0001:00032a8c  _CRYPTO_set_ex_data
0001:0003295b* _CRYPTO_ex_data_new_class
0001:0003297a* _CRYPTO_cleanup_all_ex_data
0001:0003299a  _CRYPTO_get_ex_new_index
0001:000329f0  _CRYPTO_new_ex_data
0001:00032a24  _CRYPTO_dup_ex_data
0001:00032a58  _CRYPTO_free_ex_data
Module: U:\extras\lib\libcrypto.lib(lhash.obj)
0001:00032bc0* _lh_version
0001:00032bf0  _lh_new
0001:0003352a  _lh_strhash
0001:00032d8d  _lh_free
0001:00032e01  _lh_insert
0001:00032f1f  _lh_delete
0001:00032ff9  _lh_retrieve
0001:000330da  _lh_doall
0001:0003310c  _lh_doall_arg
0001:000335a1  _lh_num_items
Module: U:\extras\lib\libcrypto.lib(x_exten.obj)
0001:00033630  _X509_EXTENSION_it
0001:00033690  _X509_EXTENSIONS_it
0001:000336ac* _d2i_X509_EXTENSION
0001:000336d5* _i2d_X509_EXTENSION
0001:000336f7  _X509_EXTENSION_new
0001:0003370b  _X509_EXTENSION_free
0001:00033726  _d2i_X509_EXTENSIONS
0001:0003374f  _i2d_X509_EXTENSIONS
0001:00033771  _X509_EXTENSION_dup
Module: U:\extras\lib\libcrypto.lib(ocsp_asn.obj)
0001:00033810* _OCSP_SIGNATURE_it
0001:0003382c* _d2i_OCSP_SIGNATURE
0001:00033855* _i2d_OCSP_SIGNATURE
0001:00033877* _OCSP_SIGNATURE_new
0001:0003388b* _OCSP_SIGNATURE_free
0001:00033940* _OCSP_CERTID_it
0001:0003395c* _d2i_OCSP_CERTID
0001:00033985* _i2d_OCSP_CERTID
0001:000339a7* _OCSP_CERTID_new
0001:000339bb* _OCSP_CERTID_free
0001:00033a40* _OCSP_ONEREQ_it
0001:00033a5c* _d2i_OCSP_ONEREQ
0001:00033a85* _i2d_OCSP_ONEREQ
0001:00033aa7* _OCSP_ONEREQ_new
0001:00033abb* _OCSP_ONEREQ_free
0001:00033b70* _OCSP_REQINFO_it
0001:00033b8c* _d2i_OCSP_REQINFO
0001:00033bb5* _i2d_OCSP_REQINFO
0001:00033bd7* _OCSP_REQINFO_new
0001:00033beb* _OCSP_REQINFO_free
0001:00033c70* _OCSP_REQUEST_it
0001:00033c8c* _d2i_OCSP_REQUEST
0001:00033cb5* _i2d_OCSP_REQUEST
0001:00033cd7* _OCSP_REQUEST_new
0001:00033ceb* _OCSP_REQUEST_free
0001:00033d60* _OCSP_RESPBYTES_it
0001:00033d7c* _d2i_OCSP_RESPBYTES
0001:00033da5* _i2d_OCSP_RESPBYTES
0001:00033dc7* _OCSP_RESPBYTES_new
0001:00033ddb* _OCSP_RESPBYTES_free
0001:00033e60* _OCSP_RESPONSE_it
0001:00033e7c* _d2i_OCSP_RESPONSE
0001:00033ea5* _i2d_OCSP_RESPONSE
0001:00033ec7* _OCSP_RESPONSE_new
0001:00033edb* _OCSP_RESPONSE_free
0001:00033f50* _OCSP_RESPID_it
0001:00033f6c  _d2i_OCSP_RESPID
0001:00033f95  _i2d_OCSP_RESPID
0001:00033fb7* _OCSP_RESPID_new
0001:00033fcb  _OCSP_RESPID_free
0001:00034050* _OCSP_REVOKEDINFO_it
0001:0003406c* _d2i_OCSP_REVOKEDINFO
0001:00034095* _i2d_OCSP_REVOKEDINFO
0001:000340b7* _OCSP_REVOKEDINFO_new
0001:000340cb* _OCSP_REVOKEDINFO_free
0001:00034160* _OCSP_CERTSTATUS_it
0001:0003417c* _d2i_OCSP_CERTSTATUS
0001:000341a5* _i2d_OCSP_CERTSTATUS
0001:000341c7* _OCSP_CERTSTATUS_new
0001:000341db* _OCSP_CERTSTATUS_free
0001:000342b0* _OCSP_SINGLERESP_it
0001:000342cc* _d2i_OCSP_SINGLERESP
0001:000342f5* _i2d_OCSP_SINGLERESP
0001:00034317* _OCSP_SINGLERESP_new
0001:0003432b* _OCSP_SINGLERESP_free
0001:00034400* _OCSP_RESPDATA_it
0001:0003441c* _d2i_OCSP_RESPDATA
0001:00034445* _i2d_OCSP_RESPDATA
0001:00034467* _OCSP_RESPDATA_new
0001:0003447b* _OCSP_RESPDATA_free
0001:00034510* _OCSP_BASICRESP_it
0001:0003452c* _d2i_OCSP_BASICRESP
0001:00034555* _i2d_OCSP_BASICRESP
0001:00034577* _OCSP_BASICRESP_new
0001:0003458b* _OCSP_BASICRESP_free
0001:00034610  _OCSP_CRLID_it
0001:0003462c* _d2i_OCSP_CRLID
0001:00034655* _i2d_OCSP_CRLID
0001:00034677* _OCSP_CRLID_new
0001:0003468b* _OCSP_CRLID_free
0001:00034700  _OCSP_SERVICELOC_it
0001:0003471c* _d2i_OCSP_SERVICELOC
0001:00034745* _i2d_OCSP_SERVICELOC
0001:00034767* _OCSP_SERVICELOC_new
0001:0003477b* _OCSP_SERVICELOC_free
Module: U:\extras\lib\libcrypto.lib(x_name.obj)
0001:00034870  _X509_NAME_ENTRY_it
0001:0003488c* _d2i_X509_NAME_ENTRY
0001:000348b5* _i2d_X509_NAME_ENTRY
0001:000348d7  _X509_NAME_ENTRY_new
0001:000348eb  _X509_NAME_ENTRY_free
0001:00034906  _X509_NAME_ENTRY_dup
0001:00034960* _X509_NAME_ENTRIES_it
0001:000349c0* _X509_NAME_INTERNAL_it
0001:000349e0* _x509_name_ff
0001:00034a10  _X509_NAME_it
0001:00034a2c  _d2i_X509_NAME
0001:00034a55  _i2d_X509_NAME
0001:00034a77  _X509_NAME_new
0001:00034a8b  _X509_NAME_free
0001:00034aa6  _X509_NAME_dup
0001:00035556  _X509_NAME_set
Module: U:\extras\lib\libcrypto.lib(bss_sock.obj)
0001:000355c7  _BIO_s_socket
0001:000355d1* _BIO_new_socket
0001:000358a7* _BIO_sock_should_retry
0001:000358d7* _BIO_sock_non_fatal_error
Module: U:\extras\lib\libssl.lib(s3_pkt.obj)
0001:00035919* _ssl3_read_n
0001:0003630a* _ssl3_do_uncompress
0001:00037bcd  _ssl3_send_alert
0001:00036388* _ssl3_do_compress
0001:00036406  _ssl3_write_bytes
0001:00036a02* _ssl3_write_pending
0001:00036bd5  _ssl3_read_bytes
0001:00037a55* _ssl3_do_change_cipher_spec
0001:00037c9c  _ssl3_dispatch_alert
Module: U:\extras\lib\libcrypto.lib(x509_lu.obj)
0001:00037e3a* _X509_LOOKUP_new
0001:00037ecf* _X509_LOOKUP_free
0001:00037f13* _X509_LOOKUP_init
0001:00037f51* _X509_LOOKUP_shutdown
0001:00037f8f  _X509_LOOKUP_ctrl
0001:00037fe9* _X509_LOOKUP_by_subject
0001:00038046* _X509_LOOKUP_by_issuer_serial
0001:00038099* _X509_LOOKUP_by_fingerprint
0001:000380ec* _X509_LOOKUP_by_alias
0001:000381c8  _X509_STORE_new
0001:0003834a  _X509_STORE_free
0001:00038411  _X509_STORE_add_lookup
0001:000384b5* _X509_STORE_get_by_subject
0001:00038a86* _X509_OBJECT_retrieve_by_subject
0001:000388ad* _X509_OBJECT_up_ref_count
0001:000385f7  _X509_STORE_add_cert
0001:00038f63* _X509_OBJECT_retrieve_match
0001:0003892b* _X509_OBJECT_free_contents
0001:00038752  _X509_STORE_add_crl
0001:00038a5d* _X509_OBJECT_idx_by_subject
0001:00038ac9  _X509_STORE_get1_certs
0001:00038d1b  _X509_STORE_get1_crls
0001:0003906f  _X509_STORE_CTX_get1_issuer
0001:0003928e* _X509_STORE_set_flags
0001:000392ab* _X509_STORE_set_depth
0001:000392cd* _X509_STORE_set_purpose
0001:000392ea* _X509_STORE_set_trust
0001:00039307* _X509_STORE_set1_param
0001:00039324* _X509_STORE_set_verify_cb
Module: U:\extras\lib\libcrypto.lib(names.obj)
0001:00039340  _EVP_add_cipher
0001:000393b8  _EVP_add_digest
0001:000394cd  _EVP_get_cipherbyname
0001:000394ee  _EVP_get_digestbyname
0001:0003950f* _EVP_cleanup
0001:000395d5* _EVP_CIPHER_do_all
0001:00039604* _EVP_CIPHER_do_all_sorted
0001:000396aa* _EVP_MD_do_all
0001:000396d9* _EVP_MD_do_all_sorted
Module: U:\extras\lib\libcrypto.lib(rsa_lib.obj)
0001:00039710* _RSA_version
0001:00039736  _RSA_new
0001:00039803* _RSA_new_method
0001:00039750* _RSA_set_default_method
0001:0003975d* _RSA_get_default_method
0001:0003977d* _RSA_get_method
0001:00039788* _RSA_set_method
0001:00039ac3  _RSA_free
0001:00039c7c  _RSA_up_ref
0001:00039cbf* _RSA_get_ex_new_index
0001:00039cf6* _RSA_set_ex_data
0001:00039d1a* _RSA_get_ex_data
0001:00039d37  _RSA_size
0001:00039d5a  _RSA_public_encrypt
0001:00039d8f  _RSA_private_encrypt
0001:00039dc4  _RSA_private_decrypt
0001:00039df9  _RSA_public_decrypt
0001:00039e2e  _RSA_flags
0001:00039e49* _RSA_blinding_off
0001:00039e95* _RSA_blinding_on
0001:0003a014  _RSA_setup_blinding
0001:0003a299* _RSA_memory_lock
Module: U:\extras\lib\libcrypto.lib(dh_lib.obj)
0001:0003a490* _DH_version
0001:0003a4c1* _DH_set_default_method
0001:0003a4ce* _DH_get_default_method
0001:0003a4ee* _DH_set_method
0001:0003a55f  _DH_new
0001:0003a57c* _DH_new_method
0001:0003a7f0  _DH_free
0001:0003a961  _DH_up_ref
0001:0003a9a4* _DH_get_ex_new_index
0001:0003a9db* _DH_set_ex_data
0001:0003a9ff* _DH_get_ex_data
0001:0003aa1c  _DH_size
Module: U:\extras\lib\libcrypto.lib(p_lib.obj)
0001:0003aa40  _EVP_PKEY_bits
0001:0003aa7d  _EVP_PKEY_size
0001:0003aaba* _EVP_PKEY_save_parameters
0001:0003ab1f  _EVP_PKEY_copy_parameters
0001:0003abd6  _EVP_PKEY_missing_parameters
0001:0003ac0d  _EVP_PKEY_cmp_parameters
0001:0003ac60  _EVP_PKEY_cmp
0001:0003ace6  _EVP_PKEY_new
0001:0003aec0  _EVP_PKEY_set_type
0001:0003aeea  _EVP_PKEY_set_type_str
0001:0003af13  _EVP_PKEY_assign
0001:0003af4b* _EVP_PKEY_get0
0001:0003af56  _EVP_PKEY_set1_RSA
0001:0003af8f  _EVP_PKEY_get1_RSA
0001:0003afe8  _EVP_PKEY_set1_DSA
0001:0003b021  _EVP_PKEY_get1_DSA
0001:0003b07a  _EVP_PKEY_set1_EC_KEY
0001:0003b0b3  _EVP_PKEY_get1_EC_KEY
0001:0003b10e* _EVP_PKEY_set1_DH
0001:0003b147* _EVP_PKEY_get1_DH
0001:0003b1a0  _EVP_PKEY_type
0001:0003b1e9  _EVP_PKEY_id
0001:0003b1f3* _EVP_PKEY_base_id
0001:0003b208  _EVP_PKEY_free
0001:0003b364  _EVP_PKEY_print_public
0001:0003b3d8  _EVP_PKEY_print_private
0001:0003b44b  _EVP_PKEY_print_params
0001:0003b4b3  _EVP_PKEY_get_default_digest_nid
Module: U:\extras\lib\libcrypto.lib(v3_purp.obj)
0001:0003b611  _X509_check_purpose
0001:0003b7ea  _X509_PURPOSE_get_by_id
0001:0003b74d  _X509_PURPOSE_get0
0001:0003b6cd  _X509_PURPOSE_set
0001:0003b725* _X509_PURPOSE_get_count
0001:0003b79b* _X509_PURPOSE_get_by_sname
0001:0003b844* _X509_PURPOSE_add
0001:0003baba* _X509_PURPOSE_cleanup
0001:0003bb14* _X509_PURPOSE_get_id
0001:0003bb1e* _X509_PURPOSE_get0_name
0001:0003bb29* _X509_PURPOSE_get0_sname
0001:0003bb34* _X509_PURPOSE_get_trust
0001:0003bbab* _X509_supported_extension
0001:0003c49b  _X509_check_ca
0001:0003c948  _X509_check_issued
0001:0003ca22  _X509_check_akid
Module: U:\extras\lib\libcrypto.lib(evp_enc.obj)
0001:0003cb70* _EVP_version
0001:0003cb96  _EVP_CIPHER_CTX_init
0001:0003cbc3* _EVP_CIPHER_CTX_new
0001:0003cbfe* _EVP_CipherInit
0001:0003ccde  _EVP_CipherInit_ex
0001:0003da31  _EVP_CIPHER_CTX_cleanup
0001:0003dbb8  _EVP_CIPHER_CTX_ctrl
0001:0003d10a  _EVP_CipherUpdate
0001:0003d2e2  _EVP_EncryptUpdate
0001:0003d683  _EVP_DecryptUpdate
0001:0003d16c  _EVP_CipherFinal_ex
0001:0003d551  _EVP_EncryptFinal_ex
0001:0003d816  _EVP_DecryptFinal_ex
0001:0003d1b2* _EVP_CipherFinal
0001:0003d515  _EVP_EncryptFinal
0001:0003d7ef  _EVP_DecryptFinal
0001:0003d1f8* _EVP_EncryptInit
0001:0003d228  _EVP_EncryptInit_ex
0001:0003d25f* _EVP_DecryptInit
0001:0003d28f  _EVP_DecryptInit_ex
0001:0003da0d* _EVP_CIPHER_CTX_free
0001:0003dadf  _EVP_CIPHER_CTX_set_key_length
0001:0003db84* _EVP_CIPHER_CTX_set_padding
0001:0003dca2  _EVP_CIPHER_CTX_rand_key
0001:0003dd04  _EVP_CIPHER_CTX_copy
Module: U:\extras\lib\libcrypto.lib(comp_lib.obj)
0001:0003debb  _COMP_CTX_new
0001:0003df47  _COMP_CTX_free
0001:0003df7f  _COMP_compress_block
0001:0003dff4  _COMP_expand_block
Module: U:\extras\lib\libcrypto.lib(bf_buff.obj)
0001:0003e077  _BIO_f_buffer
Module: U:\extras\lib\libcrypto.lib(x509_d2.obj)
0001:0003ee50  _X509_STORE_set_default_paths
0001:0003ef03  _X509_STORE_load_locations
Module: U:\extras\lib\libcrypto.lib(digest.obj)
0001:0003eff0  _EVP_MD_CTX_init
0001:0003f01c  _EVP_MD_CTX_create
0001:0003f057  _EVP_DigestInit
0001:0003f084  _EVP_DigestInit_ex
0001:0003f34d  _EVP_DigestUpdate
0001:0003f371  _EVP_DigestFinal
0001:0003f3cc  _EVP_DigestFinal_ex
0001:0003f781  _EVP_MD_CTX_cleanup
0001:0003f482  _EVP_MD_CTX_copy
0001:0003f4a7  _EVP_MD_CTX_copy_ex
0001:0003f6c9  _EVP_Digest
0001:0003f763  _EVP_MD_CTX_destroy
Module: U:\extras\lib\libcrypto.lib(mem_dbg.obj)
0001:0003f8ce  _CRYPTO_mem_ctrl
0001:0003fac2* _CRYPTO_is_mem_check_on
0001:0003fb69* _CRYPTO_dbg_set_options
0001:0003fb76* _CRYPTO_dbg_get_options
0001:0003fddb  _CRYPTO_push_info_
0001:0003fee2  _CRYPTO_pop_info
0001:0003ff25* _CRYPTO_remove_all_info
0001:0003ff66* _CRYPTO_dbg_malloc
0001:00040194* _CRYPTO_dbg_free
0001:00040227* _CRYPTO_dbg_realloc
0001:0004074b* _CRYPTO_mem_leaks
0001:0004089d* _CRYPTO_mem_leaks_fp
0001:00040988* _CRYPTO_mem_leaks_cb
Module: U:\extras\lib\libcrypto.lib(b_print.obj)
0001:00041e53  _BIO_printf
0001:00041e88* _BIO_vprintf
0001:00041f7c  _BIO_snprintf
0001:00041fb0* _BIO_vsnprintf
Module: U:\extras\lib\libcrypto.lib(ameth_lib.obj)
0001:00042090* _EVP_PKEY_asn1_get_count
0001:000420bb* _EVP_PKEY_asn1_get0
0001:00042191  _EVP_PKEY_asn1_find
0001:00042207  _EVP_PKEY_asn1_find_str
0001:000422f1* _EVP_PKEY_asn1_add0
0001:00042355* _EVP_PKEY_asn1_add_alias
0001:00042428* _EVP_PKEY_asn1_new
0001:000423a4  _EVP_PKEY_asn1_get0_info
0001:00042411* _EVP_PKEY_get0_asn1
0001:0004269a  _EVP_PKEY_asn1_free
0001:000425b1* _EVP_PKEY_asn1_copy
0001:000426f0* _EVP_PKEY_asn1_set_public
0001:0004272b* _EVP_PKEY_asn1_set_private
0001:0004274b* _EVP_PKEY_asn1_set_param
0001:00042786* _EVP_PKEY_asn1_set_free
0001:00042794* _EVP_PKEY_asn1_set_ctrl
Module: U:\extras\lib\libcrypto.lib(evp_lib.obj)
0001:000427b0  _EVP_CIPHER_param_to_asn1
0001:000427ea  _EVP_CIPHER_asn1_to_param
0001:00042841  _EVP_CIPHER_get_asn1_iv
0001:00042b2b  _EVP_CIPHER_CTX_iv_length
0001:000428f3  _EVP_CIPHER_set_asn1_iv
0001:0004295a  _EVP_CIPHER_type
0001:00042b4e  _EVP_CIPHER_nid
0001:00042aa0  _EVP_CIPHER_block_size
0001:00042aab  _EVP_CIPHER_CTX_block_size
0001:00042ab8  _EVP_Cipher
0001:00042ae5  _EVP_CIPHER_CTX_cipher
0001:00042aef* _EVP_CIPHER_flags
0001:00042afa  _EVP_CIPHER_CTX_flags
0001:00042b07* _EVP_CIPHER_CTX_get_app_data
0001:00042b12* _EVP_CIPHER_CTX_set_app_data
0001:00042b20  _EVP_CIPHER_iv_length
0001:00042b38  _EVP_CIPHER_key_length
0001:00042b43  _EVP_CIPHER_CTX_key_length
0001:00042b58* _EVP_CIPHER_CTX_nid
0001:00042b64  _EVP_MD_block_size
0001:00042b6f  _EVP_MD_type
0001:00042b79  _EVP_MD_pkey_type
0001:00042b84  _EVP_MD_size
0001:00042bcb* _EVP_MD_flags
0001:00042bd6  _EVP_MD_CTX_md
0001:00042bed  _EVP_MD_CTX_set_flags
0001:00042c03  _EVP_MD_CTX_clear_flags
0001:00042c1b  _EVP_MD_CTX_test_flags
0001:00042c2b* _EVP_CIPHER_CTX_set_flags
0001:00042c41* _EVP_CIPHER_CTX_clear_flags
0001:00042c59* _EVP_CIPHER_CTX_test_flags
Module: U:\extras\lib\libcrypto.lib(c_zlib.obj)
0001:00042c78  _COMP_zlib
0001:00042c8a* _COMP_zlib_cleanup
Module: U:\extras\lib\libcrypto.lib(e_null.obj)
0001:00042cc4  _EVP_enc_null
Module: U:\extras\lib\libcrypto.lib(tasn_typ.obj)
0001:00042d20  _ASN1_INTEGER_it
0001:00042d3c  _d2i_ASN1_INTEGER
0001:00042d65  _i2d_ASN1_INTEGER
0001:00042d87  _ASN1_INTEGER_new
0001:00042d9b  _ASN1_INTEGER_free
0001:00042dd0  _ASN1_ENUMERATED_it
0001:00042dec  _d2i_ASN1_ENUMERATED
0001:00042e15* _i2d_ASN1_ENUMERATED
0001:00042e37* _ASN1_ENUMERATED_new
0001:00042e4b  _ASN1_ENUMERATED_free
0001:00042e80  _ASN1_BIT_STRING_it
0001:00042e9c  _d2i_ASN1_BIT_STRING
0001:00042ec5  _i2d_ASN1_BIT_STRING
0001:00042ee7  _ASN1_BIT_STRING_new
0001:00042efb  _ASN1_BIT_STRING_free
0001:00042f30  _ASN1_OCTET_STRING_it
0001:00042f4c  _d2i_ASN1_OCTET_STRING
0001:00042f75  _i2d_ASN1_OCTET_STRING
0001:00042f97  _ASN1_OCTET_STRING_new
0001:00042fab  _ASN1_OCTET_STRING_free
0001:00042fd0  _ASN1_NULL_it
0001:00042fec* _d2i_ASN1_NULL
0001:00043015* _i2d_ASN1_NULL
0001:00043037  _ASN1_NULL_new
0001:0004304b* _ASN1_NULL_free
0001:00043080  _ASN1_OBJECT_it
0001:000430b0  _ASN1_UTF8STRING_it
0001:000430cc* _d2i_ASN1_UTF8STRING
0001:000430f5* _i2d_ASN1_UTF8STRING
0001:00043117  _ASN1_UTF8STRING_new
0001:0004312b  _ASN1_UTF8STRING_free
0001:00043160* _ASN1_PRINTABLESTRING_it
0001:0004317c* _d2i_ASN1_PRINTABLESTRING
0001:000431a5* _i2d_ASN1_PRINTABLESTRING
0001:000431c7* _ASN1_PRINTABLESTRING_new
0001:000431db* _ASN1_PRINTABLESTRING_free
0001:00043210* _ASN1_T61STRING_it
0001:0004322c* _d2i_ASN1_T61STRING
0001:00043255* _i2d_ASN1_T61STRING
0001:00043277* _ASN1_T61STRING_new
0001:0004328b* _ASN1_T61STRING_free
0001:000432c0  _ASN1_IA5STRING_it
0001:000432dc* _d2i_ASN1_IA5STRING
0001:00043305* _i2d_ASN1_IA5STRING
0001:00043327* _ASN1_IA5STRING_new
0001:0004333b* _ASN1_IA5STRING_free
0001:00043370* _ASN1_GENERALSTRING_it
0001:0004338c* _d2i_ASN1_GENERALSTRING
0001:000433b5* _i2d_ASN1_GENERALSTRING
0001:000433d7* _ASN1_GENERALSTRING_new
0001:000433eb* _ASN1_GENERALSTRING_free
0001:00043420* _ASN1_UTCTIME_it
0001:0004343c* _d2i_ASN1_UTCTIME
0001:00043465* _i2d_ASN1_UTCTIME
0001:00043487* _ASN1_UTCTIME_new
0001:0004349b* _ASN1_UTCTIME_free
0001:000434d0  _ASN1_GENERALIZEDTIME_it
0001:000434ec* _d2i_ASN1_GENERALIZEDTIME
0001:00043515* _i2d_ASN1_GENERALIZEDTIME
0001:00043537  _ASN1_GENERALIZEDTIME_new
0001:0004354b* _ASN1_GENERALIZEDTIME_free
0001:00043580* _ASN1_VISIBLESTRING_it
0001:0004359c* _d2i_ASN1_VISIBLESTRING
0001:000435c5* _i2d_ASN1_VISIBLESTRING
0001:000435e7* _ASN1_VISIBLESTRING_new
0001:000435fb* _ASN1_VISIBLESTRING_free
0001:00043630* _ASN1_UNIVERSALSTRING_it
0001:0004364c* _d2i_ASN1_UNIVERSALSTRING
0001:00043675* _i2d_ASN1_UNIVERSALSTRING
0001:00043697* _ASN1_UNIVERSALSTRING_new
0001:000436ab* _ASN1_UNIVERSALSTRING_free
0001:000436e0* _ASN1_BMPSTRING_it
0001:000436fc* _d2i_ASN1_BMPSTRING
0001:00043725* _i2d_ASN1_BMPSTRING
0001:00043747* _ASN1_BMPSTRING_new
0001:0004375b* _ASN1_BMPSTRING_free
0001:00043780  _ASN1_ANY_it
0001:000437b0  _ASN1_SEQUENCE_it
0001:000437cc  _d2i_ASN1_TYPE
0001:000437f5  _i2d_ASN1_TYPE
0001:00043817  _ASN1_TYPE_new
0001:0004382b  _ASN1_TYPE_free
0001:00043860  _ASN1_PRINTABLE_it
0001:0004387c* _d2i_ASN1_PRINTABLE
0001:000438a5* _i2d_ASN1_PRINTABLE
0001:000438c7* _ASN1_PRINTABLE_new
0001:000438db* _ASN1_PRINTABLE_free
0001:00043910  _DISPLAYTEXT_it
0001:0004392c* _d2i_DISPLAYTEXT
0001:00043955* _i2d_DISPLAYTEXT
0001:00043977* _DISPLAYTEXT_new
0001:0004398b* _DISPLAYTEXT_free
0001:000439c0  _DIRECTORYSTRING_it
0001:000439dc* _d2i_DIRECTORYSTRING
0001:00043a05* _i2d_DIRECTORYSTRING
0001:00043a27* _DIRECTORYSTRING_new
0001:00043a3b* _DIRECTORYSTRING_free
0001:00043a70  _ASN1_BOOLEAN_it
0001:00043aa0* _ASN1_TBOOLEAN_it
0001:00043ad0  _ASN1_FBOOLEAN_it
0001:00043b10  _ASN1_OCTET_STRING_NDEF_it
0001:00043b60* _ASN1_SEQUENCE_ANY_it
0001:00043bb0* _ASN1_SET_ANY_it
0001:00043bcc  _d2i_ASN1_SEQUENCE_ANY
0001:00043bf5  _i2d_ASN1_SEQUENCE_ANY
0001:00043c17* _d2i_ASN1_SET_ANY
0001:00043c40  _i2d_ASN1_SET_ANY
Module: U:\extras\lib\libcrypto.lib(x_algor.obj)
0001:00043cd0  _X509_ALGOR_it
0001:00043d20  _X509_ALGORS_it
0001:00043d3c  _d2i_X509_ALGOR
0001:00043d65* _i2d_X509_ALGOR
0001:00043d87  _X509_ALGOR_new
0001:00043d9b  _X509_ALGOR_free
0001:00043db6* _d2i_X509_ALGORS
0001:00043ddf  _i2d_X509_ALGORS
0001:00043e01* _X509_ALGOR_dup
0001:00043e1c  _X509_ALGOR_set0
0001:00043edc  _X509_ALGOR_get0
Module: U:\extras\lib\libcrypto.lib(x_val.obj)
0001:00043f90  _X509_VAL_it
0001:00043fac* _d2i_X509_VAL
0001:00043fd5* _i2d_X509_VAL
0001:00043ff7* _X509_VAL_new
0001:0004400b* _X509_VAL_free
Module: U:\extras\lib\libcrypto.lib(x_pubkey.obj)
0001:000440d0  _X509_PUBKEY_it
0001:000440ec* _d2i_X509_PUBKEY
0001:00044115* _i2d_X509_PUBKEY
0001:00044137* _X509_PUBKEY_new
0001:0004414b* _X509_PUBKEY_free
0001:00044171  _X509_PUBKEY_set
0001:000442a6  _X509_PUBKEY_get
0001:00044480  _d2i_PUBKEY
0001:000444f6  _i2d_PUBKEY
0001:00044552  _d2i_RSA_PUBKEY
0001:000445d8  _i2d_RSA_PUBKEY
0001:00044663  _d2i_DSA_PUBKEY
0001:000446e9  _i2d_DSA_PUBKEY
0001:00044774  _d2i_EC_PUBKEY
0001:000447fa  _i2d_EC_PUBKEY
0001:00044885  _X509_PUBKEY_set0_param
0001:00044924  _X509_PUBKEY_get0_param
Module: U:\extras\lib\libcrypto.lib(tasn_enc.obj)
0001:00044980  _ASN1_item_ndef_i2d
0001:000449a9  _ASN1_item_i2d
0001:00044ac4  _ASN1_item_ex_i2d
0001:00044fec* _ASN1_template_i2d
0001:000457d1* _asn1_ex_i2c
Module: U:\extras\lib\libcrypto.lib(tasn_new.obj)
0001:00045a80  _ASN1_item_new
0001:00045aaf  _ASN1_item_ex_new
0001:00046000* _ASN1_template_new
0001:00046116* _ASN1_primitive_new
Module: U:\extras\lib\libcrypto.lib(tasn_fre.obj)
0001:00046310  _ASN1_item_free
0001:00046332  _ASN1_item_ex_free
0001:000466e6  _ASN1_template_free
0001:0004678c  _ASN1_primitive_free
Module: U:\extras\lib\libcrypto.lib(x_x509a.obj)
0001:00046970* _X509_CERT_AUX_it
0001:0004698c  _d2i_X509_CERT_AUX
0001:000469b5  _i2d_X509_CERT_AUX
0001:000469d7* _X509_CERT_AUX_new
0001:000469eb  _X509_CERT_AUX_free
0001:00046a47* _X509_alias_set1
0001:00046afe* _X509_keyid_set1
0001:00046bb5* _X509_alias_get0
0001:00046bfa* _X509_keyid_get0
0001:00046c3f* _X509_add1_trust_object
0001:00046cb6* _X509_add1_reject_object
0001:00046d31* _X509_trust_clear
0001:00046d74* _X509_reject_clear
0001:00046e10* _X509_CERT_PAIR_it
0001:00046e2c  _d2i_X509_CERT_PAIR
0001:00046e55  _i2d_X509_CERT_PAIR
0001:00046e77* _X509_CERT_PAIR_new
0001:00046e8b* _X509_CERT_PAIR_free
Module: U:\extras\lib\libcrypto.lib(v3_akeya.obj)
0001:00046f20  _AUTHORITY_KEYID_it
0001:00046f3c* _d2i_AUTHORITY_KEYID
0001:00046f65* _i2d_AUTHORITY_KEYID
0001:00046f87  _AUTHORITY_KEYID_new
0001:00046f9b  _AUTHORITY_KEYID_free
Module: U:\extras\lib\libcrypto.lib(v3_crld.obj)
0001:00046fc0  _v3_crld
0001:00047d30* _CRL_DIST_POINTS_it
0001:00047000  _v3_freshest_crl
0001:00047bc7* _DIST_POINT_NAME_new
0001:00047cb7* _DIST_POINT_new
0001:00047ccb* _DIST_POINT_free
0001:00047b60* _DIST_POINT_NAME_it
0001:00047b7c* _d2i_DIST_POINT_NAME
0001:00047ba5* _i2d_DIST_POINT_NAME
0001:00047bdb* _DIST_POINT_NAME_free
0001:00047c50* _DIST_POINT_it
0001:00047c6c* _d2i_DIST_POINT
0001:00047c95* _i2d_DIST_POINT
0001:00047d4c* _d2i_CRL_DIST_POINTS
0001:00047d75* _i2d_CRL_DIST_POINTS
0001:00047d97* _CRL_DIST_POINTS_new
0001:00047dab  _CRL_DIST_POINTS_free
0001:00047e90* _ISSUING_DIST_POINT_it
0001:00047eac* _d2i_ISSUING_DIST_POINT
0001:00047ed5* _i2d_ISSUING_DIST_POINT
0001:00047ef7* _ISSUING_DIST_POINT_new
0001:00047f0b  _ISSUING_DIST_POINT_free
0001:00047f30  _v3_idp
0001:0004866a  _DIST_POINT_set_dpname
Module: U:\extras\lib\libcrypto.lib(pcy_cache.obj)
0001:00048b9a  _policy_cache_free
0001:00048bed  _policy_cache_set
0001:00048c58  _policy_cache_find_data
Module: U:\extras\lib\libcrypto.lib(v3_genn.obj)
0001:00048d60* _OTHERNAME_it
0001:00048d7c* _d2i_OTHERNAME
0001:00048da5* _i2d_OTHERNAME
0001:00048dc7  _OTHERNAME_new
0001:00048ddb* _OTHERNAME_free
0001:00048e50* _EDIPARTYNAME_it
0001:00048e6c* _d2i_EDIPARTYNAME
0001:00048e95* _i2d_EDIPARTYNAME
0001:00048eb7* _EDIPARTYNAME_new
0001:00048ecb* _EDIPARTYNAME_free
0001:00049040  _GENERAL_NAME_it
0001:0004905c* _d2i_GENERAL_NAME
0001:00049085* _i2d_GENERAL_NAME
0001:000490a7  _GENERAL_NAME_new
0001:000490bb  _GENERAL_NAME_free
0001:00049120  _GENERAL_NAMES_it
0001:0004913c* _d2i_GENERAL_NAMES
0001:00049165* _i2d_GENERAL_NAMES
0001:00049187  _GENERAL_NAMES_new
0001:0004919b  _GENERAL_NAMES_free
0001:000491b6* _GENERAL_NAME_dup
0001:000491db  _GENERAL_NAME_cmp
0001:000492fd* _OTHERNAME_cmp
0001:00049361* _GENERAL_NAME_set0_value
0001:000493eb* _GENERAL_NAME_get0_value
0001:0004946f* _GENERAL_NAME_set0_othername
0001:000494bc* _GENERAL_NAME_get0_otherName
Module: U:\extras\lib\libcrypto.lib(v3_ncons.obj)
0001:00049500  _v3_name_constraints
0001:00049620* _NAME_CONSTRAINTS_it
0001:000495a0* _GENERAL_SUBTREE_it
0001:0004963c* _GENERAL_SUBTREE_new
0001:00049650* _GENERAL_SUBTREE_free
0001:0004966b* _NAME_CONSTRAINTS_new
0001:0004967f  _NAME_CONSTRAINTS_free
0001:00049bd8  _NAME_CONSTRAINTS_check
Module: U:\extras\lib\libcrypto.lib(a_dup.obj)
0001:0004a2d8  _ASN1_dup
0001:0004a3ac  _ASN1_item_dup
Module: U:\extras\lib\libcrypto.lib(asn1_lib.obj)
0001:0004a460* _ASN1_version
0001:0004a4d0* _ASN1_check_infinite_end
0001:0004a4ea  _ASN1_const_check_infinite_end
0001:0004a50f  _ASN1_get_object
0001:0004a7d1  _ASN1_put_object
0001:0004a8d1  _ASN1_put_eoc
0001:0004a984  _ASN1_object_size
0001:0004aa5e* _asn1_Finish
0001:0004aa71  _asn1_const_Finish
0001:0004aa84  _asn1_GetSequence
0001:0004ab89  _ASN1_STRING_copy
0001:0004ac39  _ASN1_STRING_set
0001:0004abe4  _ASN1_STRING_dup
0001:0004ad98  _ASN1_STRING_new
0001:0004ae35  _ASN1_STRING_free
0001:0004ad67  _ASN1_STRING_set0
0001:0004adac  _ASN1_STRING_type_new
0001:0004ae76  _ASN1_STRING_cmp
0001:0004aef8  _asn1_add_error
0001:0004af6e* _ASN1_STRING_length
0001:0004af78* _ASN1_STRING_length_set
0001:0004af85* _ASN1_STRING_type
0001:0004af90  _ASN1_STRING_data
Module: U:\extras\lib\libcrypto.lib(m_md5.obj)
0001:0004b04c  _EVP_md5
Module: U:\extras\lib\libcrypto.lib(m_sha1.obj)
0001:0004b10c  _EVP_sha1
0001:0004b1dc  _EVP_sha224
0001:0004b23c  _EVP_sha256
0001:0004b30c  _EVP_sha384
0001:0004b36c  _EVP_sha512
Module: U:\extras\lib\libcrypto.lib(a_object.obj)
0001:0004b380* _i2d_ASN1_OBJECT
0001:0004b449  _a2d_ASN1_OBJECT
0001:0004b8e0  _i2t_ASN1_OBJECT
0001:0004b918  _i2a_ASN1_OBJECT
0001:0004ba13  _d2i_ASN1_OBJECT
0001:0004bad9  _c2i_ASN1_OBJECT
0001:0004bce1  _ASN1_OBJECT_new
0001:0004bd7f  _ASN1_OBJECT_free
0001:0004be35  _ASN1_OBJECT_create
Module: U:\extras\lib\libcrypto.lib(err_all.obj)
0001:0004be70  _ERR_load_crypto_strings
Module: U:\extras\lib\libssl.lib(ssl_err.obj)
0001:0004ea59  _ERR_load_SSL_strings
Module: U:\extras\lib\libcrypto.lib(e_des.obj)
0001:0004ef74  _EVP_des_cbc
0001:0004efb4  _EVP_des_cfb64
0001:0004eff4  _EVP_des_ofb
0001:0004f034  _EVP_des_ecb
0001:0004f074  _EVP_des_cfb1
0001:0004f0b4  _EVP_des_cfb8
Module: U:\extras\lib\libcrypto.lib(e_des3.obj)
0001:0004f704  _EVP_des_ede_cbc
0001:0004f744  _EVP_des_ede_cfb64
0001:0004f784  _EVP_des_ede_ofb
0001:0004f7c4* _EVP_des_ede_ecb
0001:0004f804  _EVP_des_ede3_cbc
0001:0004f844  _EVP_des_ede3_cfb64
0001:0004f884  _EVP_des_ede3_ofb
0001:0004f8c4* _EVP_des_ede3_ecb
0001:0004f904  _EVP_des_ede3_cfb1
0001:0004f944  _EVP_des_ede3_cfb8
0001:0004fa9d  _EVP_des_ede
0001:0004faa7  _EVP_des_ede3
Module: U:\extras\lib\libcrypto.lib(e_idea.obj)
0001:0004fd54  _EVP_idea_cbc
0001:0004fd94  _EVP_idea_cfb64
0001:0004fdd4  _EVP_idea_ofb
0001:0004fe14  _EVP_idea_ecb
Module: U:\extras\lib\libcrypto.lib(e_rc4.obj)
0001:0004ff44  _EVP_rc4
0001:0004ff4e  _EVP_rc4_40
Module: U:\extras\lib\libcrypto.lib(e_rc2.obj)
0001:00050274  _EVP_rc2_cbc
0001:000502b4  _EVP_rc2_cfb64
0001:000502f4  _EVP_rc2_ofb
0001:00050334  _EVP_rc2_ecb
0001:000503b4  _EVP_rc2_64_cbc
0001:000503be  _EVP_rc2_40_cbc
Module: U:\extras\lib\libcrypto.lib(e_aes.obj)
0001:00050964  _EVP_aes_128_cbc
0001:000509a4  _EVP_aes_128_cfb128
0001:000509e4  _EVP_aes_128_ofb
0001:00050a24  _EVP_aes_128_ecb
0001:00050cc4  _EVP_aes_192_cbc
0001:00050d04  _EVP_aes_192_cfb128
0001:00050d44  _EVP_aes_192_ofb
0001:00050d84  _EVP_aes_192_ecb
0001:00051024  _EVP_aes_256_cbc
0001:00051064  _EVP_aes_256_cfb128
0001:000510a4  _EVP_aes_256_ofb
0001:000510e4  _EVP_aes_256_ecb
0001:000511e4  _EVP_aes_128_cfb1
0001:000512e4  _EVP_aes_192_cfb1
0001:000513e4  _EVP_aes_256_cfb1
0001:000514c4  _EVP_aes_128_cfb8
0001:000515a4  _EVP_aes_192_cfb8
0001:00051684  _EVP_aes_256_cfb8
Module: U:\extras\lib\libcrypto.lib(e_camellia.obj)
0001:000519f4  _EVP_camellia_128_cbc
0001:00051a34  _EVP_camellia_128_cfb128
0001:00051a74  _EVP_camellia_128_ofb
0001:00051ab4  _EVP_camellia_128_ecb
0001:00051d54  _EVP_camellia_192_cbc
0001:00051d94  _EVP_camellia_192_cfb128
0001:00051dd4  _EVP_camellia_192_ofb
0001:00051e14  _EVP_camellia_192_ecb
0001:000520b4  _EVP_camellia_256_cbc
0001:000520f4  _EVP_camellia_256_cfb128
0001:00052134  _EVP_camellia_256_ofb
0001:00052174  _EVP_camellia_256_ecb
0001:00052274  _EVP_camellia_128_cfb1
0001:00052374  _EVP_camellia_192_cfb1
0001:00052474  _EVP_camellia_256_cfb1
0001:00052554  _EVP_camellia_128_cfb8
0001:00052634  _EVP_camellia_192_cfb8
0001:00052714  _EVP_camellia_256_cfb8
Module: U:\extras\lib\libcrypto.lib(e_seed.obj)
0001:00052a34  _EVP_seed_cbc
0001:00052a74  _EVP_seed_cfb128
0001:00052ab4  _EVP_seed_ofb
0001:00052af4  _EVP_seed_ecb
Module: U:\extras\lib\libcrypto.lib(o_names.obj)
0001:00052b5f* _OBJ_NAME_init
0001:00052bbf* _OBJ_NAME_new_index
0001:00052e4e  _OBJ_NAME_get
0001:00052ef9  _OBJ_NAME_add
0001:0005301e* _OBJ_NAME_remove
0001:0005312f  _OBJ_NAME_do_all
0001:000531d6  _OBJ_NAME_do_all_sorted
0001:000532fa  _OBJ_NAME_cleanup
Module: U:\extras\lib\libcrypto.lib(m_dss1.obj)
0001:0005343c  _EVP_dss1
Module: U:\extras\lib\libcrypto.lib(m_ecdsa.obj)
0001:000534fc  _EVP_ecdsa
Module: U:\extras\lib\libcrypto.lib(c_allc.obj)
0001:00053685  _OpenSSL_add_all_ciphers
Module: U:\extras\lib\libcrypto.lib(c_alld.obj)
0001:00053e51  _OpenSSL_add_all_digests
Module: U:\extras\lib\libcrypto.lib(x_all.obj)
0001:00054010  _X509_verify
0001:0005404d* _X509_REQ_verify
0001:0005408a* _NETSCAPE_SPKI_verify
0001:000540c7* _X509_sign
0001:00054125  _X509_REQ_sign
0001:00054171* _X509_CRL_sign
0001:000541cf* _NETSCAPE_SPKI_sign
0001:0005421b* _d2i_X509_fp
0001:0005423d* _i2d_X509_fp
0001:0005425f  _d2i_X509_bio
0001:00054281* _i2d_X509_bio
0001:000542a3* _d2i_X509_CRL_fp
0001:000542c5* _i2d_X509_CRL_fp
0001:000542e7  _d2i_X509_CRL_bio
0001:00054309* _i2d_X509_CRL_bio
0001:0005432b* _d2i_PKCS7_fp
0001:0005434d* _i2d_PKCS7_fp
0001:0005436f* _d2i_PKCS7_bio
0001:00054391* _i2d_PKCS7_bio
0001:000543b3* _d2i_X509_REQ_fp
0001:000543d5* _i2d_X509_REQ_fp
0001:000543f7* _d2i_X509_REQ_bio
0001:00054419* _i2d_X509_REQ_bio
0001:0005443b* _d2i_RSAPrivateKey_fp
0001:0005445d* _i2d_RSAPrivateKey_fp
0001:0005447f* _d2i_RSAPublicKey_fp
0001:000544a1* _d2i_RSA_PUBKEY_fp
0001:000544cd* _i2d_RSAPublicKey_fp
0001:000544ef* _i2d_RSA_PUBKEY_fp
0001:00054512  _d2i_RSAPrivateKey_bio
0001:00054534* _i2d_RSAPrivateKey_bio
0001:00054556* _d2i_RSAPublicKey_bio
0001:00054578* _d2i_RSA_PUBKEY_bio
0001:000545a4* _i2d_RSAPublicKey_bio
0001:000545c6* _i2d_RSA_PUBKEY_bio
0001:000545e9* _d2i_DSAPrivateKey_fp
0001:00054615* _i2d_DSAPrivateKey_fp
0001:00054638* _d2i_DSA_PUBKEY_fp
0001:00054664* _i2d_DSA_PUBKEY_fp
0001:00054687* _d2i_DSAPrivateKey_bio
0001:000546b3* _i2d_DSAPrivateKey_bio
0001:000546d6* _d2i_DSA_PUBKEY_bio
0001:00054702* _i2d_DSA_PUBKEY_bio
0001:00054725* _d2i_EC_PUBKEY_fp
0001:00054751* _i2d_EC_PUBKEY_fp
0001:00054774* _d2i_ECPrivateKey_fp
0001:000547a0* _i2d_ECPrivateKey_fp
0001:000547c3* _d2i_EC_PUBKEY_bio
0001:000547ef* _i2d_EC_PUBKEY_bio
0001:00054812* _d2i_ECPrivateKey_bio
0001:0005483e* _i2d_ECPrivateKey_bio
0001:00054861* _X509_pubkey_digest
0001:000548ba  _X509_digest
0001:000548ea  _X509_CRL_digest
0001:0005491a* _X509_REQ_digest
0001:0005494a* _X509_NAME_digest
0001:0005497a* _PKCS7_ISSUER_AND_SERIAL_digest
0001:000549aa* _d2i_PKCS8_fp
0001:000549d6* _i2d_PKCS8_fp
0001:000549f9  _d2i_PKCS8_bio
0001:00054a25  _i2d_PKCS8_bio
0001:00054a48* _d2i_PKCS8_PRIV_KEY_INFO_fp
0001:00054a74* _i2d_PKCS8_PRIV_KEY_INFO_fp
0001:00054a97* _i2d_PKCS8PrivateKeyInfo_fp
0001:00054add* _i2d_PrivateKey_fp
0001:00054b00* _d2i_PrivateKey_fp
0001:00054b2c* _i2d_PUBKEY_fp
0001:00054b4f* _d2i_PUBKEY_fp
0001:00054b7b* _d2i_PKCS8_PRIV_KEY_INFO_bio
0001:00054ba7  _i2d_PKCS8_PRIV_KEY_INFO_bio
0001:00054bca* _i2d_PKCS8PrivateKeyInfo_bio
0001:00054c10* _i2d_PrivateKey_bio
0001:00054c33  _d2i_PrivateKey_bio
0001:00054c5f* _i2d_PUBKEY_bio
0001:00054c82* _d2i_PUBKEY_bio
Module: U:\extras\lib\libcrypto.lib(pem_x509.obj)
0001:00054cbc  _PEM_read_bio_X509
0001:00054cf5* _PEM_read_X509
0001:00054d2e  _PEM_write_bio_X509
0001:00054d81* _PEM_write_X509
Module: U:\extras\lib\libssl.lib(s3_both.obj)
0001:00054de0  _ssl3_do_write
0001:00054f17  _ssl3_send_finished
0001:000550e0  _ssl3_get_finished
0001:0005532b  _ssl3_send_change_cipher_spec
0001:0005545c  _ssl3_output_cert_chain
0001:00055720  _ssl3_get_message
0001:00055c3a  _ssl_cert_type
0001:00055cee  _ssl_verify_alarm_type
0001:00056016  _ssl3_setup_read_buffer
0001:00056157  _ssl3_setup_write_buffer
0001:00056287  _ssl3_setup_buffers
0001:000562c0  _ssl3_release_write_buffer
0001:00056326  _ssl3_release_read_buffer
Module: U:\extras\lib\libcrypto.lib(pem_all.obj)
0001:000563a4* _PEM_read_bio_X509_REQ
0001:000563dd* _PEM_read_X509_REQ
0001:00056416* _PEM_write_bio_X509_REQ
0001:00056469* _PEM_write_X509_REQ
0001:000564d4* _PEM_write_bio_X509_REQ_NEW
0001:00056527* _PEM_write_X509_REQ_NEW
0001:00056583  _PEM_read_bio_X509_CRL
0001:000565bc* _PEM_read_X509_CRL
0001:000565f5* _PEM_write_bio_X509_CRL
0001:00056648* _PEM_write_X509_CRL
0001:000566a1* _PEM_read_bio_PKCS7
0001:000566da* _PEM_read_PKCS7
0001:00056713* _PEM_write_bio_PKCS7
0001:00056766* _PEM_write_PKCS7
0001:000567c5* _PEM_read_bio_NETSCAPE_CERT_SEQUENCE
0001:000567fe* _PEM_read_NETSCAPE_CERT_SEQUENCE
0001:00056837* _PEM_write_bio_NETSCAPE_CERT_SEQUENCE
0001:0005688a* _PEM_write_NETSCAPE_CERT_SEQUENCE
0001:00056936  _PEM_read_bio_RSAPrivateKey
0001:00056974* _PEM_read_RSAPrivateKey
0001:000569c2  _PEM_write_bio_RSAPrivateKey
0001:00056a10* _PEM_write_RSAPrivateKey
0001:00056a6d* _PEM_read_bio_RSAPublicKey
0001:00056aa6* _PEM_read_RSAPublicKey
0001:00056adf* _PEM_write_bio_RSAPublicKey
0001:00056b32* _PEM_write_RSAPublicKey
0001:00056b90* _PEM_read_bio_RSA_PUBKEY
0001:00056bc9* _PEM_read_RSA_PUBKEY
0001:00056c02* _PEM_write_bio_RSA_PUBKEY
0001:00056c55* _PEM_write_RSA_PUBKEY
0001:00056d01* _PEM_read_bio_DSAPrivateKey
0001:00056d4f* _PEM_write_bio_DSAPrivateKey
0001:00056d9d* _PEM_write_DSAPrivateKey
0001:00056deb* _PEM_read_bio_DSA_PUBKEY
0001:00056e24* _PEM_read_DSA_PUBKEY
0001:00056e5d* _PEM_write_bio_DSA_PUBKEY
0001:00056eb0* _PEM_write_DSA_PUBKEY
0001:00056f03* _PEM_read_DSAPrivateKey
0001:00056f50* _PEM_read_bio_DSAparams
0001:00056f89* _PEM_read_DSAparams
0001:00056fc2* _PEM_write_bio_DSAparams
0001:00057015* _PEM_write_DSAparams
0001:000570c1* _PEM_read_bio_ECPrivateKey
0001:0005710d* _PEM_read_bio_ECPKParameters
0001:00057146* _PEM_read_ECPKParameters
0001:0005717f* _PEM_write_bio_ECPKParameters
0001:000571d2* _PEM_write_ECPKParameters
0001:00057234* _PEM_write_bio_ECPrivateKey
0001:00057282* _PEM_write_ECPrivateKey
0001:000572d0* _PEM_read_bio_EC_PUBKEY
0001:00057309* _PEM_read_EC_PUBKEY
0001:00057342* _PEM_write_bio_EC_PUBKEY
0001:00057395* _PEM_write_EC_PUBKEY
0001:000573e8* _PEM_read_ECPrivateKey
0001:00057434* _PEM_read_bio_DHparams
0001:0005746d* _PEM_read_DHparams
0001:000574a6* _PEM_write_bio_DHparams
0001:000574f9* _PEM_write_DHparams
0001:0005754c* _PEM_read_bio_PUBKEY
0001:00057585* _PEM_read_PUBKEY
0001:000575be* _PEM_write_bio_PUBKEY
0001:00057611* _PEM_write_PUBKEY
Module: U:\extras\lib\libcrypto.lib(rsa_asn1.obj)
0001:000577d0  _RSAPrivateKey_it
0001:00057840  _RSAPublicKey_it
0001:0005785c  _d2i_RSAPrivateKey
0001:00057885  _i2d_RSAPrivateKey
0001:000578a7  _d2i_RSAPublicKey
0001:000578d0  _i2d_RSAPublicKey
0001:000578f2* _RSAPublicKey_dup
0001:0005790d  _RSAPrivateKey_dup
Module: U:\extras\lib\libcrypto.lib(pem_pkey.obj)
0001:0005796d  _PEM_read_bio_PrivateKey
0001:00057c92* _PEM_write_bio_PrivateKey
0001:00057d63* _PEM_read_bio_Parameters
0001:00057ee6* _PEM_write_bio_Parameters
0001:00057f85  _PEM_read_PrivateKey
0001:00058029* _PEM_write_PrivateKey
Module: U:\extras\lib\libcrypto.lib(d2i_pr.obj)
0001:000580d9  _d2i_PrivateKey
0001:0005829e  _d2i_AutoPrivateKey
Module: U:\extras\lib\libssl.lib(s2_lib.obj)
0001:000583f0* _ssl2_version_str
0001:00058470* _ssl2_ciphers
0001:000585c0  _ssl2_default_timeout
0001:000585ca  _ssl2_num_ciphers
0001:000585d4  _ssl2_get_cipher
0001:000585fe  _ssl2_pending
0001:00058633  _ssl2_new
0001:000587b5  _ssl2_clear
0001:00058743  _ssl2_free
0001:0005882e  _ssl2_ctrl
0001:00058854  _ssl2_callback_ctrl
0001:0005885e  _ssl2_ctx_ctrl
0001:00058868  _ssl2_ctx_callback_ctrl
0001:00058872  _ssl2_get_cipher_by_char
0001:000588e7  _ssl2_put_cipher_by_char
0001:000589aa  _ssl2_generate_key_material
0001:00058be8  _ssl2_return_error
0001:00058c4c  _ssl2_write_error
0001:00058d56  _ssl2_shutdown
Module: U:\extras\lib\libssl.lib(s2_srvr.obj)
0001:00058d8a  _SSLv2_server_method
0001:00058d9e  _ssl2_accept
Module: U:\extras\lib\libssl.lib(s2_clnt.obj)
0001:0005b4ba  _SSLv2_client_method
0001:0005b4ce  _ssl2_connect
0001:0005d666* _ssl2_set_certificate
Module: U:\extras\lib\libssl.lib(s2_pkt.obj)
0001:0005e0ee  _ssl2_read
0001:0005e117  _ssl2_peek
0001:0005e418  _ssl2_write
0001:0005eacb  _ssl2_part_read
0001:0005eba7  _ssl2_do_write
Module: U:\extras\lib\libssl.lib(s3_lib.obj)
0001:0005ece0* _ssl3_version_str
0001:0005f388  _ssl3_default_timeout
0001:0005f392  _ssl3_num_ciphers
0001:0005f39c  _ssl3_get_cipher
0001:0005f3c6  _ssl3_pending
0001:0005f40c  _ssl3_new
0001:0005f4bb  _ssl3_free
0001:0005f617  _ssl3_clear
0001:0005f816  _ssl3_ctrl
0001:0006005b  _ssl3_callback_ctrl
0001:00060120  _ssl3_ctx_ctrl
0001:00060770  _ssl3_ctx_callback_ctrl
0001:00060805  _ssl3_get_cipher_by_char
0001:0006086a  _ssl3_put_cipher_by_char
0001:000608b4  _ssl3_choose_cipher
0001:00060fd4  _ssl3_get_req_cert_type
0001:000610de  _ssl3_shutdown
0001:00061210  _ssl3_write
0001:000614e6  _ssl3_renegotiate_check
0001:00061453  _ssl3_read
0001:0006147c  _ssl3_peek
0001:000614a5  _ssl3_renegotiate
0002:00001f10* _ssl3_ciphers
0002:00002ff0  _SSLv3_enc_data
Module: U:\extras\lib\libssl.lib(s3_srvr.obj)
0001:000615ad  _SSLv3_server_method
0001:000615c1  _ssl3_accept
0001:000624de* _ssl3_send_hello_request
0001:00062609* _ssl3_get_client_hello
0001:000634ef* _ssl3_send_server_hello
0001:00066a6a* _ssl3_send_server_certificate
0001:00063800* _ssl3_send_server_key_exchange
0001:00064914* _ssl3_send_certificate_request
0001:0006378a* _ssl3_send_server_done
0001:00062554* _ssl3_check_client_hello
0001:000663ff* _ssl3_get_client_certificate
0001:00064bfd* _ssl3_get_client_key_exchange
0001:00065dc4* _ssl3_get_cert_verify
0001:00066b39* _ssl3_send_newsession_ticket
0001:00066fa9* _ssl3_send_cert_status
Module: U:\extras\lib\libssl.lib(s3_clnt.obj)
0001:0006719d  _SSLv3_client_method
0001:000671b1  _ssl3_connect
0001:00067e0e* _ssl3_client_hello
0001:0006824f* _ssl3_get_server_hello
0001:0006cf11* _ssl3_check_finished
0001:00068a6d* _ssl3_get_server_certificate
0001:00069175* _ssl3_get_key_exchange
0001:0006ca75* _ssl3_check_cert_and_algorithm
0001:0006a4d9* _ssl3_get_certificate_request
0001:0006b045* _ssl3_get_server_done
0001:0006c82c* _ssl3_send_client_certificate
0001:0006b0f9* _ssl3_send_client_key_exchange
0001:0006c382* _ssl3_send_client_verify
0001:0006aa0a* _ssl3_get_new_session_ticket
0001:0006ad85* _ssl3_get_cert_status
0001:0006cfc0* _ssl_do_client_cert_cb
Module: U:\extras\lib\libssl.lib(t1_lib.obj)
0001:0006d100* _tls1_version_str
0001:0006d148  _tls1_default_timeout
0001:0006d152  _tls1_new
0001:0006d186  _tls1_free
0001:0006d1b7  _tls1_clear
0001:0006d1d3  _tls1_ec_curve_id2nid
0001:0006d1f8  _tls1_ec_nid2curve_id
0001:0006d426  _ssl_add_clienthello_tlsext
0001:0006dd9d  _ssl_add_serverhello_tlsext
0001:0006e24c  _ssl_parse_clienthello_tlsext
0001:0006eca1  _ssl_parse_serverhello_tlsext
0001:0006f17a  _ssl_prepare_clienthello_tlsext
0001:0006f3c6  _ssl_prepare_serverhello_tlsext
0001:0006f508  _ssl_check_clienthello_tlsext
0001:0006f703  _ssl_check_serverhello_tlsext
0001:0006fa27  _tls1_process_ticket
0002:00003030  _TLSv1_enc_data
Module: U:\extras\lib\libssl.lib(s23_srvr.obj)
0001:0007006a* _SSLv23_server_method
0001:0007007f  _ssl23_accept
0001:00070361* _ssl23_get_client_hello
Module: U:\extras\lib\libssl.lib(s23_clnt.obj)
0001:00070eca* _SSLv23_client_method
0001:00070edf  _ssl23_connect
Module: U:\extras\lib\libssl.lib(s23_lib.obj)
0001:00072180  _ssl23_default_timeout
0001:0007218a  _ssl23_num_ciphers
0001:000721a6  _ssl23_get_cipher
0001:000721df  _ssl23_get_cipher_by_char
0001:0007220c  _ssl23_put_cipher_by_char
0001:00072258  _ssl23_read
0001:00072309  _ssl23_peek
0001:000723ba  _ssl23_write
Module: U:\extras\lib\libcrypto.lib(obj_lib.obj)
0001:0007247a  _OBJ_dup
0001:000726e7  _OBJ_cmp
Module: U:\extras\lib\libcrypto.lib(bn_word.obj)
0001:00072740  _BN_mod_word
0001:000727c4  _BN_div_word
0001:000728e4  _BN_add_word
0001:00072a3c  _BN_sub_word
0001:00072bb6  _BN_mul_word
Module: U:\extras\lib\libcrypto.lib(bn_lib.obj)
0001:00072c90* _BN_version
0001:00072cbd* _BN_set_params
0001:00072d84* _BN_get_params
0001:00072dc2  _BN_value_one
0001:00072dd6* _BN_options
0001:00072e23  _BN_num_bits_word
0001:00072e94  _BN_num_bits
0001:00072ede  _BN_clear_free
0001:00072f60  _BN_free
0001:00072fc8  _BN_init
0001:00072ff4  _BN_new
0001:00073246* _bn_dup_expand
0001:00073331  _BN_dup
0001:000732d2  _bn_expand2
0001:00073386  _BN_copy
0001:000734bf* _BN_swap
0001:00073579  _BN_clear
0001:000735c4* _BN_get_word
0001:000735f4  _BN_set_word
0001:0007365b  _BN_bin2bn
0001:000737ca  _BN_bn2bin
0001:00073851  _BN_ucmp
0001:000738dd  _BN_cmp
0001:000739f3  _BN_set_bit
0001:00073aeb* _BN_clear_bit
0001:00073bc0  _BN_is_bit_set
0001:00073c2d  _BN_mask_bits
0001:00073d22  _BN_set_negative
0001:00073d4d  _bn_cmp_words
0001:00073de4  _bn_cmp_part_words
Module: U:\extras\lib\libcrypto.lib(bn_shift.obj)
0001:00073fa0  _BN_lshift1
0001:000740bb  _BN_rshift1
0001:000741fc  _BN_lshift
0001:000743e1  _BN_rshift
Module: U:\extras\lib\libcrypto.lib(bn_print.obj)
0001:0007464c* _BN_bn2hex
0001:00074780  _BN_bn2dec
0001:00074a03  _BN_hex2bn
0001:00074c78  _BN_dec2bn
0001:00074eaa  _BN_asc2bn
0001:00074f38* _BN_print_fp
0001:00074fa6* _BN_print
Module: U:\extras\lib\libcrypto.lib(a_utf8.obj)
0001:000750b0  _UTF8_getc
0001:00075560  _UTF8_putc
Module: U:\extras\lib\libcrypto.lib(asn1_par.obj)
0001:000765cb  _ASN1_tag2str
0001:000759be* _ASN1_parse
0001:000759fe  _ASN1_parse_dump
Module: U:\extras\lib\libcrypto.lib(a_mbstr.obj)
0001:000767e0  _ASN1_mbstring_copy
0001:0007683f  _ASN1_mbstring_ncopy
Module: U:\extras\lib\libcrypto.lib(mem_clr.obj)
0001:00077200  _OPENSSL_cleanse
0002:00009500  _cleanse_ctr
Module: U:\extras\lib\libcrypto.lib(a_strnid.obj)
0001:00077290* _ASN1_STRING_set_default_mask
0001:0007729d* _ASN1_STRING_get_default_mask
0001:000772cb* _ASN1_STRING_set_default_mask_asc
0001:000773d6  _ASN1_STRING_set_by_NID
0001:000776b1* _ASN1_STRING_TABLE_get
0001:0007773b* _ASN1_STRING_TABLE_add
0001:00077887* _ASN1_STRING_TABLE_cleanup
Module: U:\extras\lib\libcrypto.lib(a_print.obj)
0001:000778e0  _ASN1_PRINTABLE_type
0001:000779ee* _ASN1_UNIVERSALSTRING_to_string
Module: U:\extras\lib\libcrypto.lib(err_prn.obj)
0001:00077b02  _ERR_print_errors_cb
0001:00077c75* _ERR_print_errors_fp
0001:00077cb1  _ERR_print_errors
Module: U:\extras\lib\libcrypto.lib(v3_prn.obj)
0001:00077ce9* _X509V3_EXT_val_prn
0001:00077e5a* _X509V3_EXT_print
0001:000780cd  _X509V3_extensions_print
0001:000783a6* _X509V3_EXT_print_fp
Module: U:\extras\lib\libcrypto.lib(t_x509a.obj)
0001:0007848f  _X509_CERT_AUX_print
Module: U:\extras\lib\libcrypto.lib(x509_v3.obj)
0001:00078790  _X509v3_get_ext_count
0001:000787b0  _X509v3_get_ext_by_NID
0001:000787ec  _X509v3_get_ext_by_OBJ
0001:00078863  _X509v3_get_ext_by_critical
0001:000788e2  _X509v3_get_ext
0001:0007891f  _X509v3_delete_ext
0001:0007896c  _X509v3_add_ext
0001:00078aa2  _X509_EXTENSION_create_by_NID
0001:00078b28  _X509_EXTENSION_create_by_OBJ
0001:00078c10* _X509_EXTENSION_set_object
0001:00078c4d* _X509_EXTENSION_set_critical
0001:00078c7c* _X509_EXTENSION_set_data
0001:00078cc7  _X509_EXTENSION_get_object
0001:00078cde  _X509_EXTENSION_get_data
0001:00078cf6  _X509_EXTENSION_get_critical
Module: U:\extras\lib\libcrypto.lib(v3_bitst.obj)
0001:00078ec0  _v3_nscert
0001:00078f38* _i2v_ASN1_BIT_STRING
0001:00078fb4* _v2i_ASN1_BIT_STRING
0001:00078f00  _v3_key_usage
Module: U:\extras\lib\libcrypto.lib(v3_ia5.obj)
0001:00079190  _v3_ns_ia5_list
Module: U:\extras\lib\libcrypto.lib(v3_skey.obj)
0001:000794d0  _v3_skey_id
0001:00079508* _i2s_ASN1_OCTET_STRING
0001:00079531* _s2i_ASN1_OCTET_STRING
Module: U:\extras\lib\libcrypto.lib(v3_pku.obj)
0001:000797b0  _v3_pkey_usage_period
0001:00079840* _PKEY_USAGE_PERIOD_it
0001:0007985c* _d2i_PKEY_USAGE_PERIOD
0001:00079885* _i2d_PKEY_USAGE_PERIOD
0001:000798a7* _PKEY_USAGE_PERIOD_new
0001:000798bb* _PKEY_USAGE_PERIOD_free
Module: U:\extras\lib\libcrypto.lib(v3_bcons.obj)
0001:000799c0  _v3_bcons
0001:00079a50* _BASIC_CONSTRAINTS_it
0001:00079a6c* _d2i_BASIC_CONSTRAINTS
0001:00079a95* _i2d_BASIC_CONSTRAINTS
0001:00079ab7* _BASIC_CONSTRAINTS_new
0001:00079acb  _BASIC_CONSTRAINTS_free
Module: U:\extras\lib\libcrypto.lib(v3_int.obj)
0001:00079cd0  _v3_crl_num
0001:00079d10  _v3_delta_crl
0001:00079d70  _v3_inhibit_anyp
Module: U:\extras\lib\libcrypto.lib(v3_cpols.obj)
0001:00079db0  _v3_cpols
0001:00079e20* _CERTIFICATEPOLICIES_it
0001:00079f10* _POLICYINFO_it
0001:00079e3c* _d2i_CERTIFICATEPOLICIES
0001:00079e65* _i2d_CERTIFICATEPOLICIES
0001:00079e87* _CERTIFICATEPOLICIES_new
0001:00079e9b* _CERTIFICATEPOLICIES_free
0001:0007a080* _POLICYQUALINFO_it
0001:00079f2c* _d2i_POLICYINFO
0001:00079f55* _i2d_POLICYINFO
0001:00079f77* _POLICYINFO_new
0001:00079f8b  _POLICYINFO_free
0001:0007a170* _USERNOTICE_it
0001:0007a09c* _d2i_POLICYQUALINFO
0001:0007a0c5* _i2d_POLICYQUALINFO
0001:0007a0e7* _POLICYQUALINFO_new
0001:0007a0fb  _POLICYQUALINFO_free
0001:0007a260* _NOTICEREF_it
0001:0007a18c* _d2i_USERNOTICE
0001:0007a1b5* _i2d_USERNOTICE
0001:0007a1d7* _USERNOTICE_new
0001:0007a1eb* _USERNOTICE_free
0001:0007a27c* _d2i_NOTICEREF
0001:0007a2a5* _i2d_NOTICEREF
0001:0007a2c7* _NOTICEREF_new
0001:0007a2db* _NOTICEREF_free
0001:0007b3cd* _X509_POLICY_NODE_print
Module: U:\extras\lib\libcrypto.lib(v3_akey.obj)
0001:0007b4c0  _v3_akey_id
Module: U:\extras\lib\libcrypto.lib(v3_extku.obj)
0001:0007b9a0  _v3_ext_ku
0001:0007ba50* _EXTENDED_KEY_USAGE_it
0001:0007b9e0  _v3_ocsp_accresp
0001:0007ba6c* _d2i_EXTENDED_KEY_USAGE
0001:0007ba95* _i2d_EXTENDED_KEY_USAGE
0001:0007bab7* _EXTENDED_KEY_USAGE_new
0001:0007bacb* _EXTENDED_KEY_USAGE_free
Module: U:\extras\lib\libcrypto.lib(v3_enum.obj)
0001:0007be20  _v3_crl_reason
0001:0007be58* _i2s_ASN1_ENUMERATED_TABLE
Module: U:\extras\lib\libcrypto.lib(v3_ocsp.obj)
0001:0007bec0  _v3_ocsp_crlid
0001:0007bf00  _v3_ocsp_acutoff
0001:0007bf40  _v3_crl_invdate
0001:0007bf80  _v3_crl_hold
0001:0007bfc0  _v3_ocsp_nonce
0001:0007c000  _v3_ocsp_nocheck
0001:0007c040  _v3_ocsp_serviceloc
Module: U:\extras\lib\libcrypto.lib(v3_sxnet.obj)
0001:0007c5d0  _v3_sxnet
0001:0007c730* _SXNET_it
0001:0007c650* _SXNETID_it
0001:0007c66c* _d2i_SXNETID
0001:0007c695* _i2d_SXNETID
0001:0007c6b7* _SXNETID_new
0001:0007c6cb* _SXNETID_free
0001:0007c74c* _d2i_SXNET
0001:0007c775* _i2d_SXNET
0001:0007c797* _SXNET_new
0001:0007c7ab* _SXNET_free
0001:0007c960* _SXNET_add_id_asc
0001:0007ca76* _SXNET_add_id_INTEGER
0001:0007c9de* _SXNET_add_id_ulong
0001:0007cd9d* _SXNET_get_id_INTEGER
0001:0007cc81* _SXNET_get_id_asc
0001:0007cd02* _SXNET_get_id_ulong
Module: U:\extras\lib\libcrypto.lib(v3_info.obj)
0001:0007ce10  _v3_info
0001:0007cfc0* _AUTHORITY_INFO_ACCESS_it
0001:0007ce50  _v3_sinfo
0001:0007cee0  _ACCESS_DESCRIPTION_it
0001:0007cefc* _d2i_ACCESS_DESCRIPTION
0001:0007cf25* _i2d_ACCESS_DESCRIPTION
0001:0007cf47* _ACCESS_DESCRIPTION_new
0001:0007cf5b* _ACCESS_DESCRIPTION_free
0001:0007cfdc* _d2i_AUTHORITY_INFO_ACCESS
0001:0007d005* _i2d_AUTHORITY_INFO_ACCESS
0001:0007d027* _AUTHORITY_INFO_ACCESS_new
0001:0007d03b  _AUTHORITY_INFO_ACCESS_free
0001:0007d4a6* _i2a_ACCESS_DESCRIPTION
Module: U:\extras\lib\libcrypto.lib(v3_pcons.obj)
0001:0007d4d0  _v3_policy_constraints
0001:0007d580* _POLICY_CONSTRAINTS_it
0001:0007d59c* _POLICY_CONSTRAINTS_new
0001:0007d5b0  _POLICY_CONSTRAINTS_free
Module: U:\extras\lib\libcrypto.lib(v3_pci.obj)
0001:0007d830  _v3_pci
Module: U:\extras\lib\libcrypto.lib(v3_pmaps.obj)
0001:0007e800  _v3_policy_mappings
0001:0007e8f0* _POLICY_MAPPINGS_it
0001:0007e8a0* _POLICY_MAPPING_it
0001:0007e90c* _POLICY_MAPPING_new
0001:0007e920  _POLICY_MAPPING_free
Module: U:\extras\lib\libcrypto.lib(v3_conf.obj)
0001:0007ecdb* _X509V3_EXT_nconf
0001:0007edc7* _X509V3_EXT_nconf_nid
0001:0007f289  _X509V3_EXT_i2d
0001:0007f667* _X509V3_EXT_add_nconf_sk
0001:0007f72f* _X509V3_EXT_add_nconf
0001:0007f76f* _X509V3_EXT_CRL_add_nconf
0001:0007f7af* _X509V3_EXT_REQ_add_nconf
0001:0007f831* _X509V3_get_string
0001:0007f8c0  _X509V3_get_section
0001:0007f94b* _X509V3_string_free
0001:0007f984  _X509V3_section_free
0001:0007f9f8  _X509V3_set_nconf
0001:0007fa10* _X509V3_set_ctx
0001:0007fa41* _X509V3_EXT_conf
0001:0007fa7b* _X509V3_EXT_conf_nid
0001:0007faf0* _X509V3_set_conf_lhash
0001:0007fb08* _X509V3_EXT_add_conf
0001:0007fb42* _X509V3_EXT_CRL_add_conf
0001:0007fb7c* _X509V3_EXT_REQ_add_conf
Module: U:\extras\lib\libcrypto.lib(tasn_utl.obj)
0001:0007fbc0  _asn1_get_choice_selector
0001:0007fbe0  _asn1_set_choice_selector
0001:0007fc19  _asn1_do_lock
0001:0007fd09  _asn1_enc_init
0001:0007fd49  _asn1_enc_free
0001:0007fd9f  _asn1_enc_save
0001:0007fe44  _asn1_enc_restore
0001:0007fec8  _asn1_get_field_ptr
0001:0007fef9  _asn1_do_adb
Module: U:\extras\lib\libcrypto.lib(a_type.obj)
0001:00080010  _ASN1_TYPE_get
0001:00080035  _ASN1_TYPE_set
0001:00080091  _ASN1_TYPE_set1
0001:0008013b  _ASN1_TYPE_cmp
Module: U:\extras\lib\libcrypto.lib(a_bitstr.obj)
0001:000801d0  _ASN1_BIT_STRING_set
0001:000801f1  _i2c_ASN1_BIT_STRING
0001:000803b1  _c2i_ASN1_BIT_STRING
0001:0008057a  _ASN1_BIT_STRING_set_bit
0001:0008075c  _ASN1_BIT_STRING_get_bit
0001:000807d1* _ASN1_BIT_STRING_check
Module: U:\extras\lib\libcrypto.lib(v3_utl.obj)
0001:000808db  _X509V3_add_value
0001:00080a22  _X509V3_add_value_uchar
0001:00080a43  _X509V3_conf_free
0001:00080ab0  _X509V3_add_value_bool
0001:00080af4* _X509V3_add_value_bool_nf
0001:00080b23  _i2s_ASN1_ENUMERATED
0001:00080bb0  _i2s_ASN1_INTEGER
0001:00080c3d  _s2i_ASN1_INTEGER
0001:00080ded  _X509V3_add_value_int
0001:00080e88  _X509V3_get_value_bool
0001:0008104d  _X509V3_get_value_int
0001:000810c9  _X509V3_parse_list
0001:00081438  _hex_to_string
0001:0008151f  _string_to_hex
0001:00081773  _name_cmp
0001:000817f1* _X509_get1_email
0001:00081853* _X509_get1_ocsp
0001:00081914* _X509_REQ_get1_email
0001:00081b60* _X509_email_free
0001:00081b7c  _a2i_IPADDRESS
0001:00081d1b* _a2i_ipadd
0001:00081bed  _a2i_IPADDRESS_NC
0001:000821af  _X509V3_NAME_from_section
Module: U:\extras\lib\libcrypto.lib(asn1_gen.obj)
0001:000822e0* _ASN1_generate_nconf
0001:00082332  _ASN1_generate_v3
Module: U:\extras\lib\libcrypto.lib(pem_oth.obj)
0001:00083cda  _PEM_ASN1_read_bio
Module: U:\extras\lib\libcrypto.lib(pem_lib.obj)
0001:00083da0* _PEM_version
0001:00083e1c  _PEM_def_callback
0001:00083f6a  _PEM_proc_type
0001:00084003  _PEM_dek_info
0001:000840f3  _PEM_ASN1_read
0001:00085f94  _pem_check_suffix
0001:0008459a  _PEM_bytes_read_bio
0001:00085775  _PEM_read_bio
0001:00084f2e  _PEM_get_EVP_CIPHER_INFO
0001:00084cf4  _PEM_do_header
0001:000846fd  _PEM_ASN1_write
0001:00084815  _PEM_ASN1_write_bio
0001:000853e1  _PEM_write_bio
0001:00085319* _PEM_write
0001:000856ca* _PEM_read
Module: U:\tmp\ldconv_libgcc_so_d_a_ddb24f08029a1a0e38.lib(emx-eh.obj)
0001:00086075  ___ehInit
0001:00086040* ___ehTerm
Module: U:\extras\lib\libcrypto.lib(eng_lib.obj)
0001:000860ba  _ENGINE_new
0001:0008615f* _engine_set_all_null
0001:0008620d  _engine_free_util
0001:0008630a  _ENGINE_free
0001:000863a0  _engine_cleanup_add_first
0001:000863eb  _engine_cleanup_add_last
0001:00086448* _ENGINE_cleanup
0001:0008648c* _ENGINE_get_ex_new_index
0001:000864c3* _ENGINE_set_ex_data
0001:000864e7* _ENGINE_get_ex_data
0001:00086504* _ENGINE_set_id
0001:00086552* _ENGINE_set_name
0001:000865a1* _ENGINE_set_destroy_function
0001:000865b4* _ENGINE_set_init_function
0001:000865c7* _ENGINE_set_finish_function
0001:000865da* _ENGINE_set_ctrl_function
0001:000865ed* _ENGINE_set_flags
0001:00086600* _ENGINE_set_cmd_defns
0001:00086613* _ENGINE_get_id
0001:0008661d* _ENGINE_get_name
0001:00086628* _ENGINE_get_destroy_function
0001:00086633* _ENGINE_get_init_function
0001:0008663e* _ENGINE_get_finish_function
0001:00086649* _ENGINE_get_ctrl_function
0001:00086654* _ENGINE_get_flags
0001:0008665f* _ENGINE_get_cmd_defns
0001:0008666a* _ENGINE_get_static_state
Module: U:\extras\lib\libcrypto.lib(eng_table.obj)
0001:00086680* _ENGINE_get_table_flags
0001:0008668a* _ENGINE_set_table_flags
0001:00086757  _engine_table_register
0001:00086a18  _engine_table_unregister
0001:00086af5  _engine_table_cleanup
0001:00086b79  _engine_table_select
0001:00086d9b  _engine_table_doall
Module: U:\extras\lib\libcrypto.lib(eng_list.obj)
0001:00087442* _ENGINE_remove
0001:000870d3  _ENGINE_get_first
0001:00087143* _ENGINE_get_last
0001:000871b3  _ENGINE_get_next
0001:0008726f* _ENGINE_get_prev
0001:0008732b* _ENGINE_add
0001:00087658* _ENGINE_by_id
0001:000878c3* _ENGINE_up_ref
Module: U:\extras\lib\libcrypto.lib(rand_os2.obj)
0001:0008795b  _RAND_poll
Module: U:\extras\lib\libcrypto.lib(eng_pkey.obj)
0001:00087d00* _ENGINE_set_load_privkey_function
0001:00087d13* _ENGINE_set_load_pubkey_function
0001:00087d26* _ENGINE_set_load_ssl_client_cert_function
0001:00087d39* _ENGINE_get_load_privkey_function
0001:00087d44* _ENGINE_get_load_pubkey_function
0001:00087d4f  _ENGINE_get_ssl_client_cert_function
0001:00087d65* _ENGINE_load_private_key
0001:00087ef4* _ENGINE_load_public_key
0001:00088083  _ENGINE_load_ssl_client_cert
Module: U:\extras\lib\libssl.lib(ssl_asn1.obj)
0001:000881f0  _i2d_SSL_SESSION
0001:00088f39  _d2i_SSL_SESSION
Module: U:\extras\lib\libcrypto.lib(x509_vfy.obj)
0001:0008a4b0* _X509_version
0001:0008a4eb  _X509_verify_cert
0001:0008d224* _X509_get_pubkey_parameters
0001:0008ce56* _X509_cmp_time
0001:0008d7a1  _X509_STORE_CTX_init
0001:0008dd04* _X509_STORE_CTX_set0_param
0001:0008db72  _X509_STORE_CTX_cleanup
0001:0008ce3b* _X509_cmp_current_time
0001:0008d14b* _X509_time_adj
0001:0008d129  _X509_gmtime_adj
0001:0008d174* _X509_time_adj_ex
0001:0008d39c  _X509_STORE_CTX_get_ex_new_index
0001:0008d3d3  _X509_STORE_CTX_set_ex_data
0001:0008d3fa* _X509_STORE_CTX_get_ex_data
0001:0008d41a* _X509_STORE_CTX_get_error
0001:0008d425* _X509_STORE_CTX_set_error
0001:0008d433* _X509_STORE_CTX_get_error_depth
0001:0008d43e* _X509_STORE_CTX_get_current_cert
0001:0008d449* _X509_STORE_CTX_get_chain
0001:0008d454* _X509_STORE_CTX_get1_chain
0001:0008d4e6* _X509_STORE_CTX_get0_current_issuer
0001:0008d4f1* _X509_STORE_CTX_get0_current_crl
0001:0008d4fc* _X509_STORE_CTX_get0_parent_ctx
0001:0008d507* _X509_STORE_CTX_set_cert
0001:0008d515* _X509_STORE_CTX_set_chain
0001:0008d523* _X509_STORE_CTX_set0_crls
0001:0008d531  _X509_STORE_CTX_set_purpose
0001:0008d585* _X509_STORE_CTX_purpose_inherit
0001:0008d55b* _X509_STORE_CTX_set_trust
0001:0008d6fd* _X509_STORE_CTX_new
0001:0008d77b* _X509_STORE_CTX_free
0001:0008db5a* _X509_STORE_CTX_trusted_stack
0001:0008dc46* _X509_STORE_CTX_set_depth
0001:0008dc63* _X509_STORE_CTX_set_flags
0001:0008dc80* _X509_STORE_CTX_set_time
0001:0008dc9d  _X509_STORE_CTX_set_verify_cb
0001:0008dcab* _X509_STORE_CTX_get0_policy_tree
0001:0008dcb6* _X509_STORE_CTX_get_explicit_policy
0001:0008dcc1  _X509_STORE_CTX_set_default
0001:0008dcf9  _X509_STORE_CTX_get0_param
Module: U:\extras\lib\libcrypto.lib(dh_asn1.obj)
0001:0008de00* _DHparams_it
0001:0008de1c  _d2i_DHparams
0001:0008de45  _i2d_DHparams
0001:0008de67  _DHparams_dup
Module: U:\extras\lib\libcrypto.lib(ec_key.obj)
0001:0008de99  _EC_KEY_new
0001:0008df4b* _EC_KEY_new_by_curve_name
0001:0008df98  _EC_KEY_free
0001:0008e05b* _EC_KEY_copy
0001:0008e2a6  _EC_KEY_dup
0001:0008e2ee  _EC_KEY_up_ref
0001:0008e331  _EC_KEY_generate_key
0001:0008e51a* _EC_KEY_check_key
0001:0008e8a1  _EC_KEY_get0_group
0001:0008e8ac  _EC_KEY_set_group
0001:0008e8eb  _EC_KEY_get0_private_key
0001:0008e8f6  _EC_KEY_set_private_key
0001:0008e935  _EC_KEY_get0_public_key
0001:0008e940  _EC_KEY_set_public_key
0001:0008e989  _EC_KEY_get_enc_flags
0001:0008e994  _EC_KEY_set_enc_flags
0001:0008e9a2  _EC_KEY_get_conv_form
0001:0008e9ad* _EC_KEY_set_conv_form
0001:0008e9dd  _EC_KEY_get_key_method_data
0001:0008ea08  _EC_KEY_insert_key_method_data
0001:0008eaae* _EC_KEY_set_asn1_flag
0001:0008ead5* _EC_KEY_precompute_mult
Module: U:\extras\lib\libcrypto.lib(o_dir.obj)
0001:0008eb10  _OPENSSL_DIR_read
0001:0008eb28  _OPENSSL_DIR_end
Module: U:\extras\lib\libcrypto.lib(x509_trs.obj)
0001:0008ebbc* _X509_TRUST_set_default
0001:0008ebd7  _X509_check_trust
0001:0008ecb7  _X509_TRUST_get_by_id
0001:0008ec70* _X509_TRUST_get0
0001:0008ec48* _X509_TRUST_get_count
0001:0008ed1c  _X509_TRUST_set
0001:0008ed74* _X509_TRUST_add
0001:0008efb3* _X509_TRUST_cleanup
0001:0008f006* _X509_TRUST_get_flags
0001:0008f011* _X509_TRUST_get0_name
0001:0008f01c* _X509_TRUST_get_trust
Module: U:\usr\local446\lib\libc_dll.lib(shutdown.obj)
0001:0008f1d0  _shutdown
Module: U:\extras\lib\libcrypto.lib(x_crl.obj)
0001:0008f2f0* _X509_REVOKED_it
0001:0008f450  _X509_CRL_INFO_it
0001:0008fb50  _X509_CRL_it
0001:0008fb6c* _d2i_X509_REVOKED
0001:0008fb95* _i2d_X509_REVOKED
0001:0008fbb7* _X509_REVOKED_new
0001:0008fbcb* _X509_REVOKED_free
0001:0008fbe6* _d2i_X509_CRL_INFO
0001:0008fc0f* _i2d_X509_CRL_INFO
0001:0008fc31* _X509_CRL_INFO_new
0001:0008fc45* _X509_CRL_INFO_free
0001:0008fc60  _d2i_X509_CRL
0001:0008fc89  _i2d_X509_CRL
0001:0008fcab* _X509_CRL_new
0001:0008fcbf  _X509_CRL_free
0001:0008fcda* _X509_CRL_dup
0001:0008fd1f* _X509_CRL_add0_revoked
0001:0008fdb3  _X509_CRL_verify
0001:0008fde7* _X509_CRL_get0_by_serial
0001:0008fe2a  _X509_CRL_get0_by_cert
0001:000900ce* _X509_CRL_set_default_method
0001:000900ed* _X509_CRL_METHOD_new
0001:00090151* _X509_CRL_METHOD_free
0001:00090173* _X509_CRL_set_meth_data
0001:00090181* _X509_CRL_get_meth_data
Module: U:\extras\lib\libcrypto.lib(evp_pbe.obj)
0001:00090335  _EVP_PBE_CipherInit
0001:00090756  _EVP_PBE_find
0001:0009062c* _EVP_PBE_alg_add_type
0001:000906ec* _EVP_PBE_alg_add
0001:0009083a  _EVP_PBE_cleanup
Module: U:\extras\lib\libcrypto.lib(obj_xref.obj)
0002:00009b70+ _sig_app
0002:00009b80+ _sigx_app
0001:00090b62  _OBJ_find_sigid_algs
0001:00090c00  _OBJ_find_sigid_by_algs
0001:00090cb1* _OBJ_add_sigid
0001:00090dd9  _OBJ_sigid_free
Module: U:\extras\lib\libcrypto.lib(rsa_eay.obj)
0001:00090e48  _RSA_PKCS1_SSLeay
Module: U:\extras\lib\libcrypto.lib(tb_rsa.obj)
0001:00092f04* _ENGINE_unregister_RSA
0001:00092f33* _ENGINE_register_RSA
0001:00092f7f* _ENGINE_register_all_RSA
0001:00092fb0* _ENGINE_set_default_RSA
0001:00092ffc  _ENGINE_get_default_RSA
0001:00093019  _ENGINE_get_RSA
0001:00093024* _ENGINE_set_RSA
Module: U:\extras\lib\libcrypto.lib(bn_blind.obj)
0001:0009304b* _BN_BLINDING_new
0001:00093187  _BN_BLINDING_free
0001:00093201* _BN_BLINDING_update
0001:00093582  _BN_BLINDING_create_param
0001:00093362* _BN_BLINDING_convert
0001:0009338b  _BN_BLINDING_convert_ex
0001:00093440* _BN_BLINDING_invert
0001:00093469  _BN_BLINDING_invert_ex
0001:00093545* _BN_BLINDING_get_thread_id
0001:00093550* _BN_BLINDING_set_thread_id
0001:0009355e  _BN_BLINDING_thread_id
0001:00093569* _BN_BLINDING_get_flags
0001:00093574* _BN_BLINDING_set_flags
Module: U:\extras\lib\libcrypto.lib(bn_ctx.obj)
0001:000937f0* _BN_CTX_init
0001:00093838  _BN_CTX_new
0001:000938d2  _BN_CTX_free
0001:00093907  _BN_CTX_start
0001:0009398b  _BN_CTX_end
0001:000939f7  _BN_CTX_get
Module: U:\extras\lib\libcrypto.lib(bn_add.obj)
0001:00093ed0  _BN_add
0001:00094139  _BN_usub
0001:00093fab  _BN_uadd
0001:00094352  _BN_sub
Module: U:\extras\lib\libcrypto.lib(bn_mul.obj)
0001:000944c0* _bn_sub_part_words
0001:00094808* _bn_add_part_words
0001:00094c58* _bn_mul_recursive
0001:00096926* _bn_mul_normal
0001:0009538f* _bn_mul_part_recursive
0001:00095bb4* _bn_mul_low_recursive
0001:00096ac9* _bn_mul_low_normal
0001:00095d95* _bn_mul_high
0001:000964cb  _BN_mul
Module: U:\extras\lib\libcrypto.lib(bn_gcd.obj)
0001:00096be0  _BN_gcd
0001:00096ecd  _BN_mod_inverse
Module: U:\extras\lib\libcrypto.lib(dh_key.obj)
0001:00097b30  _DH_generate_key
0001:00097b49  _DH_compute_key
0001:00097b82  _DH_OpenSSL
Module: U:\extras\lib\libcrypto.lib(tb_dh.obj)
0001:00098124* _ENGINE_unregister_DH
0001:00098153* _ENGINE_register_DH
0001:0009819f* _ENGINE_register_all_DH
0001:000981d0* _ENGINE_set_default_DH
0001:0009821c  _ENGINE_get_default_DH
0001:00098239  _ENGINE_get_DH
0001:00098244* _ENGINE_set_DH
Module: U:\extras\lib\libcrypto.lib(dsa_lib.obj)
0001:00098260* _DSA_version
0001:00098286* _DSA_set_default_method
0001:00098293* _DSA_get_default_method
0001:000982b3  _DSA_new
0001:00098342* _DSA_new_method
0001:000982c7* _DSA_set_method
0001:000985a2  _DSA_free
0001:000986fb  _DSA_up_ref
0001:0009873e  _DSA_size
0001:000987ba* _DSA_get_ex_new_index
0001:000987f1* _DSA_set_ex_data
0001:00098815* _DSA_get_ex_data
0001:00098832* _DSA_dup_DH
Module: U:\extras\lib\libcrypto.lib(x_attrib.obj)
0001:000989b0* _X509_ATTRIBUTE_SET_it
0001:00098a10  _X509_ATTRIBUTE_it
0001:00098a2c* _d2i_X509_ATTRIBUTE
0001:00098a55* _i2d_X509_ATTRIBUTE
0001:00098a77  _X509_ATTRIBUTE_new
0001:00098a8b  _X509_ATTRIBUTE_free
0001:00098aa6  _X509_ATTRIBUTE_dup
0001:00098ac1  _X509_ATTRIBUTE_create
Module: U:\extras\lib\libcrypto.lib(v3_pcia.obj)
0001:00098c00* _PROXY_POLICY_it
0001:00098c1c* _d2i_PROXY_POLICY
0001:00098c45* _i2d_PROXY_POLICY
0001:00098c67* _PROXY_POLICY_new
0001:00098c7b* _PROXY_POLICY_free
0001:00098d10  _PROXY_CERT_INFO_EXTENSION_it
0001:00098d2c* _d2i_PROXY_CERT_INFO_EXTENSION
0001:00098d55* _i2d_PROXY_CERT_INFO_EXTENSION
0001:00098d77  _PROXY_CERT_INFO_EXTENSION_new
0001:00098d8b  _PROXY_CERT_INFO_EXTENSION_free
Module: U:\extras\lib\libcrypto.lib(a_octet.obj)
0001:00098db0  _ASN1_OCTET_STRING_dup
0001:00098dc3  _ASN1_OCTET_STRING_cmp
0001:00098ddd  _ASN1_OCTET_STRING_set
Module: U:\extras\lib\libcrypto.lib(tb_cipher.obj)
0001:00098e00* _ENGINE_unregister_ciphers
0001:00098e2f* _ENGINE_register_ciphers
0001:00098ea7* _ENGINE_register_all_ciphers
0001:00098ed8* _ENGINE_set_default_ciphers
0001:00098f50  _ENGINE_get_cipher_engine
0001:00098f77  _ENGINE_get_cipher
0001:00098fee* _ENGINE_get_ciphers
0001:00098ff9* _ENGINE_set_ciphers
Module: U:\extras\lib\libcrypto.lib(by_file.obj)
0001:00099025  _X509_LOOKUP_file
0001:000995bf* _X509_load_cert_crl_file
0001:00099151  _X509_load_cert_file
0001:00099387  _X509_load_crl_file
0002:00003450* _x509_file_lookup
Module: U:\extras\lib\libcrypto.lib(by_dir.obj)
0001:00099775  _X509_LOOKUP_hash_dir
0002:00003480* _x509_dir_lookup
Module: U:\extras\lib\libcrypto.lib(tb_digest.obj)
0001:0009a210* _ENGINE_unregister_digests
0001:0009a23f* _ENGINE_register_digests
0001:0009a2b7* _ENGINE_register_all_digests
0001:0009a2e8* _ENGINE_set_default_digests
0001:0009a360  _ENGINE_get_digest_engine
0001:0009a387  _ENGINE_get_digest
0001:0009a3fe* _ENGINE_get_digests
0001:0009a409* _ENGINE_set_digests
Module: U:\extras\lib\libcrypto.lib(pmeth_lib.obj)
0001:0009a490* _EVP_PKEY_meth_find
0001:0009aafb  _EVP_PKEY_CTX_free
0001:0009a747* _EVP_PKEY_meth_new
0001:0009a891  _EVP_PKEY_meth_free
0001:0009a8b7  _EVP_PKEY_CTX_new
0001:0009a8d9  _EVP_PKEY_CTX_new_id
0001:0009a8fb  _EVP_PKEY_CTX_dup
0001:0009aa97* _EVP_PKEY_meth_add0
0001:0009ab84  _EVP_PKEY_CTX_ctrl
0001:0009ace3* _EVP_PKEY_CTX_ctrl_str
0001:0009adf6* _EVP_PKEY_CTX_get_operation
0001:0009ae01* _EVP_PKEY_CTX_set0_keygen_info
0001:0009ae18* _EVP_PKEY_CTX_set_data
0001:0009ae26* _EVP_PKEY_CTX_get_data
0001:0009ae31* _EVP_PKEY_CTX_get0_pkey
0001:0009ae3c* _EVP_PKEY_CTX_get0_peerkey
0001:0009ae47* _EVP_PKEY_CTX_set_app_data
0001:0009ae55* _EVP_PKEY_CTX_get_app_data
0001:0009ae60* _EVP_PKEY_meth_set_init
0001:0009ae6e* _EVP_PKEY_meth_set_copy
0001:0009ae7c* _EVP_PKEY_meth_set_cleanup
0001:0009ae8a* _EVP_PKEY_meth_set_paramgen
0001:0009aea1* _EVP_PKEY_meth_set_keygen
0001:0009aeb8* _EVP_PKEY_meth_set_sign
0001:0009aecf* _EVP_PKEY_meth_set_verify
0001:0009aee6* _EVP_PKEY_meth_set_verify_recover
0001:0009aefd* _EVP_PKEY_meth_set_signctx
0001:0009af14* _EVP_PKEY_meth_set_verifyctx
0001:0009af2b* _EVP_PKEY_meth_set_encrypt
0001:0009af42* _EVP_PKEY_meth_set_decrypt
0001:0009af59* _EVP_PKEY_meth_set_derive
0001:0009af70* _EVP_PKEY_meth_set_ctrl
0002:00009630* _app_pkey_methods
Module: U:\extras\lib\libcrypto.lib(rsa_ameth.obj)
0001:0009b9a0  _rsa_asn1_meths
Module: U:\extras\lib\libcrypto.lib(dh_ameth.obj)
0001:0009c7e7* _DHparams_print
0001:0009c840  _dh_asn1_meth
Module: U:\extras\lib\libcrypto.lib(dsa_ameth.obj)
0001:0009db60  _dsa_asn1_meths
Module: U:\extras\lib\libcrypto.lib(ec_ameth.obj)
0001:0009f0b0  _eckey_asn1_meth
Module: U:\extras\lib\libcrypto.lib(hm_ameth.obj)
0001:0009f2a0  _hmac_asn1_meth
Module: U:\extras\lib\libcrypto.lib(tb_asnmth.obj)
0001:0009f300* _ENGINE_unregister_pkey_asn1_meths
0001:0009f32f* _ENGINE_register_pkey_asn1_meths
0001:0009f3a7* _ENGINE_register_all_pkey_asn1_meths
0001:0009f3d8* _ENGINE_set_default_pkey_asn1_meths
0001:0009f450  _ENGINE_get_pkey_asn1_meth_engine
0001:0009f477  _ENGINE_get_pkey_asn1_meth
0001:0009f4ee* _ENGINE_get_pkey_asn1_meths
0001:0009f4f9* _ENGINE_set_pkey_asn1_meths
0001:0009f50c  _engine_pkey_asn1_meths_free
0001:0009f597* _ENGINE_get_pkey_asn1_meth_str
0001:0009f73e  _ENGINE_pkey_asn1_find_str
Module: U:\extras\lib\libcrypto.lib(evp_asn1.obj)
0001:0009f7e0  _ASN1_TYPE_set_octetstring
0001:0009f852  _ASN1_TYPE_get_octetstring
0001:0009f8ea  _ASN1_TYPE_set_int_octetstring
0001:0009fa57  _ASN1_TYPE_get_int_octetstring
Module: U:\extras\lib\libcrypto.lib(a_time.obj)
0001:0009fc70  _ASN1_TIME_it
0001:0009fc8c* _d2i_ASN1_TIME
0001:0009fcb5* _i2d_ASN1_TIME
0001:0009fcd7* _ASN1_TIME_new
0001:0009fceb  _ASN1_TIME_free
0001:0009fd06* _ASN1_TIME_set
0001:0009fd39  _ASN1_TIME_adj
0001:0009fe1c  _ASN1_TIME_check
0001:0009fe5f* _ASN1_TIME_to_generalizedtime
0001:0009ff9d* _ASN1_TIME_set_string
Module: U:\extras\lib\libcrypto.lib(pcy_data.obj)
0001:000a0020  _policy_data_free
0001:000a0086  _policy_data_new
Module: U:\extras\lib\libcrypto.lib(pcy_map.obj)
0001:000a01b0  _policy_cache_set_mapping
Module: U:\extras\lib\libcrypto.lib(md5_dgst.obj)
0001:000a0380  _MD5_Update
0001:000a0725* _md5_block_data_order
0001:000a0537* _MD5_Transform
0001:000a0559  _MD5_Final
0001:000a06b0* _MD5_version
0001:000a06d6  _MD5_Init
Module: U:\extras\lib\libcrypto.lib(rsa_sign.obj)
0001:000a129b  _RSA_sign
0001:000a15ad  _int_rsa_verify
0001:000a1a27  _RSA_verify
Module: U:\extras\lib\libcrypto.lib(sha1dgst.obj)
0001:000a1ac0* _SHA1_version
0001:000a1ae7  _SHA1_Update
0001:000a1c9e* _SHA1_Transform
0001:000a1cc0  _SHA1_Final
0001:000a1ea1  _SHA1_Init
Module: U:\extras\lib\libcrypto.lib(sha256.obj)
0001:000a4530* _SHA256_version
0001:000a455a  _SHA224_Init
0001:000a45db  _SHA256_Init
0001:000a465c* _SHA224
0001:000a475f  _SHA256_Update
0001:000a4938  _SHA256_Final
0001:000a46c0* _SHA256
0001:000a4724* _SHA224_Update
0001:000a4745* _SHA224_Final
0001:000a4916* _SHA256_Transform
Module: U:\extras\lib\libcrypto.lib(sha512.obj)
0001:000a6f90* _SHA512_version
0001:000a6fba  _SHA384_Init
0001:000a7087  _SHA512_Init
0001:000a7154  _SHA512_Final
0001:000a7566* _SHA384_Final
0001:000a7580  _SHA512_Update
0001:000a7739* _SHA384_Update
0001:000a775a* _SHA512_Transform
0001:000a777c* _SHA384
0001:000a77ec* _SHA512
Module: U:\extras\lib\libcrypto.lib(bn_err.obj)
0001:000a87de  _ERR_load_BN_strings
Module: U:\extras\lib\libcrypto.lib(rsa_err.obj)
0001:000a902d  _ERR_load_RSA_strings
Module: U:\extras\lib\libcrypto.lib(dh_err.obj)
0001:000a91e8  _ERR_load_DH_strings
Module: U:\extras\lib\libcrypto.lib(evp_err.obj)
0001:000a9bbb  _ERR_load_EVP_strings
Module: U:\extras\lib\libcrypto.lib(buf_err.obj)
0001:000a9c4e  _ERR_load_BUF_strings
Module: U:\extras\lib\libcrypto.lib(obj_err.obj)
0001:000a9d02  _ERR_load_OBJ_strings
Module: U:\extras\lib\libcrypto.lib(pem_err.obj)
0001:000aa1c7  _ERR_load_PEM_strings
Module: U:\extras\lib\libcrypto.lib(dsa_err.obj)
0001:000aa3f7  _ERR_load_DSA_strings
Module: U:\extras\lib\libcrypto.lib(x509_err.obj)
0001:000aa9f7  _ERR_load_X509_strings
Module: U:\extras\lib\libcrypto.lib(asn1_err.obj)
0001:000abb21  _ERR_load_ASN1_strings
Module: U:\extras\lib\libcrypto.lib(conf_err.obj)
0001:000abde0  _ERR_load_CONF_strings
Module: U:\extras\lib\libcrypto.lib(cpt_err.obj)
0001:000abef2  _ERR_load_CRYPTOlib_strings
Module: U:\extras\lib\libcrypto.lib(comp_err.obj)
0001:000abfb2  _ERR_load_COMP_strings
Module: U:\extras\lib\libcrypto.lib(ec_err.obj)
0001:000aceb6  _ERR_load_EC_strings
Module: U:\extras\lib\libcrypto.lib(ecs_err.obj)
0001:000acfdc  _ERR_load_ECDSA_strings
Module: U:\extras\lib\libcrypto.lib(ech_err.obj)
0001:000ad07b  _ERR_load_ECDH_strings
Module: U:\extras\lib\libcrypto.lib(bio_err.obj)
0001:000ad471  _ERR_load_BIO_strings
Module: U:\extras\lib\libcrypto.lib(pkcs7err.obj)
0001:000adc6e  _ERR_load_PKCS7_strings
Module: U:\extras\lib\libcrypto.lib(v3err.obj)
0001:000ae6e6  _ERR_load_X509V3_strings
Module: U:\extras\lib\libcrypto.lib(pk12err.obj)
0001:000aeb0b  _ERR_load_PKCS12_strings
Module: U:\extras\lib\libcrypto.lib(rand_err.obj)
0001:000aeb87  _ERR_load_RAND_strings
Module: U:\extras\lib\libcrypto.lib(dso_err.obj)
0001:000af048  _ERR_load_DSO_strings
Module: U:\extras\lib\libcrypto.lib(ts_err.obj)
0001:000af7bb  _ERR_load_TS_strings
Module: U:\extras\lib\libcrypto.lib(eng_err.obj)
0001:000afdf8  _ERR_load_ENGINE_strings
Module: U:\extras\lib\libcrypto.lib(ocsp_err.obj)
0001:000b021f  _ERR_load_OCSP_strings
Module: U:\extras\lib\libcrypto.lib(ui_err.obj)
0001:000b03cf  _ERR_load_UI_strings
Module: U:\extras\lib\libcrypto.lib(cms_err.obj)
0001:000b1058  _ERR_load_CMS_strings
Module: U:\extras\lib\libcrypto.lib(ecb_enc.obj)
0001:000b10a0* _OSSL_libdes_version
0001:000b10d0* _OSSL_DES_version
0001:000b1119* _DES_options
0001:000b118d  _DES_ecb_encrypt
Module: U:\extras\lib\libcrypto.lib(ofb64enc.obj)
0001:000b12c0  _DES_ofb64_encrypt
Module: U:\extras\lib\libcrypto.lib(des_enc.obj)
0001:000b14f0* _DES_SPtrans
0001:000b1cf0  _DES_encrypt1
0001:000b4a13* _DES_encrypt2
0001:000b764e  _DES_encrypt3
0001:000b77c5  _DES_decrypt3
0001:000b793c  _DES_ncbc_encrypt
0001:000b809c  _DES_ede3_cbc_encrypt
Module: U:\extras\lib\libcrypto.lib(cfb64enc.obj)
0001:000b87f0  _DES_cfb64_encrypt
Module: U:\extras\lib\libcrypto.lib(cfb_enc.obj)
0001:000b8b10  _DES_cfb_encrypt
Module: U:\extras\lib\libcrypto.lib(set_key.obj)
0001:000b9510  _DES_set_odd_parity
0001:000b9549* _DES_check_key_parity
0001:000b9620* _DES_is_weak_key
0001:000b9e70* _DES_set_key
0001:000b9eac* _DES_set_key_checked
0001:000b9ef7  _DES_set_key_unchecked
0001:000ba1e4* _DES_key_sched
0002:00009730* __shadow_DES_check_key
Module: U:\extras\lib\libcrypto.lib(ecb3_enc.obj)
0001:000ba240  _DES_ecb3_encrypt
Module: U:\extras\lib\libcrypto.lib(ofb64ede.obj)
0001:000ba3a0  _DES_ede3_ofb64_encrypt
Module: U:\extras\lib\libcrypto.lib(cfb64ede.obj)
0001:000ba5d0  _DES_ede3_cfb64_encrypt
0001:000ba8fe  _DES_ede3_cfb_encrypt
Module: U:\extras\lib\libcrypto.lib(i_ecb.obj)
0001:000bb260* _IDEA_version
0001:000bb291* _idea_options
0001:000bb29b  _idea_ecb_encrypt
Module: U:\extras\lib\libcrypto.lib(i_cbc.obj)
0001:000bb3f0  _idea_cbc_encrypt
0001:000bbb36  _idea_encrypt
Module: U:\extras\lib\libcrypto.lib(i_ofb64.obj)
0001:000bc620  _idea_ofb64_encrypt
Module: U:\extras\lib\libcrypto.lib(i_cfb64.obj)
0001:000bc840  _idea_cfb64_encrypt
Module: U:\extras\lib\libcrypto.lib(i_skey.obj)
0001:000bcb50  _idea_set_encrypt_key
0001:000bcdc0  _idea_set_decrypt_key
Module: U:\extras\lib\libcrypto.lib(rc4_skey.obj)
0001:000bcf40* _RC4_version
0001:000bcf73* _RC4_options
0001:000bcf7d  _RC4_set_key
Module: U:\extras\lib\libcrypto.lib(rc4_enc.obj)
0001:000bd150  _RC4
Module: U:\extras\lib\libcrypto.lib(rc2_cbc.obj)
0001:000bd850  _RC2_cbc_encrypt
0001:000bdf86  _RC2_encrypt
0001:000be143  _RC2_decrypt
Module: U:\extras\lib\libcrypto.lib(rc2cfb64.obj)
0001:000be350  _RC2_cfb64_encrypt
Module: U:\extras\lib\libcrypto.lib(rc2_ecb.obj)
0001:000be660* _RC2_version
0001:000be686  _RC2_ecb_encrypt
Module: U:\extras\lib\libcrypto.lib(rc2ofb64.obj)
0001:000be7f0  _RC2_ofb64_encrypt
Module: U:\extras\lib\libcrypto.lib(rc2_skey.obj)
0001:000beb10  _RC2_set_key
Module: U:\extras\lib\libcrypto.lib(aes_cbc.obj)
0001:000becb0  _AES_cbc_encrypt
Module: U:\extras\lib\libcrypto.lib(aes_cfb.obj)
0001:000bed20  _AES_cfb128_encrypt
0001:000bed66  _AES_cfb1_encrypt
0001:000bedac  _AES_cfb8_encrypt
Module: U:\extras\lib\libcrypto.lib(aes_ecb.obj)
0001:000bee00  _AES_ecb_encrypt
Module: U:\extras\lib\libcrypto.lib(aes_ofb.obj)
0001:000bee50  _AES_ofb128_encrypt
Module: U:\extras\lib\libcrypto.lib(aes_core.obj)
0001:000c0fb8  _AES_set_encrypt_key
0001:000c1655  _AES_set_decrypt_key
0001:000c1a18  _AES_encrypt
0001:000c2077  _AES_decrypt
Module: U:\extras\lib\libcrypto.lib(cmll_cbc.obj)
0001:000c26d0  _Camellia_cbc_encrypt
Module: U:\extras\lib\libcrypto.lib(cmll_cfb.obj)
0001:000c2740  _Camellia_cfb128_encrypt
0001:000c2786  _Camellia_cfb1_encrypt
0001:000c27cc  _Camellia_cfb8_encrypt
Module: U:\extras\lib\libcrypto.lib(cmll_ecb.obj)
0001:000c2820  _Camellia_ecb_encrypt
Module: U:\extras\lib\libcrypto.lib(cmll_ofb.obj)
0001:000c2870  _Camellia_ofb128_encrypt
Module: U:\extras\lib\libcrypto.lib(cmll_misc.obj)
0001:000c28b0* _CAMELLIA_version
0001:000c28db  _Camellia_set_key
0001:000c293f  _Camellia_encrypt
0001:000c296d  _Camellia_decrypt
Module: U:\extras\lib\libcrypto.lib(seed_cbc.obj)
0001:000c29a0  _SEED_cbc_encrypt
Module: U:\extras\lib\libcrypto.lib(seed_cfb.obj)
0001:000c2a10  _SEED_cfb128_encrypt
Module: U:\extras\lib\libcrypto.lib(seed_ecb.obj)
0001:000c2a60  _SEED_ecb_encrypt
Module: U:\extras\lib\libcrypto.lib(seed_ofb.obj)
0001:000c2ab0  _SEED_ofb128_encrypt
Module: U:\extras\lib\libcrypto.lib(seed.obj)
0001:000c3af0  _SEED_set_key
0001:000c4c14  _SEED_encrypt
0001:000c6199  _SEED_decrypt
Module: U:\extras\lib\libcrypto.lib(dsa_sign.obj)
0001:000c7720* _DSA_do_sign
0001:000c7747  _DSA_sign
0001:000c77bc  _DSA_sign_setup
Module: U:\extras\lib\libcrypto.lib(dsa_vrf.obj)
0001:000c77f0* _DSA_do_verify
0001:000c781e  _DSA_verify
Module: U:\extras\lib\libcrypto.lib(ecs_sign.obj)
0001:000c78a0* _ECDSA_do_sign
0001:000c78d1* _ECDSA_do_sign_ex
0001:000c7921  _ECDSA_sign
0001:000c7967* _ECDSA_sign_ex
0001:000c79ea  _ECDSA_sign_setup
Module: U:\extras\lib\libcrypto.lib(ecs_vrf.obj)
0001:000c7a40* _ECDSA_do_verify
0001:000c7a89  _ECDSA_verify
Module: U:\extras\lib\libcrypto.lib(e_xcbc_d.obj)
0001:000c7b34  _EVP_desx_cbc
Module: U:\extras\lib\libcrypto.lib(e_bf.obj)
0001:000c7f44  _EVP_bf_cbc
0001:000c7f84  _EVP_bf_cfb64
0001:000c7fc4  _EVP_bf_ofb
0001:000c8004  _EVP_bf_ecb
Module: U:\extras\lib\libcrypto.lib(e_cast.obj)
0001:000c82e4  _EVP_cast5_cbc
0001:000c8324  _EVP_cast5_cfb64
0001:000c8364  _EVP_cast5_ofb
0001:000c83a4  _EVP_cast5_ecb
Module: U:\extras\lib\libcrypto.lib(m_md4.obj)
0001:000c848c  _EVP_md4
Module: U:\extras\lib\libcrypto.lib(m_sha.obj)
0001:000c854c  _EVP_sha
Module: U:\extras\lib\libcrypto.lib(m_dss.obj)
0001:000c860c  _EVP_dss
Module: U:\extras\lib\libcrypto.lib(m_mdc2.obj)
0001:000c86cc  _EVP_mdc2
Module: U:\extras\lib\libcrypto.lib(m_ripemd.obj)
0001:000c878c  _EVP_ripemd160
Module: U:\extras\lib\libcrypto.lib(m_wp.obj)
0001:000c884c  _EVP_whirlpool
Module: U:\extras\lib\libcrypto.lib(a_verify.obj)
0001:000c886b* _ASN1_verify
0001:000c8a31  _ASN1_item_verify
Module: U:\extras\lib\libcrypto.lib(x_req.obj)
0001:000c8d80  _X509_REQ_INFO_it
0001:000c8d9c* _d2i_X509_REQ_INFO
0001:000c8dc5* _i2d_X509_REQ_INFO
0001:000c8de7* _X509_REQ_INFO_new
0001:000c8dfb* _X509_REQ_INFO_free
0001:000c8eb0  _X509_REQ_it
0001:000c8ecc  _d2i_X509_REQ
0001:000c8ef5  _i2d_X509_REQ
0001:000c8f17  _X509_REQ_new
0001:000c8f2b  _X509_REQ_free
0001:000c8f46* _X509_REQ_dup
Module: U:\extras\lib\libcrypto.lib(x_spki.obj)
0001:000c8fd0  _NETSCAPE_SPKAC_it
0001:000c8fec* _d2i_NETSCAPE_SPKAC
0001:000c9015* _i2d_NETSCAPE_SPKAC
0001:000c9037* _NETSCAPE_SPKAC_new
0001:000c904b* _NETSCAPE_SPKAC_free
0001:000c90d0* _NETSCAPE_SPKI_it
0001:000c90ec* _d2i_NETSCAPE_SPKI
0001:000c9115* _i2d_NETSCAPE_SPKI
0001:000c9137* _NETSCAPE_SPKI_new
0001:000c914b* _NETSCAPE_SPKI_free
Module: U:\extras\lib\libcrypto.lib(a_sign.obj)
0001:000c9179* _ASN1_sign
0001:000c94e4  _ASN1_item_sign
Module: U:\extras\lib\libcrypto.lib(a_d2i_fp.obj)
0001:000c986b  _ASN1_d2i_fp
0001:000c990f  _ASN1_d2i_bio
0001:000c997d  _ASN1_item_d2i_bio
0001:000c99f2  _ASN1_item_d2i_fp
Module: U:\extras\lib\libcrypto.lib(a_i2d_fp.obj)
0001:000c9dfb  _ASN1_i2d_fp
0001:000c9e98  _ASN1_i2d_bio
0001:000c9f86  _ASN1_item_i2d_fp
0001:000ca023  _ASN1_item_i2d_bio
Module: U:\extras\lib\libcrypto.lib(pk7_asn1.obj)
0001:000ca4c0* _PKCS7_SIGNED_it
0001:000ca880* _PKCS7_ENVELOPE_it
0001:000cac20* _PKCS7_SIGN_ENVELOPE_it
0001:000cae00* _PKCS7_DIGEST_it
0001:000cad00* _PKCS7_ENCRYPT_it
0001:000ca320  _PKCS7_it
0001:000ca33c  _d2i_PKCS7
0001:000ca365  _i2d_PKCS7
0001:000ca387  _PKCS7_new
0001:000ca39b  _PKCS7_free
0001:000ca3b6* _i2d_PKCS7_NDEF
0001:000ca3d8* _PKCS7_dup
0001:000ca690* _PKCS7_SIGNER_INFO_it
0001:000ca4dc* _d2i_PKCS7_SIGNED
0001:000ca505* _i2d_PKCS7_SIGNED
0001:000ca527  _PKCS7_SIGNED_new
0001:000ca53b  _PKCS7_SIGNED_free
0001:000ca780  _PKCS7_ISSUER_AND_SERIAL_it
0001:000ca6ac* _d2i_PKCS7_SIGNER_INFO
0001:000ca6d5* _i2d_PKCS7_SIGNER_INFO
0001:000ca6f7  _PKCS7_SIGNER_INFO_new
0001:000ca70b  _PKCS7_SIGNER_INFO_free
0001:000ca79c* _d2i_PKCS7_ISSUER_AND_SERIAL
0001:000ca7c5* _i2d_PKCS7_ISSUER_AND_SERIAL
0001:000ca7e7* _PKCS7_ISSUER_AND_SERIAL_new
0001:000ca7fb* _PKCS7_ISSUER_AND_SERIAL_free
0001:000ca9e0* _PKCS7_RECIP_INFO_it
0001:000caae0* _PKCS7_ENC_CONTENT_it
0001:000ca89c* _d2i_PKCS7_ENVELOPE
0001:000ca8c5* _i2d_PKCS7_ENVELOPE
0001:000ca8e7  _PKCS7_ENVELOPE_new
0001:000ca8fb* _PKCS7_ENVELOPE_free
0001:000ca9fc* _d2i_PKCS7_RECIP_INFO
0001:000caa25* _i2d_PKCS7_RECIP_INFO
0001:000caa47  _PKCS7_RECIP_INFO_new
0001:000caa5b  _PKCS7_RECIP_INFO_free
0001:000caafc* _d2i_PKCS7_ENC_CONTENT
0001:000cab25* _i2d_PKCS7_ENC_CONTENT
0001:000cab47* _PKCS7_ENC_CONTENT_new
0001:000cab5b* _PKCS7_ENC_CONTENT_free
0001:000cac3c* _d2i_PKCS7_SIGN_ENVELOPE
0001:000cac65* _i2d_PKCS7_SIGN_ENVELOPE
0001:000cac87  _PKCS7_SIGN_ENVELOPE_new
0001:000cac9b* _PKCS7_SIGN_ENVELOPE_free
0001:000cad1c* _d2i_PKCS7_ENCRYPT
0001:000cad45* _i2d_PKCS7_ENCRYPT
0001:000cad67  _PKCS7_ENCRYPT_new
0001:000cad7b* _PKCS7_ENCRYPT_free
0001:000cae1c* _d2i_PKCS7_DIGEST
0001:000cae45* _i2d_PKCS7_DIGEST
0001:000cae67  _PKCS7_DIGEST_new
0001:000cae7b* _PKCS7_DIGEST_free
0001:000caee0  _PKCS7_ATTR_SIGN_it
0001:000caf30  _PKCS7_ATTR_VERIFY_it
0001:000caf4c* _PKCS7_print_ctx
Module: U:\extras\lib\libcrypto.lib(dsa_asn1.obj)
0001:000cb070* _DSA_SIG_it
0001:000cb08c  _d2i_DSA_SIG
0001:000cb0b5  _i2d_DSA_SIG
0001:000cb0d7  _DSA_SIG_new
0001:000cb0eb  _DSA_SIG_free
0001:000cb220* _DSAPrivateKey_it
0001:000cb23c  _d2i_DSAPrivateKey
0001:000cb265  _i2d_DSAPrivateKey
0001:000cb2f0* _DSAparams_it
0001:000cb30c  _d2i_DSAparams
0001:000cb335  _i2d_DSAparams
0001:000cb3b0* _dsa_pub_internal_it
0001:000cb420* _DSAPublicKey_it
0001:000cb43c* _d2i_DSAPublicKey
0001:000cb465  _i2d_DSAPublicKey
0001:000cb487* _DSAparams_dup
Module: U:\extras\lib\libcrypto.lib(ec_asn1.obj)
0001:000cb4b0  _EC_GROUP_get_basis_type
0001:000cb520* _EC_GROUP_get_trinomial_basis
0001:000cb5b3* _EC_GROUP_get_pentanomial_basis
0001:000cb6e0* _X9_62_PENTANOMIAL_it
0001:000cb6fc* _X9_62_PENTANOMIAL_new
0001:000cb710* _X9_62_PENTANOMIAL_free
0001:000cb850* _X9_62_CHARACTERISTIC_TWO_it
0001:000cb86c* _X9_62_CHARACTERISTIC_TWO_new
0001:000cb880* _X9_62_CHARACTERISTIC_TWO_free
0001:000cb970* _X9_62_FIELDID_it
0001:000cb9f0* _X9_62_CURVE_it
0001:000cbad0* _ECPARAMETERS_it
0001:000cbaec* _ECPARAMETERS_new
0001:000cbb00* _ECPARAMETERS_free
0001:000cbbb0* _ECPKPARAMETERS_it
0001:000cbbcc* _d2i_UC_ECPKPARAMETERS
0001:000cbbf5* _i2d_UC_ECPKPARAMETERS
0001:000cbc17* _ECPKPARAMETERS_new
0001:000cbc2b* _ECPKPARAMETERS_free
0001:000cbcd0* _EC_PRIVATEKEY_it
0001:000cbcec* _d2i_EC_PRIVATEKEY
0001:000cbd15* _i2d_EC_PRIVATEKEY
0001:000cbd37* _EC_PRIVATEKEY_new
0001:000cbd4b* _EC_PRIVATEKEY_free
0001:000cd94c  _d2i_ECPKParameters
0001:000cda42  _i2d_ECPKParameters
0001:000cdb07  _d2i_ECPrivateKey
0001:000cde8a  _i2d_ECPrivateKey
0001:000ce334  _i2d_ECParameters
0001:000ce38a  _d2i_ECParameters
0001:000ce495  _o2i_ECPublicKey
0001:000ce5ee  _i2o_ECPublicKey
Module: U:\extras\lib\libcrypto.lib(a_digest.obj)
0001:000ce7bb* _ASN1_digest
0001:000ce887  _ASN1_item_digest
Module: U:\extras\lib\libcrypto.lib(x_sig.obj)
0001:000ce950  _X509_SIG_it
0001:000ce96c  _d2i_X509_SIG
0001:000ce995  _i2d_X509_SIG
0001:000ce9b7  _X509_SIG_new
0001:000ce9cb  _X509_SIG_free
Module: U:\extras\lib\libcrypto.lib(p8_pkey.obj)
0001:000ceaf0  _PKCS8_PRIV_KEY_INFO_it
0001:000ceb0c  _d2i_PKCS8_PRIV_KEY_INFO
0001:000ceb35  _i2d_PKCS8_PRIV_KEY_INFO
0001:000ceb57  _PKCS8_PRIV_KEY_INFO_new
0001:000ceb6b  _PKCS8_PRIV_KEY_INFO_free
0001:000ceb86  _PKCS8_pkey_set0
0001:000cec6e  _PKCS8_pkey_get0
Module: U:\extras\lib\libcrypto.lib(evp_pkey.obj)
0001:000ced41  _EVP_PKCS82PKEY
0001:000ceeed  _EVP_PKEY2PKCS8
0001:000cef08* _EVP_PKEY2PKCS8_broken
0001:000cf073* _PKCS8_set_broken
0001:000cf0e2* _EVP_PKEY_get_attr_count
0001:000cf0f8* _EVP_PKEY_get_attr_by_NID
0001:000cf11c* _EVP_PKEY_get_attr_by_OBJ
0001:000cf140* _EVP_PKEY_get_attr
0001:000cf15d* _EVP_PKEY_delete_attr
0001:000cf17a* _EVP_PKEY_add1_attr
0001:000cf1a7* _EVP_PKEY_add1_attr_by_OBJ
0001:000cf1e9* _EVP_PKEY_add1_attr_by_NID
0001:000cf22b* _EVP_PKEY_add1_attr_by_txt
Module: U:\extras\lib\libcrypto.lib(i2d_pr.obj)
0001:000cf279  _i2d_PrivateKey
Module: U:\extras\lib\libssl.lib(s3_enc.obj)
0001:000cf592  _ssl3_change_cipher_state
0001:000cfc97  _ssl3_setup_key_block
0001:000cfecb  _ssl3_cleanup_key_block
0001:000cff3d  _ssl3_enc
0001:000d015d  _ssl3_init_finished_mac
0001:000d01ee  _ssl3_free_digest_list
0001:000d0277  _ssl3_finish_mac
0001:000d030b  _ssl3_digest_cached_records
0001:000d04e2  _ssl3_cert_verify_mac
0001:000d0513  _ssl3_final_finish_mac
0001:000d07e0  _n_ssl3_mac
0001:000d0a35* _ssl3_record_sequence_update
0001:000d0a69  _ssl3_generate_master_secret
0001:000d0bfd  _ssl3_alert_code
Module: U:\extras\lib\libcrypto.lib(nsseq.obj)
0001:000d0fa0* _NETSCAPE_CERT_SEQUENCE_it
0001:000d0fbc  _d2i_NETSCAPE_CERT_SEQUENCE
0001:000d0fe5  _i2d_NETSCAPE_CERT_SEQUENCE
0001:000d1007* _NETSCAPE_CERT_SEQUENCE_new
0001:000d101b* _NETSCAPE_CERT_SEQUENCE_free
Module: U:\extras\lib\libcrypto.lib(x_long.obj)
0001:000d1050  _LONG_it
0001:000d1080  _ZLONG_it
Module: U:\extras\lib\libcrypto.lib(x_bignum.obj)
0001:000d1320  _BIGNUM_it
0001:000d1340  _CBIGNUM_it
Module: U:\extras\lib\libcrypto.lib(p12_p8d.obj)
0001:000d14c0  _PKCS8_decrypt
Module: U:\extras\lib\libcrypto.lib(pem_pk8.obj)
0001:000d1500* _PEM_write_bio_PKCS8PrivateKey_nid
0001:000d154d  _PEM_write_bio_PKCS8PrivateKey
0001:000d159a* _i2d_PKCS8PrivateKey_bio
0001:000d15e7* _i2d_PKCS8PrivateKey_nid_bio
0001:000d1c95* _PEM_write_bio_PKCS8
0001:000d1db9* _PEM_write_bio_PKCS8_PRIV_KEY_INFO
0001:000d1844* _d2i_PKCS8PrivateKey_bio
0001:000d19a6* _i2d_PKCS8PrivateKey_fp
0001:000d19f3* _i2d_PKCS8PrivateKey_nid_fp
0001:000d1a40* _PEM_write_PKCS8PrivateKey_nid
0001:000d1a8d* _PEM_write_PKCS8PrivateKey
0001:000d1b85* _d2i_PKCS8PrivateKey_fp
0001:000d1c23* _PEM_read_bio_PKCS8
0001:000d1c5c* _PEM_read_PKCS8
0001:000d1ce8* _PEM_write_PKCS8
0001:000d1d47* _PEM_read_bio_PKCS8_PRIV_KEY_INFO
0001:000d1d80* _PEM_read_PKCS8_PRIV_KEY_INFO
0001:000d1e0c* _PEM_write_PKCS8_PRIV_KEY_INFO
Module: U:\extras\lib\libssl.lib(s2_enc.obj)
0001:000d1ed6  _ssl2_enc_init
0001:000d21f5  _ssl2_enc
0001:000d228a  _ssl2_mac
Module: U:\extras\lib\libcrypto.lib(p_verify.obj)
0001:000d23fb  _EVP_VerifyFinal
Module: U:\extras\lib\libcrypto.lib(p_sign.obj)
0001:000d2629  _EVP_SignFinal
Module: U:\extras\lib\libcrypto.lib(ec_lib.obj)
0001:000d289e  _EC_GROUP_new
0001:000d2a0e  _EC_GROUP_free
0001:000d39a6  _EC_EX_DATA_free_all_data
0001:000d3b5f  _EC_POINT_free
0001:000d2aa4  _EC_GROUP_clear_free
0001:000d39fa* _EC_EX_DATA_clear_free_all_data
0001:000d3b97  _EC_POINT_clear_free
0001:000d2b83  _EC_GROUP_copy
0001:000d3751  _EC_EX_DATA_set_data
0001:000d3a4e  _EC_POINT_new
0001:000d3c00  _EC_POINT_copy
0001:000d2e80  _EC_GROUP_dup
0001:000d2f01  _EC_GROUP_method_of
0001:000d2f0b  _EC_METHOD_get_field_type
0001:000d2f15  _EC_GROUP_set_generator
0001:000d3025  _EC_GROUP_get0_generator
0001:000d3030  _EC_GROUP_get_order
0001:000d3066  _EC_GROUP_get_cofactor
0001:000d309c  _EC_GROUP_set_curve_name
0001:000d30aa  _EC_GROUP_get_curve_name
0001:000d30b5  _EC_GROUP_set_asn1_flag
0001:000d30c3  _EC_GROUP_get_asn1_flag
0001:000d30ce  _EC_GROUP_set_point_conversion_form
0001:000d30dc  _EC_GROUP_get_point_conversion_form
0001:000d30e7  _EC_GROUP_set_seed
0001:000d318a  _EC_GROUP_get0_seed
0001:000d3195  _EC_GROUP_get_seed_len
0001:000d31a0  _EC_GROUP_set_curve_GFp
0001:000d3213  _EC_GROUP_get_curve_GFp
0001:000d3286  _EC_GROUP_set_curve_GF2m
0001:000d32f9  _EC_GROUP_get_curve_GF2m
0001:000d336c  _EC_GROUP_get_degree
0001:000d33c3* _EC_GROUP_check_discriminant
0001:000d3421  _EC_GROUP_cmp
0001:000d484d  _EC_POINT_cmp
0001:000d384c  _EC_EX_DATA_get_data
0001:000d3898  _EC_EX_DATA_free_data
0001:000d391f* _EC_EX_DATA_clear_free_data
0001:000d3cae  _EC_POINT_dup
0001:000d3d0e* _EC_POINT_method_of
0001:000d3d18  _EC_POINT_set_to_infinity
0001:000d3db7  _EC_POINT_set_Jprojective_coordinates_GFp
0001:000d3e72* _EC_POINT_get_Jprojective_coordinates_GFp
0001:000d3f2d  _EC_POINT_set_affine_coordinates_GFp
0001:000d3fe1  _EC_POINT_set_affine_coordinates_GF2m
0001:000d4095  _EC_POINT_get_affine_coordinates_GFp
0001:000d4149  _EC_POINT_get_affine_coordinates_GF2m
0001:000d41fd  _EC_POINT_set_compressed_coordinates_GFp
0001:000d42b1  _EC_POINT_set_compressed_coordinates_GF2m
0001:000d4365  _EC_POINT_point2oct
0001:000d4420  _EC_POINT_oct2point
0001:000d44d4  _EC_POINT_add
0001:000d45a7  _EC_POINT_dbl
0001:000d4662  _EC_POINT_invert
0001:000d4708  _EC_POINT_is_at_infinity
0001:000d47a7  _EC_POINT_is_on_curve
0001:000d4908  _EC_POINT_make_affine
0001:000d49ae  _EC_POINTs_make_affine
0001:000d4a7a* _EC_POINTs_mul
0001:000d4aff  _EC_POINT_mul
0001:000d4b5d  _EC_GROUP_precompute_mult
0001:000d4baf  _EC_GROUP_have_precompute_mult
Module: U:\extras\lib\libcrypto.lib(ech_key.obj)
0001:000d4c00  _ECDH_compute_key
Module: U:\extras\lib\libcrypto.lib(pmeth_fn.obj)
0001:000d4c5b  _EVP_PKEY_sign_init
0001:000d4cf4  _EVP_PKEY_sign
0001:000d4e2c  _EVP_PKEY_verify_init
0001:000d4ec5  _EVP_PKEY_verify
0001:000d4f85* _EVP_PKEY_verify_recover_init
0001:000d501e* _EVP_PKEY_verify_recover
0001:000d5156  _EVP_PKEY_encrypt_init
0001:000d51ef  _EVP_PKEY_encrypt
0001:000d5329  _EVP_PKEY_decrypt_init
0001:000d53c2  _EVP_PKEY_decrypt
0001:000d54fc* _EVP_PKEY_derive_init
0001:000d5595  _EVP_PKEY_derive_set_peer
0001:000d582f* _EVP_PKEY_derive
Module: U:\extras\lib\libcrypto.lib(x509type.obj)
0001:000d5960  _X509_certificate_type
Module: U:\extras\lib\libcrypto.lib(hmac.obj)
0001:000d5ad9  _HMAC_Init_ex
0001:000d5d93* _HMAC_Init
0001:000d5e98  _HMAC_CTX_init
0001:000d5dda  _HMAC_Update
0001:000d5dfe  _HMAC_Final
0001:000d5eca  _HMAC_CTX_copy
0001:000d5f6f  _HMAC_CTX_cleanup
0001:000d5fbc  _HMAC
0001:000d6068* _HMAC_CTX_set_flags
Module: U:\extras\lib\libcrypto.lib(ec_curve.obj)
0001:000da1e3  _EC_GROUP_new_by_curve_name
0001:000da29b* _EC_get_builtin_curves
Module: U:\extras\lib\libssl.lib(t1_enc.obj)
0001:000daa68  _tls1_change_cipher_state
0001:000db2c8  _tls1_setup_key_block
0001:000db598  _tls1_enc
0001:000db974  _tls1_cert_verify_mac
0001:000dba9b  _tls1_final_finish_mac
0001:000dbcb3  _tls1_mac
0001:000dbf71  _tls1_generate_master_secret
0001:000dc041  _tls1_alert_code
Module: U:\extras\lib\libssl.lib(t1_reneg.obj)
0001:000dc33b  _ssl_add_clienthello_renegotiate_ext
0001:000dc3f3  _ssl_parse_clienthello_renegotiate_ext
0001:000dc56c  _ssl_add_serverhello_renegotiate_ext
0001:000dc709  _ssl_parse_serverhello_renegotiate_ext
Module: U:\extras\lib\libssl.lib(t1_srvr.obj)
0001:000dc9ad  _TLSv1_server_method
Module: U:\extras\lib\libssl.lib(s23_pkt.obj)
0001:000dca40  _ssl23_write_bytes
0001:000dcadc  _ssl23_read_bytes
Module: U:\extras\lib\libssl.lib(t1_clnt.obj)
0001:000dcb9d  _TLSv1_client_method
Module: U:\extras\lib\libcrypto.lib(bn_asm.obj)
0001:000dcc30  _bn_mul_add_words
0001:000dd0b2  _bn_mul_words
0001:000dd4ae  _bn_sqr_words
0001:000dd705  _bn_div_words
0001:000dd892  _bn_add_words
0001:000dda44  _bn_sub_words
0001:000ddbeb  _bn_mul_comba8
0001:000e2b5a  _bn_mul_comba4
0001:000e3be7  _bn_sqr_comba8
0001:000e6a29  _bn_sqr_comba4
Module: U:\extras\lib\libcrypto.lib(a_bool.obj)
0001:000e73b0* _i2d_ASN1_BOOLEAN
0001:000e7435  _d2i_ASN1_BOOLEAN
Module: U:\extras\lib\libcrypto.lib(b_dump.obj)
0001:000e7510* _BIO_dump_cb
0001:000e7573* _BIO_dump_indent_cb
0001:000e792a* _BIO_dump_fp
0001:000e7953* _BIO_dump_indent_fp
0001:000e79a4* _BIO_dump
0001:000e79cd  _BIO_dump_indent
Module: U:\extras\lib\libcrypto.lib(a_enum.obj)
0001:000e7a09* _ASN1_ENUMERATED_set
0001:000e7b4c  _ASN1_ENUMERATED_get
0001:000e7bf6* _BN_to_ASN1_ENUMERATED
0001:000e7d4c  _ASN1_ENUMERATED_to_BN
Module: U:\extras\lib\libcrypto.lib(f_string.obj)
0001:000e7dd5  _i2a_ASN1_STRING
0001:000e7f0f* _a2i_ASN1_STRING
Module: U:\extras\lib\libcrypto.lib(conf_lib.obj)
0001:000e8300* _CONF_version
0001:000e8327  _CONF_set_nconf
0001:000e835b* _CONF_set_default_method
0001:000e837b* _CONF_load
0001:000e8484* _CONF_load_bio
0001:000e8403* _CONF_load_fp
0001:000e8826* _NCONF_load_bio
0001:000e84ca  _CONF_get_section
0001:000e8885  _NCONF_get_section
0001:000e8503  _CONF_get_string
0001:000e891f  _NCONF_get_string
0001:000e8558* _CONF_get_number
0001:000e89e5* _NCONF_get_number_e
0001:000e85d6  _CONF_free
0001:000e8725* _NCONF_free_data
0001:000e85fb* _CONF_dump_fp
0001:000e8675* _CONF_dump_bio
0001:000e8b38* _NCONF_dump_bio
0001:000e86a1  _NCONF_new
0001:000e8704  _NCONF_free
0001:000e8746  _NCONF_load
0001:000e87a5* _NCONF_load_fp
0001:000e8abe* _NCONF_dump_fp
Module: U:\extras\lib\libcrypto.lib(x509_req.obj)
0001:000e8b9b* _X509_to_X509_REQ
0001:000e8cd1* _X509_REQ_get_pubkey
0001:000e8cff* _X509_REQ_check_private_key
0001:000e8e74* _X509_REQ_extension_nid
0001:000e8eb6* _X509_REQ_get_extension_nids
0001:000e8ec0* _X509_REQ_set_extension_nids
0001:000e8ecd  _X509_REQ_get_extensions
0001:000e9165* _X509_REQ_get_attr_by_NID
0001:000e91b1* _X509_REQ_get_attr
0001:000e8fe7* _X509_REQ_add_extensions_nid
0001:000e912b  _X509_REQ_add_extensions
0001:000e914d* _X509_REQ_get_attr_count
0001:000e918b* _X509_REQ_get_attr_by_OBJ
0001:000e91d0* _X509_REQ_delete_attr
0001:000e91ef* _X509_REQ_add1_attr
0001:000e921e* _X509_REQ_add1_attr_by_OBJ
0001:000e9262* _X509_REQ_add1_attr_by_NID
0001:000e92a6* _X509_REQ_add1_attr_by_txt
Module: U:\extras\lib\libcrypto.lib(conf_mod.obj)
0001:000e934f* _CONF_modules_load
0001:000e9470* _CONF_modules_load_file
0001:000e9df0* _CONF_get1_default_config_file
0001:000e9b9a* _CONF_modules_unload
0001:000e9c74* _CONF_modules_finish
0001:000e9d18* _CONF_module_add
0001:000e9d51* _CONF_modules_free
0001:000e9d6a* _CONF_imodule_get_name
0001:000e9d75* _CONF_imodule_get_value
0001:000e9d80* _CONF_imodule_get_usr_data
0001:000e9d8b* _CONF_imodule_set_usr_data
0001:000e9d99* _CONF_imodule_get_module
0001:000e9da3* _CONF_imodule_get_flags
0001:000e9dae* _CONF_imodule_set_flags
0001:000e9dbc* _CONF_module_get_usr_data
0001:000e9dc7* _CONF_module_set_usr_data
0001:000e9ec1  _CONF_parse_list
Module: U:\extras\lib\libcrypto.lib(evp_key.obj)
0001:000ea020* _EVP_set_pw_prompt
0001:000ea059  _EVP_get_pw_prompt
0001:000ea073* _EVP_read_pw_string
0001:000ea0a3  _EVP_read_pw_string_min
0001:000ea1c6  _EVP_BytesToKey
Module: U:\extras\lib\libcrypto.lib(encode.obj)
0001:000ea4e0  _EVP_EncodeInit
0001:000ea537  _EVP_EncodeUpdate
0001:000ea75e  _EVP_EncodeBlock
0001:000ea6f9  _EVP_EncodeFinal
0001:000ea8a2  _EVP_DecodeInit
0001:000ea8ef  _EVP_DecodeUpdate
0001:000eab99  _EVP_DecodeBlock
0001:000ead15  _EVP_DecodeFinal
Module: U:\extras\lib\libcrypto.lib(tb_pkmeth.obj)
0001:000ead80* _ENGINE_unregister_pkey_meths
0001:000eadaf* _ENGINE_register_pkey_meths
0001:000eae27* _ENGINE_register_all_pkey_meths
0001:000eae58* _ENGINE_set_default_pkey_meths
0001:000eaed0  _ENGINE_get_pkey_meth_engine
0001:000eaef7  _ENGINE_get_pkey_meth
0001:000eaf6e* _ENGINE_get_pkey_meths
0001:000eaf79* _ENGINE_set_pkey_meths
0001:000eaf8c  _engine_pkey_meths_free
Module: U:\extras\lib\libcrypto.lib(eng_ctrl.obj)
0001:000eb452* _ENGINE_ctrl
0001:000eb63b* _ENGINE_cmd_is_executable
0001:000eb6d3* _ENGINE_ctrl_cmd
0001:000eb7d6  _ENGINE_ctrl_cmd_string
Module: U:\extras\lib\libcrypto.lib(pcy_tree.obj)
0001:000ec8bf  _X509_policy_tree_free
0001:000ec9a4  _X509_policy_check
Module: U:\extras\lib\libcrypto.lib(a_utctm.obj)
0001:000ecb60  _ASN1_UTCTIME_check
0001:000ecda8* _ASN1_UTCTIME_set_string
0001:000ece1a* _ASN1_UTCTIME_set
0001:000ece68  _ASN1_UTCTIME_adj
0001:000ed03b* _ASN1_UTCTIME_cmp_time_t
Module: U:\extras\lib\libcrypto.lib(a_gentm.obj)
0001:000ed480  _ASN1_GENERALIZEDTIME_check
0001:000ed720* _ASN1_GENERALIZEDTIME_set_string
0001:000ed792* _ASN1_GENERALIZEDTIME_set
0001:000ed7e0  _ASN1_GENERALIZEDTIME_adj
Module: U:\extras\lib\libcrypto.lib(bn_rand.obj)
0001:000edc92  _BN_rand
0001:000edcc2  _BN_pseudo_rand
0001:000edcf2* _BN_bntest_rand
0001:000edf80  _BN_rand_range
0001:000edfa2  _BN_pseudo_rand_range
Module: U:\extras\lib\libcrypto.lib(p5_crpt.obj)
0001:000edfd0* _PKCS5_PBE_add
0001:000ee03b  _PKCS5_PBE_keyivgen
Module: U:\extras\lib\libcrypto.lib(p12_crpt.obj)
0001:000ee3b0* _PKCS12_PBE_add
0001:000ee3c0  _PKCS12_PBE_keyivgen
Module: U:\extras\lib\libcrypto.lib(p5_crpt2.obj)
0001:000ee650* _PKCS5_PBKDF2_HMAC
0001:000ee83e* _PKCS5_PBKDF2_HMAC_SHA1
0001:000ee8a4  _PKCS5_v2_PBE_keyivgen
Module: U:\extras\lib\libcrypto.lib(bn_exp.obj)
0001:000eede9* _BN_exp
0001:000eefa6  _BN_mod_exp
0001:000f0209  _BN_mod_exp_mont_word
0001:000ef54d  _BN_mod_exp_mont
0001:000ef090* _BN_mod_exp_recp
0001:000efc8f* _BN_mod_exp_mont_consttime
0001:000f072f* _BN_mod_exp_simple
Module: U:\extras\lib\libcrypto.lib(rsa_pk1.obj)
0001:000f0b4a  _RSA_padding_add_PKCS1_type_1
0001:000f0bfb  _RSA_padding_check_PKCS1_type_1
0001:000f0d9b  _RSA_padding_add_PKCS1_type_2
0001:000f0e93  _RSA_padding_check_PKCS1_type_2
Module: U:\extras\lib\libcrypto.lib(rsa_oaep.obj)
0001:000f100b  _RSA_padding_add_PKCS1_OAEP
0001:000f1296  _RSA_padding_check_PKCS1_OAEP
0001:000f15a9  _PKCS1_MGF1
Module: U:\extras\lib\libcrypto.lib(rsa_ssl.obj)
0001:000f173a  _RSA_padding_add_SSLv23
0001:000f1854  _RSA_padding_check_SSLv23
Module: U:\extras\lib\libcrypto.lib(rsa_none.obj)
0001:000f1a2b  _RSA_padding_add_none
0001:000f1ac7  _RSA_padding_check_none
Module: U:\extras\lib\libcrypto.lib(bn_mont.obj)
0001:000f1b60  _BN_mod_mul_montgomery
0001:000f20f0  _BN_from_montgomery
0001:000f2168  _BN_MONT_CTX_new
0001:000f21b4* _BN_MONT_CTX_init
0001:000f220f  _BN_MONT_CTX_free
0001:000f2262  _BN_MONT_CTX_set
0001:000f24d3  _BN_MONT_CTX_copy
0001:000f2579  _BN_MONT_CTX_set_locked
Module: U:\extras\lib\libcrypto.lib(rsa_x931.obj)
0001:000f26bb  _RSA_padding_add_X931
0001:000f2789  _RSA_padding_check_X931
0001:000f2913  _RSA_X931_hash_id
Module: U:\extras\lib\libcrypto.lib(bn_div.obj)
0001:000f2979  _BN_div
Module: U:\extras\lib\libcrypto.lib(bn_mod.obj)
0001:000f3700  _BN_nnmod
0001:000f3778  _BN_mod_add
0001:000f37c4  _BN_mod_add_quick
0001:000f3826* _BN_mod_sub
0001:000f3872  _BN_mod_sub_quick
0001:000f38c8  _BN_mod_mul
0001:000f3983  _BN_mod_sqr
0001:000f39d7* _BN_mod_lshift1
0001:000f3a1c  _BN_mod_lshift1_quick
0001:000f3a77* _BN_mod_lshift
0001:000f3b2b  _BN_mod_lshift_quick
Module: U:\extras\lib\libcrypto.lib(dh_check.obj)
0001:000f3c70* _DH_check
0001:000f3e47  _DH_check_pub_key
Module: U:\extras\lib\libcrypto.lib(dsa_ossl.obj)
0001:000f3f33  _DSA_OpenSSL
Module: U:\extras\lib\libcrypto.lib(tb_dsa.obj)
0001:000f4a54* _ENGINE_unregister_DSA
0001:000f4a83* _ENGINE_register_DSA
0001:000f4acf* _ENGINE_register_all_DSA
0001:000f4b00* _ENGINE_set_default_DSA
0001:000f4b4c  _ENGINE_get_default_DSA
0001:000f4b69  _ENGINE_get_DSA
0001:000f4b74* _ENGINE_set_DSA
Module: U:\extras\lib\libcrypto.lib(x509_def.obj)
0001:000f4ba0* _X509_get_default_private_dir
0001:000f4bb2  _X509_get_default_cert_area
0001:000f4bca  _X509_get_default_cert_dir
0001:000f4be5  _X509_get_default_cert_file
0001:000f4bfc  _X509_get_default_cert_dir_env
0001:000f4c14  _X509_get_default_cert_file_env
Module: U:\extras\lib\libcrypto.lib(pem_info.obj)
0001:000f4c2b* _PEM_X509_INFO_read
0001:000f4d38  _PEM_X509_INFO_read_bio
0001:000f547d* _PEM_X509_INFO_write_bio
Module: U:\extras\lib\libcrypto.lib(x_info.obj)
0001:000f5729  _X509_INFO_new
0001:000f57d8  _X509_INFO_free
Module: U:\extras\lib\libcrypto.lib(rsa_pmeth.obj)
0001:000f6960  _rsa_pkey_meth
Module: U:\extras\lib\libcrypto.lib(dh_pmeth.obj)
0001:000f6e10  _dh_pkey_meth
Module: U:\extras\lib\libcrypto.lib(dsa_pmeth.obj)
0001:000f7580  _dsa_pkey_meth
Module: U:\extras\lib\libcrypto.lib(ec_pmeth.obj)
0001:000f7d00  _ec_pkey_meth
Module: U:\extras\lib\libcrypto.lib(hm_pmeth.obj)
0001:000f81f0  _hmac_pkey_meth
Module: U:\extras\lib\libcrypto.lib(t_pkey.obj)
0001:000f8299  _ASN1_bn_print
Module: U:\extras\lib\libcrypto.lib(pk7_lib.obj)
0001:000f84ea  _PKCS7_ctrl
0001:000f866b* _PKCS7_content_new
0001:000f8791  _PKCS7_set_type
0001:000f86d8* _PKCS7_set_content
0001:000f8a2d* _PKCS7_set0_type_other
0001:000f8a54* _PKCS7_add_signer
0001:000f8c1d* _PKCS7_add_certificate
0001:000f8d45* _PKCS7_add_crl
0001:000f8e6d* _PKCS7_SIGNER_INFO_set
0001:000f9022* _PKCS7_add_signature
0001:000f9108* _PKCS7_set_digest
0001:000f91df* _PKCS7_get_signer_info
0001:000f9228  _PKCS7_SIGNER_INFO_get0_algs
0001:000f9260  _PKCS7_RECIP_INFO_get0_alg
0001:000f9276* _PKCS7_add_recipient
0001:000f9371* _PKCS7_RECIP_INFO_set
0001:000f92da* _PKCS7_add_recipient_info
0001:000f955f* _PKCS7_cert_from_signer_info
0001:000f95ab* _PKCS7_set_cipher
0001:000f9675  _PKCS7_stream
Module: U:\extras\lib\libcrypto.lib(cms_sd.obj)
0001:000f98ac* _CMS_SignedData_init
0001:000fa47a* _CMS_get0_SignerInfos
0001:000f9bdf  _cms_set1_SignerIdentifier
0001:000f9d47  _cms_SignerIdentifier_get0_signer_id
0001:000f9da7  _cms_SignerIdentifier_cert_cmp
0001:000f9e5c* _CMS_add1_signer
0001:000fb3af* _CMS_add_standard_smimecap
0001:000fb1d1* _CMS_add_smimecap
0001:000faa82* _CMS_SignerInfo_sign
0001:000fa4a3* _CMS_get0_signers
0001:000fa544* _CMS_SignerInfo_set1_signer_cert
0001:000fa5ca* _CMS_SignerInfo_get0_signer_id
0001:000fa5f5* _CMS_SignerInfo_cert_cmp
0001:000fa612* _CMS_set1_signers_certs
0001:000fa787  _CMS_SignerInfo_get0_algs
0001:000faa02  _cms_SignedData_final
0001:000fad36* _CMS_SignerInfo_verify
0001:000faed4  _cms_SignedData_init_bio
0001:000fafa3* _CMS_SignerInfo_verify_content
0001:000fb23c* _CMS_add_simple_smimecap
Module: U:\extras\lib\libcrypto.lib(cms_env.obj)
0001:000fb62d* _CMS_get0_RecipientInfos
0001:000fb656* _CMS_RecipientInfo_type
0001:000fb660* _CMS_EnvelopedData_create
0001:000fb701* _CMS_add1_recipient_cert
0001:000fb998  _CMS_RecipientInfo_ktri_get0_algs
0001:000fba1d* _CMS_RecipientInfo_ktri_get0_signer_id
0001:000fba8d* _CMS_RecipientInfo_ktri_cert_cmp
0001:000fbae9* _CMS_RecipientInfo_set0_pkey
0001:000fbfbc* _CMS_RecipientInfo_kekri_id_cmp
0001:000fc072* _CMS_add0_recipient_key
0001:000fc318* _CMS_RecipientInfo_kekri_get0_id
0001:000fc3f7* _CMS_RecipientInfo_set0_key
0001:000fc8b7* _CMS_RecipientInfo_decrypt
0001:000fc928  _cms_EnvelopedData_init_bio
Module: U:\extras\lib\libcrypto.lib(ecs_lib.obj)
0001:000fcac0* _ECDSA_version
0001:000fcae8* _ECDSA_set_default_method
0001:000fcaf5* _ECDSA_get_default_method
0001:000fcb15* _ECDSA_set_method
0001:000fcd3f  _ecdsa_check
0001:000fcdbd  _ECDSA_size
0001:000fcebe* _ECDSA_get_ex_new_index
0001:000fcef5* _ECDSA_set_ex_data
0001:000fcf34* _ECDSA_get_ex_data
Module: U:\extras\lib\libcrypto.lib(ec_print.obj)
0001:000fcf7b  _EC_POINT_point2bn
0001:000fd066* _EC_POINT_bn2point
0001:000fd198* _EC_POINT_point2hex
0001:000fd307* _EC_POINT_hex2point
Module: U:\extras\lib\libcrypto.lib(eck_prn.obj)
0001:000fd37a* _ECPKParameters_print_fp
0001:000fd67c  _ECPKParameters_print
0001:000fd417* _EC_KEY_print_fp
0001:000fd54a* _EC_KEY_print
0001:000fd4b4* _ECParameters_print_fp
0001:000fd5af* _ECParameters_print
Module: U:\extras\lib\libcrypto.lib(a_bytes.obj)
0001:000fe05a* _d2i_ASN1_type_bytes
0001:000fe24b  _i2d_ASN1_bytes
0001:000fe337* _d2i_ASN1_bytes
Module: U:\extras\lib\libcrypto.lib(o_time.obj)
0001:000fe7c0  _OPENSSL_gmtime
0001:000fe80d  _OPENSSL_gmtime_adj
Module: U:\extras\lib\libcrypto.lib(cbc128.obj)
0001:000fece0  _CRYPTO_cbc128_encrypt
0001:000fee0c  _CRYPTO_cbc128_decrypt
Module: U:\extras\lib\libcrypto.lib(cfb128.obj)
0001:000fefd0  _CRYPTO_cfb128_encrypt
0001:000ff3d1  _CRYPTO_cfb128_1_encrypt
0001:000ff4ae  _CRYPTO_cfb128_8_encrypt
Module: U:\extras\lib\libcrypto.lib(ofb128.obj)
0001:000ff510  _CRYPTO_ofb128_encrypt
Module: U:\extras\lib\libcrypto.lib(camellia.obj)
0001:00100650  _Camellia_Ekeygen
0001:00101e7b  _Camellia_EncryptBlock_Rounds
0001:00102536* _Camellia_EncryptBlock
0001:00102570  _Camellia_DecryptBlock_Rounds
0001:00102c26* _Camellia_DecryptBlock
Module: U:\extras\lib\libcrypto.lib(ecs_asn1.obj)
0001:00102cb0* _ECDSA_SIG_it
0001:00102ccc  _d2i_ECDSA_SIG
0001:00102cf5  _i2d_ECDSA_SIG
0001:00102d17  _ECDSA_SIG_new
0001:00102d2b  _ECDSA_SIG_free
Module: U:\extras\lib\libcrypto.lib(xcbc_enc.obj)
0001:00102d50  _DES_xcbc_encrypt
Module: U:\extras\lib\libcrypto.lib(bf_enc.obj)
0001:001035e0  _BF_encrypt
0001:00103c48  _BF_decrypt
0001:001042b0  _BF_cbc_encrypt
Module: U:\extras\lib\libcrypto.lib(bf_cfb64.obj)
0001:00104a00  _BF_cfb64_encrypt
Module: U:\extras\lib\libcrypto.lib(bf_ecb.obj)
0001:00104d10* _BF_version
0001:00104d49* _BF_options
0001:00104d53  _BF_ecb_encrypt
Module: U:\extras\lib\libcrypto.lib(bf_ofb64.obj)
0001:00104eb0  _BF_ofb64_encrypt
Module: U:\extras\lib\libcrypto.lib(bf_skey.obj)
0001:00106118  _BF_set_key
Module: U:\extras\lib\libcrypto.lib(c_enc.obj)
0001:001062b0  _CAST_encrypt
0001:00106a89  _CAST_decrypt
0001:00107262  _CAST_cbc_encrypt
Module: U:\extras\lib\libcrypto.lib(c_cfb64.obj)
0001:001079b0  _CAST_cfb64_encrypt
Module: U:\extras\lib\libcrypto.lib(c_ecb.obj)
0001:00107cc0* _CAST_version
0001:00107ce7  _CAST_ecb_encrypt
Module: U:\extras\lib\libcrypto.lib(c_ofb64.obj)
0001:00107e50  _CAST_ofb64_encrypt
Module: U:\extras\lib\libcrypto.lib(c_skey.obj)
0001:00108070  _CAST_S_table0
0001:00108470  _CAST_S_table1
0001:00108870  _CAST_S_table2
0001:00108c70  _CAST_S_table3
0001:00109070* _CAST_S_table4
0001:00109470* _CAST_S_table5
0001:00109870* _CAST_S_table6
0001:00109c70* _CAST_S_table7
0001:0010a070  _CAST_set_key
Module: U:\extras\lib\libcrypto.lib(md4_dgst.obj)
0001:0010ae30  _MD4_Update
0001:0010b1d5* _md4_block_data_order
0001:0010afe7* _MD4_Transform
0001:0010b009  _MD4_Final
0001:0010b160* _MD4_version
0001:0010b186  _MD4_Init
Module: U:\extras\lib\libcrypto.lib(sha_dgst.obj)
0001:0010ba50* _SHA_version
0001:0010ba76  _SHA_Update
0001:0010bc2d* _SHA_Transform
0001:0010bc4f  _SHA_Final
0001:0010be30  _SHA_Init
Module: U:\extras\lib\libcrypto.lib(mdc2dgst.obj)
0001:0010e170  _MDC2_Init
0001:0010e1cc  _MDC2_Update
0001:0010e579  _MDC2_Final
Module: U:\extras\lib\libcrypto.lib(rsa_saos.obj)
0001:0010e64b  _RSA_sign_ASN1_OCTET_STRING
0001:0010e7a5  _RSA_verify_ASN1_OCTET_STRING
Module: U:\extras\lib\libcrypto.lib(rmd_dgst.obj)
0001:0010e950  _RIPEMD160_Update
0001:0010ed26* _ripemd160_block_data_order
0001:0010eb07* _RIPEMD160_Transform
0001:0010eb29  _RIPEMD160_Final
0001:0010eca0* _RMD160_version
0001:0010eccd  _RIPEMD160_Init
Module: U:\extras\lib\libcrypto.lib(wp_dgst.obj)
0001:001118e0  _WHIRLPOOL_Init
0001:00111908  _WHIRLPOOL_Update
0001:00111976* _WHIRLPOOL_BitUpdate
0001:00111dac  _WHIRLPOOL_Final
0001:00111f4b* _WHIRLPOOL
Module: U:\extras\lib\libcrypto.lib(pk7_doit.obj)
0001:00112593  _PKCS7_dataInit
0001:00112b86* _PKCS7_dataDecode
0001:00114315  _PKCS7_get_signed_attribute
0001:00113a62* _PKCS7_SIGNER_INFO_sign
0001:001134b8  _PKCS7_dataFinal
0001:00113cd9* _PKCS7_dataVerify
0001:00113ea1* _PKCS7_signatureVerify
0001:00114404* _PKCS7_digest_from_attributes
0001:0011427d* _PKCS7_get_issuer_and_serial
0001:00114332* _PKCS7_get_attribute
0001:00114435* _PKCS7_set_signed_attributes
0001:001144e1* _PKCS7_set_attributes
0001:0011458d  _PKCS7_add_signed_attribute
0001:001145b8* _PKCS7_add_attribute
Module: U:\extras\lib\libcrypto.lib(tasn_prn.obj)
0001:0011474b* _ASN1_PCTX_new
0001:001147df* _ASN1_PCTX_free
0001:001147f2* _ASN1_PCTX_get_flags
0001:001147fc* _ASN1_PCTX_set_flags
0001:00114809* _ASN1_PCTX_get_nm_flags
0001:00114814* _ASN1_PCTX_set_nm_flags
0001:00114822* _ASN1_PCTX_get_cert_flags
0001:0011482d* _ASN1_PCTX_set_cert_flags
0001:0011483b* _ASN1_PCTX_get_oid_flags
0001:00114846* _ASN1_PCTX_set_oid_flags
0001:00114854* _ASN1_PCTX_get_str_flags
0001:0011485f* _ASN1_PCTX_set_str_flags
0001:0011486d  _ASN1_item_print
0001:00114ebf* _asn1_template_print_ctx
0002:00006f20* _default_pctx
Module: U:\extras\lib\libcrypto.lib(ec2_smpl.obj)
0001:00115850  _EC_GF2m_simple_method
0001:0011585a* _ec_GF2m_simple_group_init
0001:00115893* _ec_GF2m_simple_group_finish
0001:001158c7* _ec_GF2m_simple_group_clear_finish
0001:00115937* _ec_GF2m_simple_group_copy
0001:00115b3e  _ec_GF2m_simple_group_set_curve
0001:00115d58* _ec_GF2m_simple_group_get_curve
0001:00115ddd* _ec_GF2m_simple_group_get_degree
0001:00115df4* _ec_GF2m_simple_group_check_discriminant
0001:00115ed5* _ec_GF2m_simple_point_init
0001:00115f0c* _ec_GF2m_simple_point_finish
0001:00115f3e* _ec_GF2m_simple_point_clear_finish
0001:00115f7a* _ec_GF2m_simple_point_copy
0001:00115ffc* _ec_GF2m_simple_point_set_to_infinity
0001:00116029* _ec_GF2m_simple_point_set_affine_coordinates
0001:0011612a* _ec_GF2m_simple_point_get_affine_coordinates
0001:00116247* _ec_GF2m_simple_set_compressed_coordinates
0001:00116593* _ec_GF2m_simple_point2oct
0001:001169de* _ec_GF2m_simple_oct2point
0001:00116e65* _ec_GF2m_simple_add
0001:001173f6* _ec_GF2m_simple_dbl
0001:00117425* _ec_GF2m_simple_invert
0001:0011749a* _ec_GF2m_simple_is_at_infinity
0001:001174ad* _ec_GF2m_simple_is_on_curve
0001:001176c8* _ec_GF2m_simple_cmp
0001:001178c0* _ec_GF2m_simple_make_affine
0001:00117a07* _ec_GF2m_simple_points_make_affine
0001:00117a59* _ec_GF2m_simple_field_mul
0001:00117a8b* _ec_GF2m_simple_field_sqr
0001:00117ab6* _ec_GF2m_simple_field_div
Module: U:\extras\lib\libcrypto.lib(ec_cvt.obj)
0001:00117b90  _EC_GROUP_new_curve_GFp
0001:00117ca3  _EC_GROUP_new_curve_GF2m
Module: U:\extras\lib\libcrypto.lib(x509_att.obj)
0001:00117d10  _X509at_get_attr_count
0001:00117d23  _X509at_get_attr_by_NID
0001:00117d5f  _X509at_get_attr_by_OBJ
0001:00117dd6  _X509at_get_attr
0001:00117e13  _X509at_delete_attr
0001:00117e61  _X509at_add1_attr
0001:00117f66  _X509at_add1_attr_by_OBJ
0001:001181cc* _X509_ATTRIBUTE_create_by_OBJ
0001:00117fc9  _X509at_add1_attr_by_NID
0001:0011813f* _X509_ATTRIBUTE_create_by_NID
0001:0011802c  _X509at_add1_attr_by_txt
0001:001182af* _X509_ATTRIBUTE_create_by_txt
0001:0011808f  _X509at_get0_data_by_OBJ
0001:00118574* _X509_ATTRIBUTE_count
0001:001185c3* _X509_ATTRIBUTE_get0_data
0001:00118359* _X509_ATTRIBUTE_set1_object
0001:00118396* _X509_ATTRIBUTE_set1_data
0001:001185ac* _X509_ATTRIBUTE_get0_object
0001:00118636* _X509_ATTRIBUTE_get0_type
Module: U:\extras\lib\libcrypto.lib(p12_decr.obj)
0001:0011869b* _PKCS12_pbe_crypt
0001:0011884d  _PKCS12_item_decrypt_d2i
0001:00118955  _PKCS12_item_i2d_encrypt
Module: U:\extras\lib\libcrypto.lib(p12_p8e.obj)
0001:00118aba  _PKCS8_encrypt
Module: U:\extras\lib\libcrypto.lib(ec_mult.obj)
0001:00119252  _ec_wNAF_mul
0001:0011a028  _ec_wNAF_precompute_mult
0001:0011a65f  _ec_wNAF_have_precompute_mult
Module: U:\extras\lib\libcrypto.lib(ech_lib.obj)
0001:0011a6a0* _ECDH_version
0001:0011a6c7* _ECDH_set_default_method
0001:0011a6d4* _ECDH_get_default_method
0001:0011a6f4* _ECDH_set_method
0001:0011a91e  _ecdh_check
0001:0011a99c* _ECDH_get_ex_new_index
0001:0011a9d3* _ECDH_set_ex_data
0001:0011aa12* _ECDH_get_ex_data
Module: U:\extras\lib\libcrypto.lib(pmeth_gn.obj)
0001:0011aa5b* _EVP_PKEY_paramgen_init
0001:0011aaf4* _EVP_PKEY_paramgen
0001:0011abe6* _EVP_PKEY_keygen_init
0001:0011ac7f* _EVP_PKEY_keygen
0001:0011ad71* _EVP_PKEY_CTX_set_cb
0001:0011ad7f* _EVP_PKEY_CTX_get_cb
0001:0011adc2  _evp_pkey_set_cb_translate
0001:0011adec* _EVP_PKEY_CTX_get_keygen_info
0001:0011ae27  _EVP_PKEY_new_mac_key
Module: U:\extras\lib\libcrypto.lib(m_sigver.obj)
0001:0011b0de  _EVP_DigestSignInit
0001:0011b115  _EVP_DigestVerifyInit
0001:0011b14c  _EVP_DigestSignFinal
0001:0011b2e6  _EVP_DigestVerifyFinal
Module: U:\extras\lib\libcrypto.lib(conf_def.obj)
0001:0011b3e0* _CONF_def_version
0001:0011b421  _NCONF_default
0001:0011b42b* _NCONF_WIN32
Module: U:\extras\lib\libcrypto.lib(conf_api.obj)
0001:0011c9df  __CONF_get_section
0001:0011ca22  __CONF_get_section_values
0001:0011ca52  __CONF_add_string
0001:0011caf9  __CONF_get_string
0001:0011ccd3  __CONF_new_data
0001:0011cd24  __CONF_free_data
0001:0011ce6e  __CONF_new_section
Module: U:\extras\lib\libcrypto.lib(x509rset.obj)
0001:0011cfb0* _X509_REQ_set_version
0001:0011cfdc  _X509_REQ_set_subject_name
0001:0011d011  _X509_REQ_set_pubkey
Module: U:\extras\lib\libcrypto.lib(dso_lib.obj)
0001:0011d050* _DSO_new
0001:0011d0aa* _DSO_new_method
0001:0011d064* _DSO_set_default_method
0001:0011d071* _DSO_get_default_method
0001:0011d07b* _DSO_get_method
0001:0011d085* _DSO_set_method
0001:0011d1ea  _DSO_free
0001:0011d366* _DSO_flags
0001:0011d37e* _DSO_up_ref
0001:0011d3f2  _DSO_load
0001:0011d7df* _DSO_ctrl
0001:0011d97f* _DSO_set_filename
0001:0011d613* _DSO_bind_var
0001:0011d6f9  _DSO_bind_func
0001:0011d8d8* _DSO_set_name_converter
0001:0011d938* _DSO_get_filename
0001:0011dab1* _DSO_merge
0001:0011db67* _DSO_convert_filename
0001:0011dce3* _DSO_get_loaded_filename
0001:0011dd2a* _DSO_pathbyaddr
0001:0011dda1* _DSO_global_lookup
Module: U:\extras\lib\libcrypto.lib(ui_lib.obj)
0001:0011de10  _UI_new
0001:0011de2d* _UI_new_method
0001:0011ee64* _UI_get_default_method
0001:0011df4a  _UI_free
0001:0011e2c1  _UI_add_input_string
0001:0011e30f* _UI_dup_input_string
0001:0011e3b1  _UI_add_verify_string
0001:0011e3fe* _UI_dup_verify_string
0001:0011e49f* _UI_add_input_boolean
0001:0011e4ec* _UI_dup_input_boolean
0001:0011e6c9* _UI_add_info_string
0001:0011e71b* _UI_dup_info_string
0001:0011e7c1* _UI_add_error_string
0001:0011e813* _UI_dup_error_string
0001:0011e8c2* _UI_construct_prompt
0001:0011ea2d* _UI_add_user_data
0001:0011ea4a* _UI_get0_user_data
0001:0011ea55* _UI_get0_result
0001:0011f0e9  _UI_get0_result_string
0001:0011eb5c  _UI_process
0001:0011ed0b* _UI_ctrl
0001:0011eddf* _UI_get_ex_new_index
0001:0011ee16* _UI_set_ex_data
0001:0011ee3a* _UI_get_ex_data
0001:0011ee57* _UI_set_default_method
0001:0011ee84* _UI_get_method
0001:0011ee8e* _UI_set_method
0001:0011eea0* _UI_create_method
0001:0011eefb* _UI_destroy_method
0001:0011ef24* _UI_method_set_opener
0001:0011ef44* _UI_method_set_writer
0001:0011ef64* _UI_method_set_flusher
0001:0011ef84* _UI_method_set_reader
0001:0011efa4* _UI_method_set_closer
0001:0011efc4* _UI_method_set_prompt_constructor
0001:0011efe4* _UI_method_get_opener
0001:0011effc* _UI_method_get_writer
0001:0011f014* _UI_method_get_flusher
0001:0011f02c* _UI_method_get_reader
0001:0011f044* _UI_method_get_closer
0001:0011f05c* _UI_method_get_prompt_constructor
0001:0011f074  _UI_get_string_type
0001:0011f08b  _UI_get_input_flags
0001:0011f0a3  _UI_get0_output_string
0001:0011f0bb  _UI_get0_action_string
0001:0011f113  _UI_get0_test_string
0001:0011f13c* _UI_get_result_minsize
0001:0011f166* _UI_get_result_maxsize
0001:0011f1b6  _UI_set_result
Module: U:\extras\lib\libcrypto.lib(pcy_node.obj)
0001:0011f4b8  _policy_node_cmp_new
0001:0011f4cd  _tree_find_sk
0001:0011f515  _level_find_node
0001:0011f58f  _level_add_node
0001:0011f6c4  _policy_node_free
0001:0011f6d7  _policy_node_match
Module: U:\extras\lib\libcrypto.lib(pcy_lib.obj)
0001:0011f790* _X509_policy_tree_level_count
0001:0011f7a8* _X509_policy_tree_get0_level
0001:0011f7d8* _X509_policy_tree_get0_policies
0001:0011f7f0  _X509_policy_tree_get0_user_policies
0001:0011f81d* _X509_policy_level_node_count
0001:0011f86a* _X509_policy_level_get0_node
0001:0011f8af* _X509_policy_node_get0_policy
0001:0011f8c9* _X509_policy_node_get0_qualifiers
0001:0011f8e3* _X509_policy_node_get0_parent
Module: U:\extras\lib\libcrypto.lib(p5_pbe.obj)
0001:0011f950* _PBEPARAM_it
0001:0011f96c  _d2i_PBEPARAM
0001:0011f995* _i2d_PBEPARAM
0001:0011f9b7* _PBEPARAM_new
0001:0011f9cb  _PBEPARAM_free
0001:0011f9ef* _PKCS5_pbe_set0_algor
0001:0011fc04  _PKCS5_pbe_set
Module: U:\extras\lib\libcrypto.lib(p12_key.obj)
0001:0011fc9a  _PKCS12_key_gen_asc
0001:0011fd8b* _PKCS12_key_gen_uni
Module: U:\extras\lib\libcrypto.lib(p5_pbev2.obj)
0001:001202f0* _PBE2PARAM_it
0001:0012030c  _d2i_PBE2PARAM
0001:00120335* _i2d_PBE2PARAM
0001:00120357* _PBE2PARAM_new
0001:0012036b  _PBE2PARAM_free
0001:00120400* _PBKDF2PARAM_it
0001:0012041c  _d2i_PBKDF2PARAM
0001:00120445* _i2d_PBKDF2PARAM
0001:00120467* _PBKDF2PARAM_new
0001:0012047b  _PBKDF2PARAM_free
0001:001204a1* _PKCS5_pbe2_set_iv
0001:001209dd  _PKCS5_pbe2_set
Module: U:\extras\lib\libcrypto.lib(bn_sqr.obj)
0001:00120a20  _BN_sqr
0001:00120cc3* _bn_sqr_normal
0001:00120df2* _bn_sqr_recursive
Module: U:\extras\lib\libcrypto.lib(bn_recp.obj)
0001:001210a0  _BN_RECP_CTX_init
0001:001210df* _BN_RECP_CTX_new
0001:0012112b  _BN_RECP_CTX_free
0001:0012116d  _BN_RECP_CTX_set
0001:001211c8  _BN_mod_mul_reciprocal
0001:00121298* _BN_div_recp
0001:001215c3* _BN_reciprocal
Module: U:\extras\lib\libcrypto.lib(bn_prime.obj)
0001:00122650  _BN_GENCB_call
0001:001226d0  _BN_generate_prime_ex
0001:00122a1b  _BN_is_prime_fasttest_ex
0001:001229eb  _BN_is_prime_ex
Module: U:\extras\lib\libcrypto.lib(bn_exp2.obj)
0001:001234ca  _BN_mod_exp2_mont
Module: U:\extras\lib\libcrypto.lib(x_pkey.obj)
0001:00123cb0* _i2d_X509_PKEY
0001:00123cc3* _d2i_X509_PKEY
0001:00123f53  _X509_PKEY_new
0001:0012406b  _X509_PKEY_free
Module: U:\extras\lib\libcrypto.lib(rsa_pss.obj)
0001:00124142  _RSA_verify_PKCS1_PSS
0001:00124593  _RSA_padding_add_PKCS1_PSS
Module: U:\extras\lib\libcrypto.lib(rsa_gen.obj)
0001:001248c0  _RSA_generate_key_ex
Module: U:\extras\lib\libcrypto.lib(dh_gen.obj)
0001:00125140  _DH_generate_parameters_ex
Module: U:\extras\lib\libcrypto.lib(dsa_gen.obj)
0001:00125440* _DSA_generate_parameters_ex
0001:00125519  _dsa_builtin_paramgen
Module: U:\extras\lib\libcrypto.lib(dsa_key.obj)
0001:00125e60  _DSA_generate_key
Module: U:\extras\lib\libcrypto.lib(cms_asn1.obj)
0001:001260c0  _CMS_IssuerAndSerialNumber_it
0001:00126150* _CMS_OtherCertificateFormat_it
0001:00126240  _CMS_CertificateChoices_it
0001:001262d0* _CMS_SignerIdentifier_it
0001:00126360* _CMS_EncapsulatedContentInfo_it
0001:001264e0  _CMS_SignerInfo_it
0001:00126570* _CMS_OtherRevocationInfoFormat_it
0001:001265f0  _CMS_RevocationInfoChoice_it
0001:001266e0  _CMS_SignedData_it
0001:00126740* _CMS_OriginatorInfo_it
0001:00126800* _CMS_EncryptedContentInfo_it
0001:001268c0  _CMS_KeyTransRecipientInfo_it
0001:00126930  _CMS_OtherKeyAttribute_it
0001:001269d0* _CMS_RecipientKeyIdentifier_it
0001:00126a50* _CMS_KeyAgreeRecipientIdentifier_it
0001:00126ac0* _CMS_RecipientEncryptedKey_it
0001:00126b30* _CMS_OriginatorPublicKey_it
0001:00126bc0* _CMS_OriginatorIdentifierOrKey_it
0001:00126c90* _CMS_KeyAgreeRecipientInfo_it
0001:00126d10* _CMS_KEKIdentifier_it
0001:00126db0  _CMS_KEKRecipientInfo_it
0001:00126e60* _CMS_PasswordRecipientInfo_it
0001:00126ed0* _CMS_OtherRecipientInfo_it
0001:00127060  _CMS_RecipientInfo_it
0001:00127140  _CMS_EnvelopedData_it
0001:001271e0  _CMS_DigestedData_it
0001:00127250  _CMS_EncryptedData_it
0001:00127370* _CMS_AuthenticatedData_it
0001:00127400* _CMS_CompressedData_it
0001:00127690  _CMS_ContentInfo_it
0001:001276f0  _CMS_Attributes_Sign_it
0001:00127740  _CMS_Attributes_Verify_it
0001:001277c0* _CMS_ReceiptsFrom_it
0001:00127860* _CMS_ReceiptRequest_it
0001:00127900* _CMS_Receipt_it
Module: U:\extras\lib\libcrypto.lib(cms_att.obj)
0001:00127920  _CMS_signed_get_attr_count
0001:00127936  _CMS_signed_get_attr_by_NID
0001:0012795a* _CMS_signed_get_attr_by_OBJ
0001:0012797e* _CMS_signed_get_attr
0001:0012799b* _CMS_signed_delete_attr
0001:001279b8* _CMS_signed_add1_attr
0001:001279e5* _CMS_signed_add1_attr_by_OBJ
0001:00127a27  _CMS_signed_add1_attr_by_NID
0001:00127a69* _CMS_signed_add1_attr_by_txt
0001:00127aab  _CMS_signed_get0_data_by_OBJ
0001:00127ad6* _CMS_unsigned_get_attr_count
0001:00127aec* _CMS_unsigned_get_attr_by_NID
0001:00127b10* _CMS_unsigned_get_attr_by_OBJ
0001:00127b34* _CMS_unsigned_get_attr
0001:00127b51* _CMS_unsigned_delete_attr
0001:00127b6e* _CMS_unsigned_add1_attr
0001:00127b9b* _CMS_unsigned_add1_attr_by_OBJ
0001:00127bdd* _CMS_unsigned_add1_attr_by_NID
0001:00127c1f* _CMS_unsigned_add1_attr_by_txt
0001:00127c61* _CMS_unsigned_get0_data_by_OBJ
Module: U:\extras\lib\libcrypto.lib(cms_lib.obj)
0001:00127c90  _d2i_CMS_ContentInfo
0001:00127cb9  _i2d_CMS_ContentInfo
0001:00127cdb  _CMS_ContentInfo_new
0001:00127cef  _CMS_ContentInfo_free
0001:00127d0a* _CMS_ContentInfo_print_ctx
0001:00127d3a* _CMS_get0_type
0001:00127d44* _priv_cms_Data_create
0001:00128373* _CMS_set_detached
0001:00127d81* _cms_content_bio
0001:00128108  _CMS_get0_content
0001:00127e06  _CMS_dataInit
0001:00127f49  _CMS_dataFinal
0001:001282ae  _CMS_get0_eContentType
0001:001282d6* _CMS_set1_eContentType
0001:0012833b* _CMS_is_detached
0001:0012842c  _cms_DigestAlgorithm_set
0001:00128482  _cms_DigestAlgorithm_init_bio
0001:0012858a  _cms_DigestAlgorithm_find_ctx
0001:001286f7* _CMS_add0_CertificateChoices
0001:00128790* _CMS_add0_cert
0001:00128886  _CMS_add1_cert
0001:00128945* _CMS_add0_RevocationInfoChoice
0001:001289de* _CMS_add0_crl
0001:00128a18* _CMS_add1_crl
0001:00128a6c* _CMS_get1_certs
0001:00128b68* _CMS_get1_crls
Module: U:\extras\lib\libcrypto.lib(cms_enc.obj)
0001:00128c7a  _cms_EncryptedContent_init_bio
0001:0012912d  _cms_EncryptedContent_init
0001:001291b9* _CMS_EncryptedData_set1_key
0001:001292ed  _cms_EncryptedData_init_bio
Module: U:\extras\lib\libcrypto.lib(aes_wrap.obj)
0001:00129338  _AES_wrap_key
0001:001294c8  _AES_unwrap_key
Module: U:\extras\lib\libcrypto.lib(ecs_ossl.obj)
0001:001296a5  _ECDSA_OpenSSL
Module: U:\extras\lib\libcrypto.lib(tb_ecdsa.obj)
0001:0012a6e4* _ENGINE_unregister_ECDSA
0001:0012a713* _ENGINE_register_ECDSA
0001:0012a75f* _ENGINE_register_all_ECDSA
0001:0012a790* _ENGINE_set_default_ECDSA
0001:0012a7dc  _ENGINE_get_default_ECDSA
0001:0012a7f9  _ENGINE_get_ECDSA
0001:0012a804* _ENGINE_set_ECDSA
Module: U:\extras\lib\libcrypto.lib(wp_block.obj)
0001:0012b870  _whirlpool_block
Module: U:\extras\lib\libcrypto.lib(bio_md.obj)
0001:0012d9ef  _BIO_f_md
Module: U:\extras\lib\libcrypto.lib(bio_enc.obj)
0001:0012de87  _BIO_f_cipher
0001:0012e7ca* _BIO_set_cipher
Module: U:\extras\lib\libcrypto.lib(bss_null.obj)
0001:0012e8b5  _BIO_s_null
Module: U:\extras\lib\libcrypto.lib(pk7_attr.obj)
0001:0012e9bb* _PKCS7_add_attrib_smimecap
0001:0012ea48* _PKCS7_get_smimecap
0001:0012eab0* _PKCS7_simple_smimecap
0001:0012ec27* _PKCS7_add_attrib_content_type
0001:0012ec84  _PKCS7_add0_attrib_signing_time
0001:0012ed04  _PKCS7_add1_attrib_digest
Module: U:\extras\lib\libcrypto.lib(bn_gf2m.obj)
0001:0012f041  _BN_GF2m_add
0001:0012f186  _BN_GF2m_mod_arr
0001:0012f5f0* _BN_GF2m_mod
0001:00130a3e  _BN_GF2m_poly2arr
0001:0012f6c7  _BN_GF2m_mod_mul_arr
0001:0012fa33  _BN_GF2m_mod_sqr_arr
0001:0012f94a* _BN_GF2m_mod_mul
0001:0012fc77* _BN_GF2m_mod_sqr
0001:0012fd55* _BN_GF2m_mod_inv
0001:0012ff90* _BN_GF2m_mod_inv_arr
0001:00130afa* _BN_GF2m_arr2poly
0001:0013000b  _BN_GF2m_mod_div
0001:001300ad* _BN_GF2m_mod_div_arr
0001:0013012f* _BN_GF2m_mod_exp_arr
0001:0013029a* _BN_GF2m_mod_exp
0001:00130383  _BN_GF2m_mod_sqrt_arr
0001:0013042b* _BN_GF2m_mod_sqrt
0001:00130509  _BN_GF2m_mod_solve_quad_arr
0001:00130960* _BN_GF2m_mod_solve_quad
Module: U:\extras\lib\libcrypto.lib(ec2_mult.obj)
0001:00131780  _ec_GF2m_simple_mul
0001:00131a45  _ec_GF2m_precompute_mult
0001:00131a5f  _ec_GF2m_have_precompute_mult
Module: U:\extras\lib\libcrypto.lib(ecp_nist.obj)
0001:00131a80  _EC_GFp_nist_method
0001:00131a8a* _ec_GFp_nist_group_copy
0001:00131ac1* _ec_GFp_nist_group_set_curve
0001:00131c61* _ec_GFp_nist_field_mul
0001:00131d4c* _ec_GFp_nist_field_sqr
Module: U:\extras\lib\libcrypto.lib(ecp_mont.obj)
0001:00131ed0  _EC_GFp_mont_method
0001:00131eda* _ec_GFp_mont_group_init
0001:00131f0d* _ec_GFp_mont_group_finish
0001:00131f76* _ec_GFp_mont_group_clear_finish
0001:00131fdf* _ec_GFp_mont_group_copy
0001:0013212d* _ec_GFp_mont_group_set_curve
0001:00132336* _ec_GFp_mont_field_mul
0001:001323ab* _ec_GFp_mont_field_sqr
0001:00132420* _ec_GFp_mont_field_encode
0001:0013249e* _ec_GFp_mont_field_decode
0001:0013250c* _ec_GFp_mont_field_set_to_one
Module: U:\extras\lib\libcrypto.lib(ech_ossl.obj)
0001:00132634  _ECDH_OpenSSL
Module: U:\extras\lib\libcrypto.lib(tb_ecdh.obj)
0001:00132ad4* _ENGINE_unregister_ECDH
0001:00132b03* _ENGINE_register_ECDH
0001:00132b4f* _ENGINE_register_all_ECDH
0001:00132b80* _ENGINE_set_default_ECDH
0001:00132bcc  _ENGINE_get_default_ECDH
0001:00132be9  _ENGINE_get_ECDH
0001:00132bf4* _ENGINE_set_ECDH
Module: U:\extras\lib\libcrypto.lib(dso_openssl.obj)
0001:00132c10  _DSO_METHOD_openssl
Module: U:\extras\lib\libcrypto.lib(ui_openssl.obj)
0001:00132c3f  _UI_OpenSSL
Module: U:\extras\lib\libcrypto.lib(asn_pack.obj)
0001:001333bb* _ASN1_seq_unpack
0001:00133439* _ASN1_seq_pack
0001:0013355f* _ASN1_unpack_string
0001:001335c4* _ASN1_pack_string
0001:00133703  _ASN1_item_pack
0001:00133835  _ASN1_item_unpack
Module: U:\extras\lib\libcrypto.lib(p12_utl.obj)
0001:001338ba  _OPENSSL_asc2uni
0001:00133973* _OPENSSL_uni2asc
0001:00133a03* _i2d_PKCS12_bio
0001:00133a25* _i2d_PKCS12_fp
0001:00133a47* _d2i_PKCS12_bio
0001:00133a69* _d2i_PKCS12_fp
0001:00133a8b* _PKCS12_x5092certbag
0001:00133ab6* _PKCS12_x509crl2certbag
0001:00133ae1* _PKCS12_certbag2x509
0001:00133b3b* _PKCS12_certbag2x509crl
Module: U:\extras\lib\libcrypto.lib(cms_io.obj)
0001:00133ba9  _CMS_stream
0001:00133c56* _d2i_CMS_bio
0001:00133c78* _i2d_CMS_bio
0001:00133c9e* _PEM_read_bio_CMS
0001:00133cd7* _PEM_read_CMS
0001:00133d10* _PEM_write_bio_CMS
0001:00133d63* _PEM_write_CMS
0001:00133db6* _BIO_new_CMS
0001:00133dd8* _i2d_CMS_bio_stream
0001:00133e08* _PEM_write_bio_CMS_stream
0001:00133e40* _SMIME_write_CMS
0001:00133ec6* _SMIME_read_CMS
Module: U:\extras\lib\libcrypto.lib(cms_dd.obj)
0001:00133ef0* _cms_DigestedData_create
0001:00133f8f  _cms_DigestedData_init_bio
0001:00133fb7  _cms_DigestedData_do_final
Module: U:\extras\lib\libcrypto.lib(ecp_smpl.obj)
0001:00134110* _EC_GFp_simple_method
0001:0013411a  _ec_GFp_simple_group_init
0001:00134160  _ec_GFp_simple_group_finish
0001:00134194  _ec_GFp_simple_group_clear_finish
0001:001341c8  _ec_GFp_simple_group_copy
0001:00134260  _ec_GFp_simple_group_set_curve
0001:001344c8  _ec_GFp_simple_group_get_curve
0001:00134625  _ec_GFp_simple_group_get_degree
0001:0013463b  _ec_GFp_simple_group_check_discriminant
0001:00134916  _ec_GFp_simple_point_init
0001:00134957  _ec_GFp_simple_point_finish
0001:00134989  _ec_GFp_simple_point_clear_finish
0001:001349c5  _ec_GFp_simple_point_copy
0001:00134a47  _ec_GFp_simple_point_set_to_infinity
0001:00134a74  _ec_GFp_simple_set_Jprojective_coordinates_GFp
0001:00134cc4  _ec_GFp_simple_get_Jprojective_coordinates_GFp
0001:00134e45  _ec_GFp_simple_point_set_affine_coordinates
0001:00134ebc  _ec_GFp_simple_point_get_affine_coordinates
0001:001352ea  _ec_GFp_simple_set_compressed_coordinates
0001:00135900  _ec_GFp_simple_point2oct
0001:00135d02  _ec_GFp_simple_oct2point
0001:00136140  _ec_GFp_simple_add
0001:0013693e  _ec_GFp_simple_dbl
0001:00136fe6  _ec_GFp_simple_invert
0001:00137037  _ec_GFp_simple_is_at_infinity
0001:0013704a  _ec_GFp_simple_is_on_curve
0001:00137492  _ec_GFp_simple_cmp
0001:0013783c  _ec_GFp_simple_make_affine
0001:0013798e  _ec_GFp_simple_points_make_affine
0001:00138081* _ec_GFp_simple_field_mul
0001:001380b3* _ec_GFp_simple_field_sqr
Module: U:\extras\lib\libcrypto.lib(bn_nist.obj)
0001:00138624  _BN_get0_nist_prime_192
0001:0013862e  _BN_get0_nist_prime_224
0001:00138638  _BN_get0_nist_prime_256
0001:00138642  _BN_get0_nist_prime_384
0001:0013864c  _BN_get0_nist_prime_521
0001:001386eb  _BN_nist_mod_192
0001:001389fd  _BN_nist_mod_224
0001:00138e30  _BN_nist_mod_256
0001:001393ce  _BN_nist_mod_384
0001:00139a79  _BN_nist_mod_521
Module: U:\extras\lib\libcrypto.lib(dso_null.obj)
0001:00139ddb  _DSO_METHOD_null
Module: U:\extras\lib\libcrypto.lib(a_set.obj)
0001:00139e5c  _i2d_ASN1_SET
0001:0013a187  _d2i_ASN1_SET
Module: U:\extras\lib\libcrypto.lib(p12_asn.obj)
0001:0013a5e0* _PKCS12_MAC_DATA_it
0001:0013a4e0  _PKCS12_it
0001:0013a4fc* _d2i_PKCS12
0001:0013a525* _i2d_PKCS12
0001:0013a547* _PKCS12_new
0001:0013a55b* _PKCS12_free
0001:0013a5fc* _d2i_PKCS12_MAC_DATA
0001:0013a625* _i2d_PKCS12_MAC_DATA
0001:0013a647* _PKCS12_MAC_DATA_new
0001:0013a65b* _PKCS12_MAC_DATA_free
0001:0013a780* _PKCS12_BAGS_it
0001:0013a79c* _d2i_PKCS12_BAGS
0001:0013a7c5* _i2d_PKCS12_BAGS
0001:0013a7e7  _PKCS12_BAGS_new
0001:0013a7fb* _PKCS12_BAGS_free
0001:0013a980* _PKCS12_SAFEBAG_it
0001:0013a99c* _d2i_PKCS12_SAFEBAG
0001:0013a9c5* _i2d_PKCS12_SAFEBAG
0001:0013a9e7  _PKCS12_SAFEBAG_new
0001:0013a9fb* _PKCS12_SAFEBAG_free
0001:0013aa50  _PKCS12_SAFEBAGS_it
0001:0013aaa0  _PKCS12_AUTHSAFES_it
Module: U:\extras\lib\libcrypto.lib(p12_add.obj)
0001:0013aaca  _PKCS12_item_pack_safebag
0001:0013abd6* _PKCS12_MAKE_KEYBAG
0001:0013ac3c* _PKCS12_MAKE_SHKEYBAG
0001:0013ad3e* _PKCS12_pack_p7data
0001:0013ae42* _PKCS12_unpack_p7data
0001:0013aea6* _PKCS12_pack_p7encdata
0001:0013b094* _PKCS12_unpack_p7encdata
0001:0013b0f8* _PKCS12_decrypt_skey
0001:0013b11c* _PKCS12_pack_authsafes
0001:0013b154* _PKCS12_unpack_authsafes
Module: U:\extras\lib\libcrypto.lib(bio_ndef.obj)
0001:0013b1cb  _BIO_new_NDEF
Module: U:\extras\lib\libcrypto.lib(asn_mime.obj)
0001:0013b6bd  _i2d_ASN1_bio_stream
0001:0013ca26* _SMIME_crlf_copy
0001:0013b8a2  _PEM_write_bio_ASN1_stream
0001:0013be7d  _SMIME_write_ASN1
0001:0013c4a6  _SMIME_read_ASN1
0001:0013cbae* _SMIME_text
Module: U:\extras\lib\libcrypto.lib(bn_sqrt.obj)
0001:0013d7fa  _BN_mod_sqrt
Module: U:\extras\lib\libcrypto.lib(bn_kron.obj)
0001:0013e360  _BN_kronecker
Module: U:\extras\lib\libcrypto.lib(bio_asn1.obj)
0001:0013e6e5  _BIO_f_asn1
0001:0013f02b  _BIO_asn1_set_prefix
0001:0013f054* _BIO_asn1_get_prefix
0001:0013f07d  _BIO_asn1_set_suffix
0001:0013f0a6* _BIO_asn1_get_suffix
Module: U:\extras\lib\libcrypto.lib(bio_b64.obj)
0001:0013f0e0  _BIO_f_base64


                        +----------------------+
                        |   Imported Symbols   |
                        +----------------------+

Symbol                              Module
======                              ======

___libc_ForkRegisterModule          libc064
___init_dll                         libc064
___libc_Back_termDll                libc064
___libc_ForkDeregisterModule        libc064
__atfork_callback                   libc064
_PyString_FromString                python27
_PyInt_FromLong                     python27
_PyExc_TypeError                    python27
_PyErr_Format                       python27
_PyErr_SetString                    python27
_PyArg_ParseTuple                   python27
__Py_NoneStruct                     python27
_Py_FindMethod                      python27
_PyEval_SaveThread                  python27
_PyEval_RestoreThread               python27
_PyOS_snprintf                      python27
_Py_BuildValue                      python27
_PyErr_SetObject                    python27
_PyTuple_New                        python27
_PyString_FromStringAndSize         python27
_PyString_AsString                  python27
_PyErr_CheckSignals                 python27
__PyString_Resize                   python27
_PyBuffer_Release                   python27
_PyObject_Free                      python27
_PyType_Type                        python27
_Py_InitModule4                     python27
_PyModule_GetDict                   python27
_PyCapsule_Import                   python27
_PyErr_NewException                 python27
_PyDict_SetItemString               python27
_PyThread_allocate_lock             python27
_PyThread_free_lock                 python27
_PyModule_AddIntConstant            python27
_PyLong_FromUnsignedLong            python27
_PyModule_AddObject                 python27
_PyThread_get_thread_ident          python27
_PyThread_release_lock              python27
_PyThread_acquire_lock              python27
__PyObject_New                      python27
_PyUnicodeUCS2_DecodeUTF8           python27
_PyList_New                         python27
_PyList_Append                      python27
_PyList_AsTuple                     python27
_PyList_Size                        python27
_PyDict_New                         python27
_PyObject_IsTrue                    python27
__CRT_init                          libc064
__CRT_term                          libc064
__errno                             libc064
__std_select                        libc064
___stderrp                          libc064
__std_malloc                        libc064
__std_memset                        libc064
__std_free                          libc064
___libc_GLocaleCtype                libc064
__std_strchr                        libc064
___ctordtorTerm1                    libc064
___ctordtorInit1                    libc064
__std_strlen                        libc064
__libsocket_socket                  tcpip32
___libc_TcpipAllocFH44              libc064
__libsocket_soclose                 tcpip32
__libsocket_set_errno               tcpip32
__libsocket_sock_errno              tcpip32
___libc_FH                          libc064
__libsocket_connect                 tcpip32
__std_write                         libc064
__std_read                          libc064
__std_close                         libc064
__std_memcpy                        libc064
__std_strcpy                        libc064
__std_memcmp                        libc064
__std_strstr                        libc064
__std_time                          libc064
__std_strerror                      libc064
__std_strncpy                       libc064
__std_strncmp                       libc064
__std_getpid                        libc064
__std_vfprintf                      libc064
__std_abort                         libc064
__std_strcmp                        libc064
__std_fwrite                        libc064
__std_realloc                       libc064
__std_memmove                       libc064
__std_qsort                         libc064
__std_strcat                        libc064
__std_fopen                         libc064
__std_fclose                        libc064
__std_fread                         libc064
__std_ferror                        libc064
__std_fseek                         libc064
__std_feof                          libc064
__std_ftell                         libc064
__std_fileno                        libc064
__std_setmode                       libc064
__std_fflush                        libc064
__std_fgets                         libc064
___deregister_frame                 gcc446
___register_frame_table             gcc446
DosTmrQueryTime                     doscalls
DosQuerySysInfo                     doscalls
DosEnterCritSec                     doscalls
DosPerfSysCall                      doscalls
DosExitCritSec                      doscalls
DosAllocMem                         doscalls
DosQuerySysState                    doscalls
DosFreeMem                          doscalls
__libsocket_shutdown                tcpip32
__std_localtime                     libc064
__std_strnicmp                      libc064
__std_stricmp                       libc064
__std_fprintf                       libc064
__std_memchr                        libc064
__std_strtoul                       libc064
__std_sscanf                        libc064
__std_getenv                        libc064
__std_atoi                          libc064
__std_random                        libc064
__std_stat                          libc064
__std_strrchr                       libc064
__std_strtol                        libc064
__std_gmtime                        libc064
___stdinp                           libc064
__std_fputs                         libc064
__std_fputc                         libc064
__std_tcgetattr                     libc064
__std_tcsetattr                     libc064
__std_sigaction                     libc064


                        +--------------------+
                        |   Libraries Used   |
                        +--------------------+

U:\extras\lib\libssl.lib
U:\extras\lib\libcrypto.lib
U:\tmp\ldconv_python2_7_dll_a_ddb24f08029a19bc30.lib
U:\usr\local446\lib\gcc\i386-pc-os2-emx\4.4.6\libgcc.lib
U:\tmp\ldconv_libgcc_so_d_a_ddb24f08029a1a0e38.lib
U:\usr\lib\libc_alias.lib
U:\usr\local446\lib\libc_dll.lib
U:\usr\lib\libos2.lib
U:\usr\lib\libend.lib


                        +-----------------------+
                        |   Linker Statistics   |
                        +-----------------------+

Stack size:  0000 (0.)
Memory size:  00149e90 (1351312.)
Link time: 00:00.30
